:020000040800F2
:1080000008C60020A1810008C1520108C94B01081F
:10801000BF520108F5190108CD62010800000000F7
:1080200000000000000000000000000015820008B1
:108030000B1C010800000000718200088D59010826
:10804000BB810008BB810008BB810008BB81000820
:10805000BB810008BB810008BB810008BB81000810
:10806000BB810008BB810008BB810008911B01088F
:10807000BB810008BB810008BB810008BB810008F0
:10808000BB810008BB810008BB810008BB810008E0
:10809000BB810008BB810008BB810008BB810008D0
:1080A000BB810008255D0108BB810008BB81000879
:1080B000BB8100080000000000000000BB81000838
:1080C000BB8100080000000000000000BB81000828
:1080D00000000000896201089562010800000000AC
:1080E000BB810008BB810008000000000000000008
:1080F0000000000000000000000000000000000080
:10810000000000000000000000000000BB8100082B
:108110000000000000000000BB810008BB810008D7
:10812000BB810008BB810008BB810008BB8100083F
:10813000BB810008000000000000000000000000FB
:10814000BB810008BB810008BB810008BB8100081F
:10815000BB810008BB810008BB810008BB8100080F
:10816000BB810008BB810008BB8100080000000043
:10817000BB810008BB810008000000000000000077
:10818000BB810008BB810008BB810008DFF80CD070
:1081900008F060FE004800475984010808C6002026
:1081A0000648804706480047FEE7FEE7FEE7FEE791
:1081B000FEE7FEE7FEE7FEE7FEE7FEE7E15C01081B
:1081C0008D81000810B51C46029B9B1AA34205D363
:1081D0001044224608F0FEF8204610BD002010BDD5
:1081E000421C10F8011B0029FBD1801A704796230E
:1081F0000022114608F073BD0048704774C301089F
:1082000054656D636F504944393000000000003000
:10821000000000002C4B1968086800F05AB880F381
:108220000988BFF36F8F4FF0000080F3118870470B
:108230000000000008480068006880F308884FF0DC
:10824000000080F3148862B661B6BFF34F8FBFF3AE
:108250006F8F00DF00BF00BF08ED00E0DFF80C000B
:10826000016841F470010160704700BF88ED00E0D3
:10827000EFF30980BFF36F8F134B1A681EF0100FD6
:1082800008BF20ED108A20E9F04F106009B44FF0CC
:10829000500080F31188BFF34F8FBFF36F8F13F03F
:1082A0009BF84FF0000080F3118809BC196808683A
:1082B00000F014B81EF0100F08BF00F014B880F3DF
:1082C0000988BFF36F8F704720020020EFF305800D
:1082D000704730C8B0E8C04FFFF7A1BF30C8B0E862
:1082E000C04FFFF7E7BFB0EC088AB0EC08CAFFF751
:1082F000E6BF0000002801D0CE4B036011B1CD488D
:1083000008380860002A02D0CA48001F1060704771
:10831000412801D20120704700207047C6480078EC
:108320007047401C7047401E70472DE9F0410646DB
:108330000C463046FFF7F7FF00256F1E7CB1552134
:108340002180676025720421A172C2B20021012040
:1083500009F06AFD206184F87052D4F87442DCB1EF
:108360006F202080676025720820A07204F1100041
:10837000074602F017FB00221146384602F01BFBAD
:1083800000220121384602F016FB00220221384665
:1083900002F011FB84F870523046BDE8F04109F05C
:1083A00021BB10B502460C4600211046FFF7BBFF6B
:1083B000402A08D2C1B201200FF048FC01462046F5
:1083C00002F0B9FB0146084610BD2DE9F043ADF5BA
:1083D0001B7D814608469846A39DA29CFFF7A3FFFC
:1083E0000227FE1E4F2A42D008DC1C2A32D0242A43
:1083F00068D04B2A1BD04D2A08D11EE0512A66D0E6
:10840000552A39D06F2A41D0752A6CD02770202088
:1084100028703046002806DBB8F1FF3F03D02770F4
:108420003220287030460DF51B7DBDE8F0830246F2
:108430000021484601F01AFFECE7C1B201200FF01D
:1084400005FC014601A802F076FB01A9484601F0AF
:10845000CAFFDFE7C1B201200FF08CFB014601A883
:1084600002F069FB01A9484601F0BDFFD2E70021F7
:10847000484602F0BEF8CDE7C2B20021012009F063
:10848000D3FC0146484602F061F9C3E797A802F021
:1084900089FA0022114697A802F08DFA00220121E4
:1084A00097A802F088FA0022022197A802F083FA26
:1084B0000022032197A802F07EFA97A9484601F00E
:1084C00061FEA7E70021484602F093F8A2E7C1B297
:1084D000012009F077FC08B1012100E000214846A5
:1084E00001F07FFD96E7C1B201200FF0C2FB01460B
:1084F000484602F07EF88DE770B5ADF51A7D04466A
:1085000000256A4604F11000D4F8681204F027FC34
:108510000222002808DA84F86D22252084F86E02F1
:1085200000200DF51A7D70BD2089822809D0E068F1
:10853000401C06D084F86D22322084F86E020020A0
:10854000EFE76068FFF7EFFE014620890926512812
:108550005FD008DC0DF10D031C2849D024280AD077
:108560004D2808D133E055280CD0672803D06F2858
:1085700001D0752818D084F86D22202084F86E026E
:108580002846CEE79DF80200042804D084F86D2226
:1085900084F86E62F4E7CAB294F86C120120029B70
:1085A00012F096FF0125EBE79DF80200092804D0A0
:1085B00084F86D2284F86E62E2E70298CAB2C3B210
:1085C00094F86C12012012F088FF0125D8E79DF87D
:1085D0000200072804D084F86D2284F86E62CFE789
:1085E000CAB294F86C12012012F076FF0125C7E799
:1085F0009DF80200072804D084F86D2284F86E628A
:10860000BEE7CAB294F86C12012012F064FF012593
:10861000B6E79DF80200012804D084F86D2284F8A2
:108620006E62ADE79DF80820C9B2012012F051FF3B
:108630000125A5E7B8BF0108C4020020002801D029
:10864000FB4B036011B1FA4808380860002A02D0D9
:10865000F748001F10607047412801D20120704781
:1086600000207047F34800787047401C7047401E58
:1086700070472DE9F04105460024E9B2022009F0D7
:10868000A9FB0746402D11D2EB4EEAB2E1B202201F
:1086900009F0CAFBB04206D0EAB2E1B2022009F00A
:1086A000C3FB074602E0641C102CEED33846BDE83D
:1086B000F0812DE9F041054600240026402D0CD222
:1086C000DD4FEAB2E1B2022009F0AEFBB84201D0C0
:1086D000661C02E0641C102CF3D33046E7E710B5AB
:1086E0000B46002140280CD25AB1102A09D8062A7C
:1086F00007D0521EC0B2D1B20246022012F0E8FEEC
:108700000121084610BD10B5002240280CD259B1F5
:10871000102909D8062907D0C2B2491EC9B2C64BD2
:10872000022012F0D5FE0122104610BD10B50246FF
:108730000C4600211046FFF79AFF402A08D2C1B22A
:1087400002200FF083FA0146204602F0F4F90146B8
:10875000084610BD2DE9FF4FADF51B7D8246DDF8C3
:10876000A492DDF8A08208461F4600240026FFF7E9
:108770007EFF05469D984FF0FF3B51287ED00CDCD4
:108780004B2830D004DC1C2842D0242811D17DE0B5
:108790004D282FD04F280CD148E068286FD004DC3A
:1087A000552849D0572804D18DE06F284DD0752821
:1087B0007FD0022088F80000202089F800005C4665
:1087C000002C0BDB9D98572808D07F1C06D0022078
:1087D00088F80000322089F800005C460DF51F7D06
:1087E000204600F0B5B92A460121504601F03EFD71
:1087F0000446E5E7E9B202200FF028FA014601A895
:1088000002F099F901A9504601F0EDFD0446D7E7C1
:10881000E9B202200FF0AEF9014601A802F08BF98F
:1088200001A9504601F0DFFD0446C9E70121504689
:1088300001F0DFFE0446C3E72846FFF71AFF0146B2
:10884000504601F083FF0446BAE797A802F0AAF861
:108850000022114697A802F0AEF80022012197A845
:1088600002F0A9F80022022197A802F0A4F8002241
:10887000032197A802F09FF897A902E00CE074E0AA
:1088800017E0504601F07EFC044699E7002150466F
:1088900001F0AFFE044693E7E9B2022009F092FA34
:1088A00008B1012100E00021504601F09AFB044686
:1088B00086E7E9B202200FF0DCF90146504601F0EC
:1088C00098FE04467CE787B1781C14D0102F44D85A
:1088D000EAB20021022009F0A7FA5749884231D1B3
:1088E000504601F0B7FB04466AE71021504601F0FC
:1088F0004EFE044664E7EAB2F1B2022009F094FAAF
:108900004D49884204D10AEB040001F0A3FB09E0C1
:10891000EAB2F1B2022009F087FA01460AEB04003C
:1089200001F014FF0444B4F5167F03DA761C102E10
:10893000E1D345E7052088F80000122089F80000FF
:108940005C463DE7EAB20021022009F06DFA0146DB
:10895000504601F0FBFE044632E7022088F8000092
:108960002A2089F800005C462AE7E9B2022009F0D3
:1089700031FA0146504601F0E9FE044620E72DE9B0
:10898000F043ADF51B7D044600256A4604F1100056
:10899000D4F8681204F0E3F902274FF02508002804
:1089A00008DA84F86D7284F86E8200200DF51B7D64
:1089B000BDE8F0832089572809D0E068401C06D024
:1089C00084F86D72322084F86E020020EEE7606851
:1089D000FFF74DFE0646208904F26E235A1E092138
:1089E0004FF02809512858D00EDC0DF10D034B280B
:1089F00004D004DC1C286FD0242811D1A3E04D281A
:108A000059D04F280CD19EE068286FD004DC55283F
:108A100014D0572804D196E06F2868D075285CD010
:108A200084F86D72202084F86E022846BEE70000AC
:108A3000E4BF0108C502002000007F439DF802004A
:108A4000042813D00021684604F00EFF05462800D4
:108A5000EBD094F86C123046FFF755FE054628001F
:108A6000E3D184F86D7284F86E82DEE794F86C22AC
:108A700030460299FFF733FE054694F86C0206284B
:108A800006D0002DD1D184F86D7284F86E82CCE7C7
:108A900084F86D7284F86E92C7E70121684604F08D
:108AA000E3FE05462800C0D09DF80820F1B2022060
:108AB00012F00FFDB9E79DF80200072804D084F8F2
:108AC0006D7284F86E12B0E7F2B294F86C12022064
:108AD00012F002FD0125A8E714E09DF80200092824
:108AE00006D084F86D7284F86E129EE71BE02AE0CF
:108AF0000298F2B2C3B294F86C12022012F0EDFCAC
:108B0000012592E79DF80200072804D084F86D72D1
:108B100084F86E1289E7F2B294F86C12022012F017
:108B2000DAFC012581E79DF80200042804D084F8CE
:108B30006D7284F86E1278E7F1B20220029A12F098
:108B4000C9FC012571E784F86D7284F86E926CE7B8
:108B500030BCBDE8C08F0000002801D0F74B036097
:108B600011B1F64808380860002A02D0F348001F07
:108B700010607047401E704710B502460C46002139
:108B80001046FFF7F7FF802A08D2C1B200200FF08D
:108B90005DF80146204601F0CEFF0146084610BDB3
:108BA000812801D20120704700207047E4480078F6
:108BB0007047401C70472DE9F0410546002700240E
:108BC000802D11D2DF4EEAB2E1B2002009F02CF97B
:108BD000B04206D0EAB2E1B2002009F025F907461A
:108BE00002E0641C102CEED33846BDE8F0812DE97C
:108BF000F041054600240026802D0CD2D14FEAB268
:108C0000E1B2002009F010F9B84201D0661C02E080
:108C1000641C102CF3D33046E7E770B504460D46CC
:108C200010460022802C11D280B110280ED80628C0
:108C30000CD0FFF7DCFA0646284607F0E7FEC1B283
:108C4000E2B23346002012F043FC0122104670BD10
:108C500010B5002280280BD251B1102908D806295E
:108C600006D0C2B2C9B2B74B002012F031FC0122CB
:108C7000104610BD2DE9F04FADF51B7D8246DDF8A5
:108C80009492DDF8908208461F4600240026FFF7E4
:108C900071FF05464FF0FF3B512A7CD00CDC4B2A7C
:108CA0002DD004DC1C2A3FD0242A11D179E04D2A92
:108CB0002CD04F2A0CD145E0682A6DD004DC552A0F
:108CC00046D0572A04D18AE06F2A4AD0752A7CD030
:108CD000022088F80000202089F800005C46002C63
:108CE00008DB7F1C06D0022088F80000322089F8BB
:108CF00000005C460DF51B7D204600F0C5B92A46F4
:108D00000221504601F0B2FA0446E8E7E9B2002039
:108D10000EF09CFF014601A801F00DFF01A950468D
:108D200001F061FB0446DAE7E9B200200EF022FF11
:108D3000014601A801F0FFFE01A9504601F053FBD6
:108D40000446CCE70221504601F053FC0446C6E736
:108D50002846FFF730FF0146504601F0F7FC044675
:108D6000BDE797A801F01EFE0022114697A801F06A
:108D700022FE0022012197A801F01DFE00220221FF
:108D800097A801F018FE0022032197A801F013FE16
:108D900097A9504601E00BE073E001F0F3F90446B7
:108DA0009DE70021504601F024FC044697E70CE0C3
:108DB000E9B2002009F006F808B1012100E0002125
:108DC000504601F00EF9044689E7E9B200200EF0A2
:108DD00050FF0146504601F00CFC04467FE787B186
:108DE000781C14D0102F44D80021EAB2084609F0AC
:108DF0001BF85449884231D1504601F02BF9044602
:108E00006DE71021504601F0C2FB044667E7EAB265
:108E1000F1B2002009F008F84A49884204D10AEB6F
:108E2000040001F017F909E0EAB2F1B2002008F0FD
:108E3000FBFF01460AEB040001F088FC0444B4F592
:108E4000167F03DA761C102EE1D348E7052088F858
:108E50000000122089F800005C4640E70021EAB2D9
:108E6000084608F0E1FF0146504601F06FFC044659
:108E700035E7022088F800002A2089F800005C46C7
:108E80002DE70021504601F061FC044627E72DE95B
:108E9000F043ADF51B7D04460E4617464FF0000823
:108EA0006068FFF767FE05462846FFF779FE4FF03A
:108EB000010988B16A4604F11000D4F8681203F081
:108EC0004EFF022100280DDA317025203870002075
:108ED0000DF51B7DBDE8F08386F800901F203870EB
:108EE0000020F5E72089572807D0E268521C04D0FB
:108EF0003170322038700020EAE7092251286CD006
:108F00000EDC0DF10D034B2879D004DC1C283ED07B
:108F100024280DD173E04D2827D04F2808D16EE0CA
:108F2000552811D057286AD06F2868D0752840D0AE
:108F30003170202038704046CAE7000018C0010890
:108F4000C602002000007F439DF80200042802D0E2
:108F500031703A70EFE74A49029841F825004948D4
:108F600000F805904FF00108E5E79DF8020007289A
:108F700004D084F86D1284F86E22DCE7EAB294F82B
:108F80006C12002012F0A8FA4FF00108D3E79DF808
:108F90000200072804D084F86D1284F86E22CAE714
:108FA000EAB294F86C12002012F095FA4FF0010822
:108FB000C1E79DF80200092804D084F86D1284F8F6
:108FC0006E22B8E70298EAB2C3B294F86C1200209D
:108FD00012F083FA4FF00108ADE79DF8020009286E
:108FE00004D084F86D1284F86E22A4E79DF808205E
:108FF000E9B2002012F06DFA4FF001089BE73170E2
:109000002820387097E72DE9F04106460C46304697
:10901000FFF7B0FD00256F1E7CB1552121806760F0
:1090200025720421A172C2B20021084608F0FCFE9C
:10903000206184F87052D4F87442DCB16F20208033
:10904000676025720820A07204F11000074601F045
:10905000A9FC00221146384601F0ADFC0022012196
:10906000384601F0A8FC00220221384601F0A3FC9A
:1090700084F870523046BDE8F04108F0B5BC0000FD
:10908000E88600203887002030BCBDE8C08F000093
:1090900030B5002203780C78A34201D0002030BD07
:1090A000072B0BD9072309E084188D1864786D7895
:1090B000AC4201D0002030BD521CD2B29A42F3D350
:1090C00002890B899A4201D0002030BD2AB1837AEF
:1090D0008A7A934203D0002030BD012030BD072B97
:1090E00000D90723002209E084188D18E47AED7A6C
:1090F000AC4201D0002030BD521CD2B29A42F3D310
:10910000012030BDFD49FE4A09E00B78DB0705D0A0
:109110004B68834202D1002008707047243191428D
:10912000F3D9704770B50020821EF449F44C0AE070
:109130000B7803F00703012B04D10B6A934201D88B
:109140001A4608462431A142F2D980254FF46166BF
:1091500010B10570066270BDE8490AE00B7803F0B3
:109160000703032B04D10B6A934201D81A46084621
:109170002431A142F2D90028EDD00570066270BDFD
:1091800042F2DC31DD4807F03EB910B5DB48002281
:10919000DB4B0CE00178CC0704D0890701D4016ACD
:1091A00001B902700178090600D502702430984296
:1091B000F0D910BD30B5D14BD14C18E01D78ED077A
:1091C00014D05D68854211D1187884070CD432B16F
:1091D00040F0040018704FF0FF30186230BD20F0EE
:1091E00004001870196230BD196230BD2433A342E7
:1091F000E4D930BD70B50D4616460022BF4CC049BB
:1092000013E02378DB070FD0636883420CD120780A
:1092100080070CD4122204F10C01304607F0DAF872
:10922000A0682860012202E024348C42E9D910466B
:1092300070BD2DE9F04180460E460027AF4CB04D81
:1092400010E0207800F0030001280AD1414604F123
:109250000C0003F07FFC20B10EB160683060012784
:1092600002E02434AC42ECD93846BDE8F0812DE967
:10927000F04706460F4691460020A04C4FF4616827
:109280009F4D24E02178C90720D06168B1421DD1EB
:109290001222494604F10C0007F09CF8A7602078E0
:1092A0009849820701D521620BE0420703D54FF0B0
:1092B000FF31216205E0020702D5C4F8208000E0FA
:1092C000216220F002002070012002E02434AC4230
:1092D000D8D94FF0010A38B9884C03E02178C90782
:1092E00017D02434AC42F9D9002810D1FFF71AFF67
:1092F0000446002C0BD084F800A06660A760122200
:10930000494604F10C0007F065F8C4F82080BDE878
:10931000F08784F800A06660A7601222494604F135
:109320000C0007F057F8C4F820800120DCE72DE995
:10933000F04105460F4610460026704C70491BE070
:109340002278D20717D06268AA4214D121788907FF
:109350000FD40126122204F10C0107F03BF8A0689B
:1093600038602078010704D520F008002070654897
:109370002062304679E724348C42E1D95F480324E7
:109380004FF4616604E0027812F0810F0AD02430B5
:109390008842F8D9FFF7C6FE10B104704560066236
:1093A000002062E704704560066200205DE770B54A
:1093B0000D461646514C524916E02378DA0712D072
:1093C000636883420FD11222314604F10C0007F08A
:1093D00001F8A560207820F002002070400701D439
:1093E0004848206270BD24348C42E6D970BD70B507
:1093F00004460D4616460020FF2C14D23F4A04EBCB
:10940000C40102EB8104217801F0030101290AD192
:10941000122204F10C01184606F0DCFF6068286097
:10942000A0683060012070BD00203449344A06E055
:109430000B7803F00303012B00D1401C243191422F
:10944000F6D97047F0B5ADF5177D064600252B4CD3
:109450002B4F28E0207800F00300012822D170195A
:109460000821626800F002FF0544A18A701901F02A
:109470008EF80544A27D52B104F1170101A801F054
:10948000B8FC701901A900F016FF05440AE0227B20
:1094900004F10D0101A801F0ACFC701901A900F064
:1094A0000AFF05442434BC42D4D90DF5177D284663
:1094B000F0BD2DE9F04FADF5197D81460D46002731
:1094C000B84605F11800989001F06CFA0022114698
:1094D000989801F070FA00220121989801F06BFA37
:1094E00000220221989801F066FAE86AC0F5167B1E
:1094F00000202863FFF798FF824605E0848C002057
:109500003CB00020805101005FEA0A0004D0A86A44
:109510000123082805D007E000200DF5197D00F093
:10952000A7B8C5F844A0AB63686C00280ADAAA6B38
:10953000511C0144012902DA6A64AB6302E0A963A9
:1095400040426864A86B504501D90020E5E7696C8A
:109550000144491E00910099514501D9CDF800A060
:10956000414C012600E02434217801F00301012957
:10957000F9D105E0217801F00301012904D0243458
:10958000B042F7D1019645E02434761CF8E7BBF1F0
:10959000110F05D201220221989801F00CFA3CE04B
:1095A00009EB07000821626800F060FE804607EBC7
:1095B0000800A18A484400F0EAFF8044A27D62B11D
:1095C00004F1170102A801F014FC07EB080048445D
:1095D00002A900F070FE40440CE0227B04F10D0172
:1095E00002A801F006FC07EB0800484402A900F0BD
:1095F00062FE4044ABEB000B0744B046761C2434BB
:10960000286B401C286300E02434207800F003001D
:109610000128F9D100988642B9D90198012804D1CE
:1096200001220021989801F0C6F9D04504D1012209
:109630001146989801F0BFF938466EE730B50A49EF
:1096400000230A4C0DE00A7812F0810F08D052076F
:1096500006D40A6A824202D3121A0A6200E00B7030
:109660002431A142EFD930BD848C00203CB00020D1
:1096700030BCBDE8C08F0000002801D0FB4B036068
:1096800011B1FA482C300860002A02D0F748001FB8
:1096900010607047412801D20120704700207047B8
:1096A000F34800787047401C7047401E70472DE912
:1096B000F0410024C5B22946042008F08BFB07F0D6
:1096C000A5F9C6B2402D13D2EA4FE1B22A460420D2
:1096D00008F0AAFBB84208D0E1B22A46042008F0FC
:1096E000A3FB07F093F9C6B202E0641C102CECD384
:1096F0003046BDE8F08110B502460C460021104608
:10970000FFF7D3FF402A08D2C1B204200EF09EFA20
:109710000146204601F00FFA0146084610BD2DE92A
:10972000FF4FADF51B7D0746DDF8A4A2DDF8A09242
:109730000846984600240026FFF7B7FF05469D9887
:109740004FF0FF3B51287DD010DC2E287BD006DC6B
:10975000042879D01C2847D0242815D185E04B282F
:109760002DD04D2832D04F280ED14BE068286CD038
:1097700006DC54286AD055284AD0572804D190E0F6
:109780006F284ED075286FD0022089F80000202065
:109790008AF800005C46002C0CDB9D98572809D005
:1097A000B8F1FF3F06D0022089F8000032208AF885
:1097B00000005C460DF51F7D204600F025BA2A46C4
:1097C0000421384600F052FD0446E4E7E9B20420E3
:1097D0000EF03CFA014601A801F0ADF901A93846A6
:1097E00000F001FE0446D6E7E9B204200EF0C2F90B
:1097F000014601A801F09FF901A9384600F0F3FDE8
:109800000446C8E70421384600F0F3FE0446C2E7E8
:109810002846FFF74CFF0146384600F0EAFE0446B2
:10982000B9E797A801F0BEF80022114697A801F009
:10983000C2F80022012197A801F0BDF801220221FF
:1098400097A804E017E09DE092E085E020E001F0B9
:10985000B2F80122032197A801F0ADF897A9384684
:1098600000F090FC044696E796E00021384600F0B0
:10987000C0FE04468FE7E9B2042008F0A3FA08B15D
:10988000012100E00021384600F0ABFB044682E7EE
:10989000284608F0ABF80146384600F0AAFE044618
:1098A00079E7B8F1000F15D0B8F1FF3F18D0B8F143
:1098B000100F49D8A8F101000446C1B2EAB2042051
:1098C00008F0B2FA6B49884231D1384600F0C2FB49
:1098D000044660E71021384600F059FE04465AE776
:1098E000EAB2F1B2042008F09FFA6249884203D13B
:1098F000381900F0AFFB0AE0EAB2F1B2042008F038
:1099000093FA07F083F8C1B2381900F072FE0444EC
:10991000B4F5167F03DA761C102EE1D33BE7052061
:1099200089F8000012208AF800005C4633E7EAB2AA
:10993000E1B2042008F078FA07F068F8C1B23846BE
:1099400000F057FE044626E7022089F800002A208E
:109950008AF800005C461EE7E9B2042008F03AFAF3
:1099600007F054F8C1B2384600F043FE044612E74F
:1099700041A101A801F0DFF801A9384600F033FD4C
:10998000044608E73DA101A801F0D5F801A9384631
:1099900000F029FD0446FEE6E9B204200EF069F964
:1099A0000146384600F025FE0446F4E62DE9F04372
:1099B000ADF51B7D044600256A4604F11000D4F87D
:1099C000681203F0CCF902274FF02509002808DAC5
:1099D00084F86D7284F86E9200200DF51B7DBDE851
:1099E000F0832089572809D0E068401C06D084F80D
:1099F0006D72322084F86E020020EEE76068FFF797
:109A000054FE0646208904F26E2309215A1E4FF0A7
:109A1000280C512871D012DC0DF10D032E2806D030
:109A200006DC042803D01C2869D0242817D1E3E0E1
:109A30004B2803D04D286ED04F2810D1DCE067288A
:109A400006D006DC542867D0552819D0572806D1EF
:109A5000D2E068286FD06F286ED075286DD084F85A
:109A60006D72202084F86E022846B6E734C00108E3
:109A7000C702002000007F436F6E00006F66660023
:109A80009DF80200092813D00021684603F0ECFE7F
:109A900005462800E8D094F86C0278B3102834D832
:109AA000401EC1B2574BF2B2042011F011FDDBE7AA
:109AB00094F86C82B8F1000F17D0B8F1100F14D8D9
:109AC000B8F1060F11D0029801280ED80298C0B242
:109AD000A8F10108FEF78BFB0346F2B208F0FF0184
:109AE000042011F0F5FC0125BEE7B8F1060F07D000
:109AF00084F86D7284F86E92B6E70EE005E02EE011
:109B000084F86D7284F86EC2AEE7002584F86D7239
:109B100084F86E92A8E711E058E00121684603F04E
:109B2000A3FE054628009FD09DF80820F1B204202E
:109B300011F0CFFC98E736E05EE021E09DF80200EE
:109B4000072804D084F86D7284F86E128CE7F2B2A4
:109B500094F86C12042011F0BFFC012584E79DF8F5
:109B60000200072804D084F86D7284F86E127BE737
:109B7000F2B294F86C12042011F0ADFC012573E7E9
:109B80009DF80200092804D084F86D7284F86E12E2
:109B90006AE70298F2B2C3B294F86C12042011F092
:109BA0009CFC012560E79DF80200092804D084F898
:109BB0006D7284F86E1257E70298FEF718FB0246A2
:109BC000F1B2042011F086FC01254DE70921684619
:109BD00003F04AFE0546002D86D00298022805D2E1
:109BE0000298C1B2606807F003FF3DE7002584F8E2
:109BF0006D7284F86E9237E784F86D7284F86EC2E5
:109C000032E7000000007F4330BCBDE8C08F000099
:109C100002460020022A1ADB042A01DA102016E08C
:109C2000082A01DA202012E0102A01DA30200EE0A2
:109C3000202A01DA40200AE0402A02DA4FF05000E0
:109C400005E002D14FF0600001E04FF070003229D2
:109C500003DD802902DC40F001007047CE2902DCE0
:109C600040F002007047B1F5F07F02DC40F00300E5
:109C70007047B1F5806F02DC40F00400704740F29D
:109C8000C4529142FADC40F00500704701460020C2
:109C900001F0F0010911082906D2DFE801F00504FE
:109CA00006080A0C0E100220704704207047082096
:109CB0007047102070472020704740207047412097
:109CC00070470146002001F00F01062905D2DFE8A8
:109CD00001F0030507090C0F322070478020704700
:109CE000CE2070474FF4F07070474FF4806070479B
:109CF00040F2C450704770B50D4619460124002348
:109D00000370002A01D0082202700E2D04D80278B8
:109D100042EA0512027005E0027842F0F002027099
:109D200045700224042903D802780A4302701CE01B
:109D3000027842F005020270FD2903D82246641C15
:109D4000815412E0B1F5803F08D2FE22651C025515
:109D500089B2284403F050FB441906E0FF22651C39
:109D60000255284403F06CFB4419204670BD0122C3
:109D7000082303700E2903D843EA0111017003E0A0
:109D8000F822027041700222017841F00601017050
:109D9000104670470122082303700E2903D843EAB6
:109DA0000111017003E0F822027041700222017873
:109DB00041F0070101701046704710B503460120BD
:109DC0001A780F24B4EB121F04D109B15878087027
:109DD000022010BD0029FCD012090A7010BD10B578
:109DE0000346002000290AD018780F24B4EB101F76
:109DF00006D1022904D30AB158781070022010BD90
:109E00000AB100091070012010BD007800F00700B1
:109E1000062801D000207047012070470078C04319
:109E2000400701D000207047012070477CB50546EF
:109E300014462846FFF7C1FF2A7802F007010529DA
:109E400003D00023062920D022E0295CFF2905D079
:109E5000FE290ED004B12160401C7CBD461CA8190F
:109E6000694603F0F6FA3044002CF6D000992160E0
:109E70007CBD461CA81901A903F0C3FA3044002C8C
:109E8000F6D0BDF8041021607CBD0CB123607CBD10
:109E9000D243520702D10CB123607CBD002CFCD010
:109EA00021607CBDF8B505460E461C463146284665
:109EB000FFF795FF002818DD321A2B7803F0070111
:109EC000052903D00022062929D02BE0295CFF298F
:109ED0000CD1052A0AD3461CA819694603F0B9FA21
:109EE0003044002C01D000992160F8BDFE290DD12D
:109EF000032A0BD3461CA819694603F082FA3044A2
:109F0000002CF2D0BDF800102160F8BDFE2904D26B
:109F10001AB104B12160401CF8BD0020F8BD0CB19D
:109F20002260F8BDDB435B0702D10CB12260F8BDB3
:109F3000002CFCD02160F8BD38B504460D46002247
:109F4000009269462046FFF738FF2078000705D5C4
:109F50009DF80000A84201D1012038BD002038BD85
:109F600078B505460E4614460020009069462846FE
:109F7000FFF723FF20602878000705D59DF8000033
:109F8000B04201D1012078BD002078BD38B504462B
:109F90000D460022009269462046FFF70EFF20780A
:109FA00000F00700062805D19DF80000A84201D165
:109FB000012038BD002038BD38B504460D460022CA
:109FC000009269462046FFF7F8FE2078C04340071C
:109FD00005D19DF80000A84201D1012038BD002024
:109FE00038BD0023002900D001230022012182E690
:109FF00070B50546144601231A462846FFF77BFE36
:10A000002C54401C70BD014600200978002900D066
:10A010000120704778B50446154600260096204674
:10A020006A46FFF79DFF50B10098205C10B10120F7
:10A03000287000E02E700098401C009002E04FF065
:10A04000FF300090009878BD01460020002900D024
:10A050000120704700231A4619464CE600230122CE
:10A0600049E601460020CA0700D080208A0701D5B2
:10A0700040F040004A0701D540F020000A0701D512
:10A0800040F01000CA0601D540F008008A0601D54C
:10A0900040F004004A0601D540F00200090601D54F
:10A0A00040F0010070472DE9F04107460E4690460A
:10A0B00000250024404600F075FCC6B1761E0F2E28
:10A0C00015D801250AE028466D1C385CFFF7C9FF4A
:10A0D0000246E1B2404600F0AFFC641CB442F2D349
:10A0E000387800F00702F1B2404600F0AFFC284695
:10A0F000BDE8F08177B581B00446164620469DF84C
:10A100000810FFF719FF68B120466A4602A9FFF759
:10A110008DFE0546601932460099FFF7C4FF2844BA
:10A1200004B070BD4FF0FF30FAE72DE9F04106466C
:10A1300088460025404600F06AFC80B1404600F0A9
:10A1400068FC0746404600F062FCC7F1010100EBE5
:10A15000C100C0B2C0F10800012430700EE0002040
:10A16000012430700CE02946404600F05CFCFFF70B
:10A1700078FF2146641C70546D1CEDB2BD42F2D3D1
:10A180002046B5E770B505460E46304600F041FC66
:10A19000431C002208212846FFF7ADFD044628197C
:10A1A0003146FFF7C2FF204470BD70B505460C462E
:10A1B0001646304600F02DFC431C0122214628465D
:10A1C000FFF799FD044628193146FFF7AEFF2044FA
:10A1D00070BD38B50C46154600230093694603F060
:10A1E00038F9009B9B0D23800099C1F3150129606C
:10A1F00038BD30B414461A46042902D030BC0020C1
:10A200007047214630BCE4E7F8B5044615461E46C3
:10A210000020009020466A46FFF7A2FE48B1009851
:10A22000324620442946FFF7D4FF009908440090A5
:10A2300002E04FF0FF3000900098F8BD0B46114649
:10A2400063F39F5103F0FCB82DE9F0410546164633
:10A250001F46042301222846FFF74DFD0446281916
:10A260003A463146FFF7EAFF204441E770B504461D
:10A27000601CFFF7E3FF05462B4600220C21204619
:10A28000FFF739FD284470BD2DE9F04105460F4622
:10A2900000260024002F0CD0384600F0EEFD0646C4
:10A2A000384600F0F0FD02E0015D2955641CB4421F
:10A2B000FADB30461CE770B506460D460020002D3F
:10A2C00015D0284600F0D9FD03460022062130466D
:10A2D000FFF711FD0446284600F0CFFD2044B0F5FD
:10A2E000167F05D230192946FFF7CEFF204470BDF6
:10A2F000002070BD70B505460C4616460020002DA6
:10A3000017D0002E15D0304600F0B7FD03460122CD
:10A3100021462846FFF7EFFC0446304600F0ADFD2D
:10A320002044B0F5167F05D228193146FFF7ACFF5F
:10A33000204470BD002070BD70B503460D46104628
:10A3400000242A46194600F054FD00B12C46204650
:10A3500070BD77B581B005461646002000902846AE
:10A360009DF80810FFF7E8FD70B128466A4602A97B
:10A37000FFF75CFD044629193046009A00F039FDCC
:10A3800020B10098044401E04FF0FF342046C7E6B6
:10A3900070B50446049D681C002C0BD0884209D877
:10A3A0002270002103E066185A5C7270491CA942B1
:10A3B000F9D370BD002070BDF8B506460F4638468B
:10A3C00000F0CAFB0446384600F0CCFB0546384690
:10A3D00000F0CEFB02462B464FF416713046009437
:10A3E000FFF7D6FFF8BD2DE9F04107460E4630468F
:10A3F00000F0B2FB451C2B46002207213846FFF730
:10A400007AFC04466019B0F5167F05DA3819314632
:10A41000FFF7D2FF20446BE6002069E62DE9F0410A
:10A4200007460C461646304600F096FB451C2B4668
:10A43000012221463846FFF75EFC04466019B0F55C
:10A44000167F05DA38193146FFF7B6FF20444FE68C
:10A4500000204DE670B50C46164600250178421CDA
:10A46000631E304600F03EFB00B12546284670BD15
:10A4700077B581B0054616460020009028469DF825
:10A480000810FFF759FD88B128466A4602A9FFF770
:10A49000CDFC0446009B2A19521C295D5B1E3046E8
:10A4A00000F020FB20B10098044401E04FF0FF349D
:10A4B000204635E638B50C46154600210091002DA2
:10A4C00008D0012C08D0022C09D0032C0ED0042C6B
:10A4D00010D02960204638BD00782860FAE7694628
:10A4E00002F08FFFBDF800002860F3E7294602F074
:10A4F00099FFEFE7294602F0ACFFEBE777B581B0B3
:10A500000446164620469DF80810FFF715FD60B179
:10A5100020466A4602A9FFF789FC054660193246C3
:10A520000099FFF7C7FF2844FAE54FF0FF30F7E541
:10A53000FF2902D8017001207047B1F5803F02D297
:10A5400089B202F059BFB1F1807F01D202F063BF3E
:10A5500002F076BF70B506461446FF2C01D80123E1
:10A560000AE0B4F5803F01D2022305E0B4F1807F18
:10A5700001D2032300E0042301223046FFF7BBFB96
:10A58000054670192146FFF7D3FF284470BD70B50A
:10A590000446601CFFF7CCFF05462B460022022133
:10A5A0002046FFF7A8FB284470BD38B514460022AA
:10A5B00000926A46FFF77EFF002C01D000992160CF
:10A5C00038BD7CB5044616462046FFF7B5FC60B1A1
:10A5D00020466A4601A9FFF729FC05466019324664
:10A5E0000099FFF7E2FF28447CBD4FF0FF307CBDAF
:10A5F0009EE770B50446601CFFF7FAFF05462B4640
:10A60000002209212046FFF776FB284470BD70B573
:10A6100006461446FF2C01D801230AE0B4F5803F1A
:10A6200001D2022305E0B4F1807F01D2032300E0D0
:10A63000042301223046FFF75EFB054670192146D0
:10A64000FFF7D6FF284470BD10B50C46114600290F
:10A6500009D0012C09D0022C0AD0032C0BD0042CD9
:10A660000CD000200860204610BD02F007FFFAE77A
:10A6700002F01AFFF7E702F032FFF4E702F051FFB1
:10A68000F1E777B581B00446164620469DF80810DC
:10A69000FFF752FC60B120466A4602A9FFF7C6FBED
:10A6A0000546601932460099FFF7CEFF284437E58A
:10A6B0004FF0FF3034E501F18002FF2A02D849B2A1
:10A6C00002F0D9BE01F50042B2F5803F02D209B2D4
:10A6D00002F0E5BEB24A6FF07F430A449A4201D2CB
:10A6E00002F0F6BE02F014BF70B50446601CFFF71E
:10A6F000E2FF05462B46002203212046FFF7FBFA26
:10A70000284470BD70B50646144604F18000FF2849
:10A7100001D801230FE004F50040B0F5803F01D2DD
:10A72000022308E09E486FF07F422044904201D20D
:10A73000032300E0042301223046FFF7DCFA05463C
:10A7400070192146FFF7B7FF284470BD70B5044665
:10A750000846611C02F02FFF05462B46002204210B
:10A760002046FFF7C8FA284470BD70B50546164666
:10A77000042301222846FFF7BEFA04462919304671
:10A7800002F019FF204470BD70B50446104619460A
:10A79000A21C02F049FF05462B4600220521204657
:10A7A000FFF7A9FA284470BD2DE9F0410746144689
:10A7B0001D46082301223846FFF79DFA0646BA19BE
:10A7C0002046294602F030FF304491E40A780270B6
:10A7D0004A7842708A788270C978C17004207047C4
:10A7E00070B50446601CFFF7F1FF05462B460022BA
:10A7F0000B212046FFF77FFA284470BD70B5044650
:10A800001546042301222046FFF775FA0346E01897
:10A810002946FFF7DBFF184470BD02780A704278C2
:10A820004A7082788A70C078C870042070470346E6
:10A8300008461146042805D000220A70CA704A70E2
:10A840008A7070471846E8E738B504460D4620463A
:10A850006946FFF7B2FA9DF800000B2802D04FF0CE
:10A86000FF3038BD601C2946FFF7D7FF401C38BDBC
:10A8700038B5044615460020009020466A46FFF78A
:10A880006FFB40B1009829462044FFF7C6FF0099AE
:10A890000844009002E04FF0FF300090009838BD6F
:10A8A0000A8840F26C739A4203D3A2F26C7202706F
:10A8B00002E0FF2A08D802708A784270CA78827053
:10A8C0000979C170042070474FF0FF30704770B5B0
:10A8D0000446601CFFF7E4FF05462B4600220A21D0
:10A8E0002046FFF708FA284470BD70B505461646A5
:10A8F000042301222846FFF7FEF9044628193146B1
:10A90000FFF7CEFF204470BD027802F26C720A801D
:10A9100042788A708278CA70C078087104207047C3
:10A92000034608461146042805D00022CA708A70E2
:10A930000A710A8070471846E6E738B504460D46A6
:10A9400020466946FFF739FA9DF800000A2802D030
:10A950004FF0FF3038BD601C2946FFF7D5FF401C83
:10A9600038BD38B5044615460020009020466A469A
:10A97000FFF7F6FA40B1009829462044FFF7C4FFDC
:10A9800000990844009002E04FF0FF3000900098DA
:10A9900038BD20230370417082700320704700008F
:10A9A000FFFF7F0000220270002143185A70491CEB
:10A9B0000F29FADB704770B5CB0801250F2B0FD29A
:10A9C00006784C1CA64200D204705B4201EBC30324
:10A9D0009D40EBB200EBD1001AB1417819434170B0
:10A9E00070BD41789943417070BD30B50446002078
:10A9F000CA080123782909D2554201EBC5018B40D1
:10AA0000D9B2224452780A4200D0012030BD0078E9
:10AA10007047014600200978002903D0491EC8B2BA
:10AA2000C008401C704702460020002A03D00F29AE
:10AA300001D250184078704703460020002B04D004
:10AA40000F2902D258184270012070470346002097
:10AA5000002B03D0C800801A18700120704700280E
:10AA600001D0782070470020704710B500220028E0
:10AA70000BD051B10A78027000228B1884185B78D1
:10AA80006370521C0F2AF8D30122104610BD70B516
:10AA90000022002824D004780B789C4220D17F2CFF
:10AAA0001ED8E30804F00704C4F10804FF25E540BC
:10AAB00008E084188E1864787678B44201D00020BB
:10AAC00070BD521C9A42F4DB18441944407849780E
:10AAD00028402940884201D0002070BD012070BD6F
:10AAE000002070BDF0B50025002822D000240460AD
:10AAF000017140F251218B421BD84D1C92B10021B3
:10AB0000471D994208D2D0F800C0565C0CF8076087
:10AB10000668761C066001E046187471491CA9425B
:10AB2000EFD305E0002142185471491CA942FAD321
:10AB300001252846F0BD70B505460C46002C03D013
:10AB40002046FDF74DFB00E0002003462246284644
:10AB5000BDE870400021C5E701460020002900D073
:10AB60000868704701460020002900D0481D704742
:10AB700001460020002900D00879704730B505460D
:10AB80000C462046FFF7E8FF03462046FFF7EAFFA2
:10AB900002462046FFF7ECFF01462846BDE830405C
:10ABA000A0E730B5002815D0A2B1137993B9136886
:10ABB0008B420FD20023002408E015689D4203D980
:10ABC000D5186D79C55400E0C4545B1C8B42F4D396
:10ABD000012030BD002030BD70B5034600200029A3
:10ABE00018D0BBB10C681A68944212D10A791D7949
:10ABF000AA420ED10120002207E08D189E186D791F
:10AC00007679B54200D00020521C944201D9002828
:10AC1000F3D170BD21B109680029FAD1012070BDBE
:10AC2000002BFCD019680029F9D1012070BD70B546
:10AC300005460E460024002E17D0B5B13046FDF76C
:10AC4000CFFA296888421BD12879C8B9012400208D
:10AC500006E02B18325C5B799A4200D00024401C3D
:10AC600081420DD9002CF4D10AE02EB13046FDF717
:10AC7000B7FA28B9012403E015B1286800B9012406
:10AC8000204670BD70B50023002811D0046840F242
:10AC900051251444AC420BD8441D06E00668CD5C37
:10ACA000355505686D1C05605B1C9342F6D3012386
:10ACB000184670BD02460020002A05D040F25123FC
:10ACC000994201D8116001207047014600200029F7
:10ACD00001D040F25120704702460020002A01D0E6
:10ACE00011710120704730B502460020002A02D0C1
:10ACF000107908B1012030BD01200021136840F215
:10AD000052258B42F7D954186479203C5F2C00D32C
:10AD10000020491CA942F4D330BDF0B546180029E3
:10AD200001D0022550E00120F0BD02783AB1802A1E
:10AD300049D30323B3EB921F03D00020F0BD0020C2
:10AD4000F0BD894B9B5C994201D20020F0BDC91A2D
:10AD5000401C0478B5EB941F01D00020F0BD062BF9
:10AD60002FD2DFE803F02E03080E151C12F03E0F61
:10AD700029D10020F0BDE02A23D1A20621D4002051
:10AD8000F0BDF02A1DD114F0300F1AD10020F0BD13
:10AD9000F82A16D114F0380F13D10020F0BDFE2A86
:10ADA00006D0FF2A04D0FC2A0BD114F03C0F08D1A6
:10ADB0000020F0BD10F8012FB5EB921F01D000204C
:10ADC000F0BD5B1EF6D1401CB042AED30120F0BDF9
:10ADD00010B500240179062901D211B101242046C1
:10ADE00010BD50F8051BFFF798FF0028F7D001248D
:10ADF000F5E7F0B50025002821D00024046040F2DA
:10AE000052239A421BD881B10023061D0AE006D2C4
:10AE10000768CD5CBD5505686D1C056001E0C5186F
:10AE20002C715B1C9342F2D308E04FF0000100EB61
:10AE30000102147101F101019942F8D3012528465C
:10AE4000F0BD30B50022494B1C88494B1B78234488
:10AE500040F25224A34202D20124036008E0002100
:10AE60000160002030BD85188B5C2B71521C92B2A2
:10AE700003689342F7D8204630BD014600200029E0
:10AE800000D00868704701460020002900D0081D46
:10AE9000704710B504460B461846FFF7EEFF024612
:10AEA0001846FFF7F0FF01462046BDE81040A0E736
:10AEB00010B50023002A0DD060B114688C4209D36C
:10AEC000002103E053181B794354491C13688B423B
:10AED000F8D81368184610BD70B50023002811D0AB
:10AEE000046840F252251444AC420BD8041D06E01D
:10AEF0000668CD5C355505686D1C05605B1C93428A
:10AF0000F6D30123184670BD02460020002A05D062
:10AF100040F25223994201D8116001207047014646
:10AF20000020002901D040F25220704730B50022A5
:10AF3000002816D0A9B103680C68A34211D140F2D1
:10AF40005224A34209D90CE084188D1824792D7954
:10AF5000AC4201D0002030BD521C9342F4D80120F5
:10AF600030BD002030BD000070C00108A4040020E6
:10AF7000A3040020414081EA410080EA810080EA88
:10AF8000C10080EA011080EA411080EA811080EA65
:10AF9000C11101F0FE00C1F3002148407047CAB260
:10AFA0004240080A80EA022080EAC20080EA0230B9
:10AFB00080EA121102F00F00414081EAC01080B215
:10AFC000704738B50546049C0020002C04D1009041
:10AFD000284601F0B0F980B238BD30B40446029B77
:10AFE0000020002B03D1204630BC01F0C4B930BC96
:10AFF0007047002901D101F023BA7047002901D11F
:10B0000001F00EBA70470000F84900200870704740
:10B01000F6484068704710B50124B0F5800F0BD298
:10B02000F2494860F2490860FDF7E1F8F1498860AB
:10B03000F1490120887000E00024204610BDEB4952
:10B040004968814201D1012070470020704706F015
:10B05000C7BE10B5FDF7AAFD441CFDF75FF9044417
:10B06000FDF700FB0444FEF71BFB204410BD2DE957
:10B07000F0410F4690460025012806D1082139608D
:10B08000DA494968C8F800100125441E01266DB947
:10B09000641EFDF78BFD0646B44207D202203860DD
:10B0A0002046FDF786FDC8F8000001256DB9A41BF8
:10B0B000FDF734F90646B44207D200203860204636
:10B0C000FDF72FF9C8F8000001256DB9A41BFDF7A5
:10B0D000C9FA0646B44207D2012038602046FDF77F
:10B0E000C4FAC8F80000012565B9A41BFEF7D8FA18
:10B0F000844207D2042038602046FEF7D4FAC8F80C
:10B10000000001252846BDE8F0812DE9FF4FADF58F
:10B110001D7D0646DDF8A892AB9F984600240025C9
:10B120000020029001909F98B0494FF0FF3A4F28BD
:10B1300078D020DC3F2870D00EDC1E286ED006DCD4
:10B140000B286CD00C286BD01C2839D165E12C2839
:10B1500067D03E2834D12FE14B284AD006DC402866
:10B1600078D0462877D049282AD139E14C2820D0F8
:10B170004D2825D144E0792860D00EDC6B286BD0B7
:10B1800006DC602869D0612868D0622818D193E075
:10B1900070284DD0782813D161E0DFF860B2B0F5A7
:10B1A0007A7F70D006DC8B286ED09B286DD0D1289A
:10B1B00006D1C4E0A0F54070E93867D0012870D00E
:10B1C000022089F80000202038705446002C0BDB48
:10B1D0009F984C2808D0B8F1FF3F05D0022089F88D
:10B1E00000003220387054460DF5217D204600F0D5
:10B1F00081BB4A6808213046FFF738F80446E5E786
:10B2000006F0DCFD014603A8FFF795FC03A93046D4
:10B21000FFF7E9F80446D9E704E00EE1F6E0D8E0EC
:10B2200040E034E008213046FFF7E3F90446CDE77B
:10B2300009783046FFF7DDF90446C7E706F0D6FD8A
:10B24000014603A8FFF777FC03A93046FFF7CBF8C8
:10B250000446BBE7F9E00AE0B5E04DE038E0FFF76F
:10B26000F6FE01463046FFF792F90446AEE706F0D7
:10B27000C1FD014603A8FFF75EFC03A93046FFF7B6
:10B28000B2F80446A2E7E8E01CE0D0E0F9E05CA1F7
:10B2900003A8FFF750FC03A93046FFF7A4F80446C3
:10B2A00094E7F5E058A103A8FFF745FC03A9304651
:10B2B000FFF799F8044689E701213046FFF767F95F
:10B2C000044683E70C213046FFF761F904467DE729
:10B2D00099A8FFF767FBE8B201F032FA0246E9B23B
:10B2E00099A8FFF768FB6D1C282DF4D399A9304667
:10B2F000FEF748FF044669E799A8FFF753FBE9B258
:10B30000002299A8FFF757FB6D1C332DF7D3374C5C
:10B3100008344FF4806509E0A06830B1804720B15F
:10B320002178012299A8FFF746FB38342088A842EB
:10B33000F2D399A93046FEF725FF044646E7FFF70A
:10B3400088FE8346B8F1000F0FD0B8F1FF3F12D04E
:10B3500001AA02A94046FFF78AFE30B3DDE90121C8
:10B360003046FEF783FF044630E759463046FFF784
:10B370000EF904462AE7012514E001AA02A928468D
:10B38000FFF775FEDDE901213019FEF76FFF044478
:10B390002044B0F5167F04DB362038706FF00104CE
:10B3A00014E76D1C5D45E8D910E7022089F800001C
:10B3B0002A203870544609E74FF416713046FFF7DB
:10B3C000E6F8044602E703213046FFF712F9044687
:10B3D000FCE64EF660213046FFF7D9F80446F5E664
:10B3E00000213046FFF7D3F80446EFE6C8020020FC
:10B3F00084020020E886002038870020EE08002024
:10B40000302E382E30000000312E30004FF41671EF
:10B410003046FEF717F80446D8E6FEA103A8FFF76A
:10B420008AFB03A93046FEF7DEFF0446CEE6002184
:10B430003046FFF7ACF80446C8E600F0E9FF0146E5
:10B440003046FFF7A4F80446C0E600F0E5FF0146E9
:10B450003046FFF79CF80446B8E6BBF800103019F8
:10B460006943FFF794F804442044B0F5167F04DBE9
:10B47000362038706FF00104A8E66D1C052DECD95C
:10B48000A4E6BBF802103046FFF781F804469DE6BB
:10B49000BBF826103046FFF77AF8044696E6F0B57A
:10B4A000ADF51B7D044600256A4604F11000D4F872
:10B4B000681201F054FC02262527002807DA84F8D8
:10B4C0006D6284F86E7200200DF51B7DF0BD208941
:10B4D0004C2809D0E168491C06D084F86D623220FE
:10B4E00084F86E020020EFE70DF10D0178285ED0A0
:10B4F0000ADC4FF00902402834D0462861D04B289E
:10B5000014D04D280BD165E0792847D0B0F57A7F6B
:10B510000AD0A0F54070E9386AD001286ED084F8CE
:10B520006D62202084F86E022846CDE79DF8020067
:10B530000C2804D084F86D6284F86E22F4E7BDF81C
:10B540000800082809D10398FFF765FD28B1039882
:10B55000C0B20AF0F2F90125E6E784F86D6284F8DA
:10B560006E72E1E79DF80200022804D084F86D6253
:10B5700084F86E22D8E70298401EFD2809D8029868
:10B58000C4B2204600F02AFF20460AF0D6F9012571
:10B59000CAE784F86D6284F86E72C5E79DF8020010
:10B5A0000728C1D108460AF0C6F90125BCE79DF875
:10B5B00002000228B8D1029880B20AF0BBF9012536
:10B5C000B2E79DF802000728AED108460AF0B4F9A8
:10B5D0000125A9E79DF80200072804D084F86D62D0
:10B5E00084F86E22A0E708460AF098F901259BE747
:10B5F0009DF80200022897D1012595E79DF80200E9
:10B60000022891D101258FE72DE9F04104460E462D
:10B61000174600252088092836D2DFE800F00524E7
:10B6200010351B3535352D006068FCF771FE10B301
:10B63000022084F86D02282084F86E0224E06068FD
:10B64000FDF7AEFAB8B13A4631462046FDF71FFC89
:10B65000054619E06068FEF71DF860B12046FEF768
:10B66000A5F9054610E06068FCF7F6FF18B1204622
:10B67000FDF785F9054607E06068FFF7E0FC18B1C3
:10B680002046FFF70CFF054628463CE501207047A1
:10B6900064484068704710B502460C460020614976
:10B6A00049688A4207D106F089FB01462046BDE879
:10B6B0001040FFF740BA10BD002801D05A4B03607C
:10B6C00011B159485C300860002A02D056487030E9
:10B6D000106070470021002802D104E0491C001DC1
:10B6E0000268521CFAD10846704702464D4808309D
:10B6F0004FF4806302E0914204D0383001889942CF
:10B70000F9D3002070472DE9FC4106464FF0FF3089
:10B710000C69002C19D04A69BAB10A890223322572
:10B720004B2A14D04F2A26D0B769002F0BD00B76A6
:10B730004D7601F11900431ECDE90030CB68B569A3
:10B7400049682046A847BDE8FC810020FBE7CA689D
:10B75000521C02D00B764D76F5E70888082802D1F6
:10B76000304A52684A604A68014602B02046BDE845
:10B77000F041FEF77BBDCA68521C02D00B764D76B5
:10B78000E1E709882046BDE8FC41FEF732BF2DE91C
:10B79000F04104464FF0FF372088FFF7A6FF05462B
:10B7A00001264FF01F0875B1296941B160688847CB
:10B7B00028B121462846FFF7A6FF074606E0267671
:10B7C00084F8198002E0267684F8198038469AE4D5
:10B7D00010B502460C4600202060A0602061104693
:10B7E000FFF783FF38B1036A2BB104F1100204F1B3
:10B7F0000801204698472068D0B1FFF76BFF6060D2
:10B80000A068B8B1FFF766FFE0602069A0B1FFF75C
:10B8100061FF0BE04261636E65742050726F647566
:10B8200063740000C802002070C10108606110BD8F
:10B830000020E4E70020E7E70020EAE710B5FFF783
:10B8400054FF08B1406A10BD002010BD70B50D4610
:10B8500016460024FFF749FF28B143691BB1314662
:10B86000284698470446204670BD2DE9F043ADF5C3
:10B87000197D81460E4617464FF00008002098902B
:10B88000FFF7E7FB054601241FE097AA98A9204689
:10B89000FFF7EDFBC0B1989880B2FFF726FF98B193
:10B8A00043698BB101A99798984768B101A94846A7
:10B8B000FFF792F940B14FF001080EB1989830604F
:10B8C0002FB19798386002E0641CAC42DDD90DF5C9
:10B8D000197D4046BDE8F08370B50D46002480B266
:10B8E000FFF703FF20B102692846904700B1012409
:10B8F000204670BD30BCBDE8C08F000010B5FF48C9
:10B90000002101714171817101724172816200F106
:10B9100024031A6822F0080222F0200222F0010219
:10B9200022F002021A60F64A12788272F54A127800
:10B9300002730122C2728182C17100F0C4FE012033
:10B9400010BD70470022FF2911D001230370417000
:10B95000012143185A70491C0729FADB02818272BF
:10B9600000214318DA72491C0729FADB704702707C
:10B970004270EDE710B588B004460020E24A00218D
:10B980001378002B0BD0117000236A4603A9DF48FF
:10B9900002F0DDF880B20121217008B010BDDC4A50
:10B9A0001378002BF9D011700022501E014602F0CE
:10B9B000B8F9082002212170EFE72DE9F043ADF539
:10B9C000197D8946A09D90461E464FF6FF770024BC
:10B9D00055218DF85C12FF218DF85D128DF85E0205
:10B9E000FFF7C8FA014648468DF85F92FFF7C2FAA2
:10B9F000014640468DF86082FFF7BCFA0146280AEE
:10BA00008DF86102FFF7B6FA0146E8B28DF86202DE
:10BA1000FFF7B0FAC0438DF863023DB90EE0305D28
:10BA20003946FFF7BCFA0746641CA4B2AC42F6D311
:10BA3000F8438DF85802000A8DF8590200F02EFEE6
:10BA4000012000F020FEB5B198999798CDE900014A
:10BA50002A46314602A804F0BDFC0DEB0500BDF8F6
:10BA6000581201810A35A9B2684600F030FE0DF582
:10BA7000197DBDE8F083082197A800F028FEF6E7BD
:10BA80002DE9F843002400949C4D4FF0010805F186
:10BA90002C07287900280CD04FF0020901282AD061
:10BAA00005F12406022865D003286FD02C71BDE86B
:10BAB000F88300F01DFE38B100F005FEE879FF289C
:10BAC000F5D2401CE871F2E75146684600F012FEDC
:10BAD0000028ECD000F0F7FDE879FF2801D2401CE7
:10BAE000E8719DF80000552801D185F8048085F89B
:10BAF00004803870DBE700F0CEFD5A2803D90BF044
:10BB000036FF2C71D3E700F0F3FD40B100F0DBFD10
:10BB1000E879FF2801D2401CE8712C71C7E7514633
:10BB2000684600F0E7FD0028C1D000F0CCFDE879C0
:10BB3000FF2801D2401CE8719DF80000FF21FF287A
:10BB400009D055280DD003280ED019280CD00BF0A1
:10BB50000DFF2C71ABE76C822970797085F8049029
:10BB6000A5E785F80480A2E76C822970787085F8D3
:10BB700004909CE700F08FFD5A2808D9306840F007
:10BB8000010030600BF0F3FE2C7190E7E6E000F06E
:10BB9000AFFD60B100F097FDE879FF2801D2401CAD
:10BBA000E871306840F0010030602C717FE7514649
:10BBB000684600F09FFD002885D000F084FDE879FC
:10BBC000FF2801D2401CE871688A98B1012839D059
:10BBD0004FF00308022842D003284DD0042859D042
:10BBE000052866D0306840F0010030600BF0BEFEE2
:10BBF0002C715CE729789DF80000FFF7BBF92870ED
:10BC00009DF800002872397855290CD17978FF29E0
:10BC100009D1072807D900F056FDE879FF2801D29D
:10BC2000401CE8712C719DF80000B8703878FF282E
:10BC300002D17878192802D0A5F8128037E70EF0E3
:10BC4000BDFF34E729789DF80000FFF793F92870CD
:10BC50009DF80000A871F870A5F8129027E72978E0
:10BC60009DF80000FFF786F928709DF800006872C3
:10BC70003871A5F812801AE729789DF80000FFF7BF
:10BC800079F928709DF800000102A98278710420DA
:10BC900068820CE729789DF80000FFF76BF928709F
:10BCA000A98A9DF800000144A982B8710520688224
:10BCB000FDE69DF80000F871104806212C300BF0CD
:10BCC00057FEF979BA7901EB0221814202D10EF0D7
:10BCD00075FFECE629789DF80000FFF74BF9287016
:10BCE00055281BD00BF042FE306840F00100306058
:10BCF00000F0E9FCE879FF280ED20BE020040020D8
:10BD00008102002080020020A004002060B00020FA
:10BD1000A1040020401CE8712C71C8E6A88A48B133
:10BD2000E98A884206D86C824FF6FF70288285F82F
:10BD30000480BCE638B1306840F0010030600BF0A0
:10BD400015FE2C71B3E6A879A97A884201D0FF28A4
:10BD5000F7D1306840F002003060F2E700F09BFC61
:10BD60005A2807D9306840F0010030600BF0FFFD21
:10BD70002C719CE600F0BCFC60B100F0A4FCE879FA
:10BD8000FF2801D2401CE871306840F001003060AB
:10BD90002C718CE65146684600F0ACFC002887D038
:10BDA00000F091FCE879FF2801D2401CE871688A14
:10BDB000A98A88420DD2298A9DF80000FFF7EFF882
:10BDC0002882688AAA6A9DF800101154401C688273
:10BDD0006DE609D1298A9DF80000FFF7E0F8288276
:10BDE000688A401C688262E6491C884295D1298A8B
:10BDF0009DF80000FFF7D3F82882A0F57041B8390C
:10BE000007D0306840F0010030600BF0AFFD2C71BE
:10BE10004DE6A879A97A884201D0FF28F7D1306889
:10BE200040F002003060F2E72DE9FF5F0024FE4E93
:10BE3000F178307B491C401CB1FBF0F200FB121181
:10BE400001F0FF08B27A511CB1FBF0F300FB1311B3
:10BE500001F0FF0BB1784B1CB3FBF0F500FB153084
:10BE6000C0B2029006F1240A96F805C0DAF8003054
:10BE7000002523F00400039030460127407A4FF05C
:10BE80000409BCF1090F79D2DFE80CF0051579DC63
:10BE9000F9F8F7F6F500B270F270322030620398CC
:10BEA0007771012420F0020020F00100CAF80000A0
:10BEB00000F009FC3BE200F0EEFBB0F5FA7F0ED398
:10BEC0000BF055FDF57106207071DAF8000020F0D6
:10BED000020020F00100CAF80000012427E2DAF88D
:10BEE0000000C10708D00BF041FDDAF8000020F097
:10BEF0000100CAF800001AE28107DBD5317A072970
:10BF000032D2DFE801F004123129311F1A00B17971
:10BF1000FF2929D020F00200757020F00400CAF833
:10BF200000000220707101241EE000950023B27A07
:10BF3000717A0220FFF741FD16E040F02000CAF8B8
:10BF4000000011E040F02000CAF80000B079FF289E
:10BF50000AD00820707107E0B08A0090B27A717A36
:10BF60000420B36AFFF729FD70790828A2D0DAF817
:10BF7000000020F00200CAF80000D8E1D6E10195E7
:10BF800001A8FFF7F7FC30839DF8041081B3022964
:10BF900008D10090A54BB27AFF210620FFF70DFDD6
:10BFA00086F805909DF8040007280BD0012814D0CE
:10BFB000032503281DD0042827D005282FD00628C4
:10BFC0002DD035E0308B0090984BB27AFF210620BF
:10BFD000FFF7F3FC86F805902AE0308B0090934B36
:10BFE000B27AFF210620FFF7E8FC86F805901FE0F3
:10BFF00022E005F0A9FF0146308B00908C4BB27A0D
:10C000000520FFF7DAFC757112E0308B0090874B4A
:10C01000B27AB17B0520FFF7D0FC757108E0308B58
:10C020000090824BB27AB17B0520FFF7C6FC757198
:10C030007078401C70707AE1F07A7070012486F894
:10C04000059074E100F027FBB0F5937F07D90BF062
:10C050008EFCF07A707086F80590012467E1DAF8BA
:10C060000000C1070CD020F00100CAF8000086F8DB
:10C07000059001245BE13AE1DCE0AAE084E024E001
:10C080008107D8D5B179B27A914215D1317A042994
:10C0900008D0062909D0072901D077710DE086F86C
:10C0A00005900AE086F8059007E040F02000CAF805
:10C0B000000086F8059000E07771DAF8000020F0C3
:10C0C0000200CAF80000012431E1707896F80BC034
:10C0D000604503D202207071012428E158070DD475
:10C0E00091420BD186F803B00023594601200095F8
:10C0F000FFF763FCF5610720707118E1306A3128A1
:10C1000018D249485B07006A00F1010007D559457C
:10C1100005D07570306202207071012407E1306231
:10C12000002318460095FFF748FCF561F5710520DE
:10C130007071FCE088451BD158070DD50299F1704C
:10C14000002301200095FFF738FCB07AB070F5614C
:10C15000376207207071EAE0F270002318460095FC
:10C16000FFF72BFCF5613762F57105207071DEE099
:10C1700086F803800023414601200095FFF71DFC4F
:10C18000F56107207071D2E000F085FA5F2805D8CC
:10C19000F079042801D977710124C8E0F06970B101
:10C1A0000299F17000950023B27A0120FFF705FC97
:10C1B000B07AB070F561356207207071B7E0F76151
:10C1C00000950023B27AB1781846FFF7F6FBF571B7
:10C1D000ADE002EB82004FF4FA7808EB400900F082
:10C1E0005AFA484505D2F079042801D9777101241B
:10C1F0009DE0B07A401C00EB800008EB400700F0A7
:10C200004AFAB8420ED286F803B000950023B27AFB
:10C2100059460120FFF7D1FBB07AB070F561356265
:10C220000720707183E000002004002060B000202F
:10C23000E8B80020990720D5B179914202D1317A2E
:10C24000022908D077710124DAF8000020F00200FA
:10C25000CAF800006BE00399CAF80010B070F571DD
:10C260000023014618460095FFF7A7FBB07AF0704F
:10C270003562F56105207071E6E700F00CFA5F2881
:10C2800003D89AF80000C00751D0DAF8000041073F
:10C2900004D5757002207071012421E0B178B27A62
:10C2A000914209D0F571002318460095FFF785FBF0
:10C2B000F5610520707113E0904509D086F8038080
:10C2C0000023414601200095FFF777FBF56107E069
:10C2D00040F00400CAF8000075700220707101245B
:10C2E000DAF8000020F00100CAF800001FE019078A
:10C2F0000ED5308B00905B4B717B0620FFF75DFB0A
:10C30000DAF8000020F00800CAF80000777106E0B3
:10C310000146002307200095FFF74FFB7771DAF8FD
:10C32000000020F00200CAF8000000E0777104B0BD
:10C33000204600F09DB82DE9F0411746069A0646C2
:10C340001C460020484D002A0FD14978286861F327
:10C350000410286022463946424804F03BF8A5F113
:10C3600024000483717841732046296841F0080154
:10C370002960BDE8F0812DE9F041064600273A4DDD
:10C38000243DA86A002801D1A962EA82364C2068BF
:10C3900081070BD4C00709D1FFF772FB216888071A
:10C3A00004D4C80702D128790028F5D1287940B9EA
:10C3B0002E49A87A0978884203D8FFF735FD00286E
:10C3C000FBD12068810607D520F020002060AF8ACD
:10C3D00001203070687A70703846CAE722492439E3
:10C3E0000873704721490978884206D81E492439C4
:10C3F0008872097B884200D9F0E770471A482438D0
:10C40000807A7047002802D017492439C8727047D3
:10C4100015482438C07A704713482438007B704789
:10C42000002101220270104A243A927A42700022BE
:10C43000028182724318DA72491C0729FADB7047BD
:10C44000002100280DD001220270FF2242704FF619
:10C45000FF720281002282724318DA72491C072996
:10C46000FADB704760B00020440400208002002006
:10C4700030BCBDE8C09F0000002803D001684068C0
:10C48000081A70470020704700B50246002A05D000
:10C490001046FFF7F1FFD168884201D1012000BDAD
:10C4A000002000BD00B502460B46002A08D0104609
:10C4B000FFF7E2FFD268101A984201D3012000BDB5
:10C4C000002000BD00B5002804D0FFF7D5FF08B15B
:10C4D000002000BD012000BD002808D04168C268CE
:10C4E000B1FBF2F302FB13118068405C704700203F
:10C4F000704700B5024600231046FFF7E3FF50B92E
:10C500005068D168B0FBF1F301FB130091680B5C3C
:10C510005068401C5060184600BD70B503460C467C
:10C520001846FFF7A9FF904200D91046824210D961
:10C5300002460EE05968DD68B1FBF5F605FB161101
:10C540009D68695C5D686D1C5D600CB104F8011B41
:10C55000401E0028EED1104670BD70B503460D4652
:10C560000024002B0AD01846FFF78EFF40B1234865
:10C570000068B0F5967F01D908F0A3FE204670BD93
:10C580001868DA68B0FBF2F102FB110099680D54EB
:10C590001868401C18600124F0E7F0B504460D4609
:10C5A0001646002731462046FFF77CFF90B175B94B
:10C5B00010E02068E168B0FBF1F201FB1200A26814
:10C5C00015F8011B11542068401C2060761E002EB7
:10C5D000EFD101273846F0BD002801D00168416045
:10C5E0007047002808D0002906D0002A04D0002374
:10C5F000036043608160C26070470000A8020020B1
:10C600002DE9F04188B007460D461646984614219C
:10C6100003A803F0F8FE0020009001900290287813
:10C62000012826D16B463A4603A9284601F0D3F9E2
:10C6300004469DF802004FF6FF71002819D1002C26
:10C6400017DDB44215DCBDF8140058B1884209D09A
:10C650000BF00EFBBDF8141088420AD19DF81600AD
:10C66000062806D1301B82B229194346384600F00D
:10C670002EF908B0BDE8F08126494FF4007201F5AB
:10C680000070FFF7AEBF002802D0012009F047B9C3
:10C69000002009F044B920480088704710B508F020
:10C6A000F7FE052809D0062809D0072809D002215D
:10C6B000FFF7F1FF8842FBD310BD0621F8E7042104
:10C6C000F6E70321F4E7144900200880704770B5AD
:10C6D00004460D460BF04CFA401C06D00BF048FA0D
:10C6E0000246294620460EF023FBBDE87040EAE7EB
:10C6F0000020704770B5044600250848FFF7E2FEA9
:10C7000028B91CB10548FFF7F4FE20700125284622
:10C7100070BD7047D4B2002054040020D4B400206F
:10C720001E2802D2F64A42F820107047F5494860A8
:10C7300070470B2803D2F24A783242F82010704733
:10C7400030B500210022002528281FD2ED4B1033E0
:10C750005C5C844206D10125E94B53F8211021B1DC
:10C76000012202E0491C1E29F2DB7DB90021E54BC4
:10C770002E335C5C844206D1E148783050F82100C9
:10C7800020B1012202E0491C0B29F2DB104630BD2A
:10C7900070B504460023002000251570282C16D201
:10C7A000D84D1035EE5CA64204D101200B60012368
:10C7B000137002E05B1C1E2BF4DB002807D1002263
:10C7C000D04B2E339D5CA54202D101200A6070BD82
:10C7D000521C0B2AF6DB70BD1D2814D2DFE800F0D6
:10C7E0000F0F0F13130F13130F0F130F1313130F39
:10C7F0000F0F130F0F130F13130F130F0F00C04A58
:10C80000A43242F820107047C21E1B2A13D2DFE860
:10C8100002F00E0E120E0E12120E120E0E0E12124A
:10C82000120E12120E120E0E120E12120E00B44A38
:10C83000A43242F8201070471E2802D2B24A42F8B1
:10C8400020107047AF4988607047AE49C860704794
:10C850002DE9F0470446DDE908890E4615461F46D6
:10C860002078C0F3C00028702078C0F38000687082
:10C870002078C0F34000A8706078FDF707FA686080
:10C880006078FDF71EFAA860A07828730320297845
:10C8900021B1E078687321790520A973411C205CDF
:10C8A0008AB23870A018C8F80000B01AA9F80000C1
:10C8B0001046BDE8F087934840887047914948800A
:10C8C00070479048007870478E4908707047F0B5FF
:10C8D0008FB007460C4616461D4600200B900C9064
:10C8E0000D900E9009900A90089007900690059080
:10C8F000049003900290002C72D0217801F0F00295
:10C900001211062A22D2DFE802F0034DA4A7EEC3DB
:10C9100006A807A9CDE9001008AB0BAA31462046AE
:10C92000FFF796FF9DF820000C2810D00E2817D096
:10C930000F281ED0102825D012282CD00BAB3A4639
:10C940000095BDF81810079802F02AFBCBE00BAB5E
:10C950003A460095BDF81810079802F0FCF9C2E0BD
:10C960000BAB3A460095BDF81810079802F0A0FDF1
:10C97000B9E00BAB3A460095BDF81810079800F0E7
:10C98000ADFEB0E00BAB3A460095BDF81810079825
:10C9900002F0F2FEA7E02B463A463146204601F06F
:10C9A000D2FAA0E061780891A31C0793B11E89B266
:10C9B00006919DF82020082A36D125B1012D1FD0DF
:10C9C000022D1DD030E0052E05D11878DF2802D1C8
:10C9D0005878FD2805D03A46184600F05BFE23E063
:10C9E0008BE008F0ABFF49490120087007984849DF
:10C9F0008078C0EB0010800008800DF0C0F813E0D4
:10CA0000019000906B4601AABDF81810079802F03B
:10CA100078FBC0B220B1FEF7FBFA0199884203D13E
:10CA200029463C4801F0BDF89DF82000042801D0BB
:10CA300038B158E02B463A463146204601F083FA99
:10CA400051E02B463A46BDF81810079802F0A5F8B9
:10CA500049E0A078089046E0C1F3C0028DF8242098
:10CA6000C1F380008DF8250060788DF82600022043
:10CA700032B1A0788DF82700E17804208DF82810D5
:10CA8000411C205C089060180790701A06902AE0FC
:10CA9000A07808900326122805D1E01C0021FDF79C
:10CAA00075FA00B10426A01904AA05A9FDF7BEF97C
:10CAB0000644A01902AA0499FDF777FD0644A019BF
:10CAC00004AA05A9FDF7B2F90644A01903AA04991E
:10CAD000FDF76BFD30449DF82010122903D120444E
:10CAE0000021FDF769FA40F2391045430A4840F247
:10CAF000722100EB450003F086FC0FB0F0BD000092
:10CB0000E4B400205804002000B60020AC0200204D
:10CB1000AE0200205ABB0020E8B8002010B5002269
:10CB2000002816D0002914D00B7803708B188418B5
:10CB30005B786370521C072AF8DB0A8902818A7AC3
:10CB4000827200228B188418DB7AE372521C072A47
:10CB5000F8DB10BD70B50022884201D1012070BD04
:10CB600004890B899C4201D0002070BD837A8D7AA4
:10CB7000AB4201D0002070BD072B0BD9072309E081
:10CB800085188E18ED7AF67AB54201D0002070BD76
:10CB9000521CD2B29A42F3D3B4B903780A789342C2
:10CBA00001D0002070BD072B00D90723002209E027
:10CBB00084188D1864786D78AC4201D0002070BD67
:10CBC000521CD2B29A42F3D3012070BD30B4044655
:10CBD0000020002911D0002C0FD08B7801F1080221
:10CBE0000D2B0AD2DFE803F0070B10151A1F252AB8
:10CBF0002F34393E43002370012030BC7047097A3E
:10CC0000204630BCFDF7EDB98968204630BCFDF701
:10CC1000BEBC8968204630BCFDF766BD89682046E9
:10CC200030BCFDF793BDD1E90223204630BCFDF7AF
:10CC3000ABBD204630BC1146FDF73DBB204630BCA5
:10CC40001146FDF7D0BB204630BC1146FDF79ABA1D
:10CC50008968204630BCFDF7CCBC204630BC11466C
:10CC6000FDF735BE204630BC1146FDF7B9BDCA6898
:10CC70000989204630BCFDF7F9BA2DE9FC4104468C
:10CC80000E4610461D460027002C5DD0002D5BD0BF
:10CC900005F108020D2E57D2DFE806F056070B11FA
:10CCA000171D23292F353B414700FDF7CDF9287289
:10CCB0004AE001462046FDF7FDFB074644E00146F9
:10CCC0002046FDF7C1FC07463EE00146204600F045
:10CCD0004EFC074638E00146204600F09AFC074625
:10CCE00032E001462046FDF727FB07462CE00146CF
:10CCF0002046FDF7AFFB074626E001462046FDF73C
:10CD0000D2F9074620E001462046FDF74EFC0746D3
:10CD10001AE001462046FDF703FE074614E00146EF
:10CD20002046FDF784FD07460EE0002101910091A9
:10CD300001466B4601AA2046FDF75BFA0746BDF89F
:10CD4000040028810098E86037B92EB1012E03D085
:10CD5000062E01D01020A8703846BDE8FC812DE9D0
:10CD6000FC41064614460025002701970097002E37
:10CD70001CD0DCB13078000718D427706A4601A9AE
:10CD80003046FDF753F878B105469DF80410A170C0
:10CD900070192346009AFFF770FFA178102901D07F
:10CDA000054401E04FF0FF35C4F860722846D4E72F
:10CDB0002DE9FC4114460026019600960027F84D07
:10CDC000002802D028606960AE6054B3696841B33E
:10CDD0002A68A868135C1B0723D4267010446B468E
:10CDE00001AAFDF75FF8D0B1A9680A18AA606968BE
:10CDF000081A68609DF80410012902D0009B834244
:10CE00000DD8A170286823461044009AFFF735FF1B
:10CE1000A9680144A9606968081A68600127C4F814
:10CE20006062384699E703460020002B0BD00D299D
:10CE300009D2DFE801F00808070707070707070717
:10CE400007070700104670477CB505460024002000
:10CE500001900090002D10D0287800070DD46A466C
:10CE600001A92846FCF7E2FF38B1044628199DF8CD
:10CE70000410009AFFF7D7FF044420467CBDF0B4AD
:10CE800004460020002A52D0002C50D0957802F1A0
:10CE900008030D2D4BD2DFE805F0070B10151A1F04
:10CEA000262B30353A3F44002046F0BCFDF7D6B87B
:10CEB000127A2046F0BCFDF79BB892682046F0BC81
:10CEC000FDF748BB92682046F0BCFDF71BBC92689A
:10CED0002046F0BCFDF749BCD2E9020302462046D9
:10CEE000F0BCFDF761BC2046F0BC1A46FDF702BA63
:10CEF0002046F0BC1A46FDF791BA2046F0BC1A460F
:10CF0000FDF753B992682046F0BCFDF780BB204680
:10CF1000F0BC1A46FDF7E9BC2046F0BC1A46FDF706
:10CF20006DBCD36812892046F0BCFDF78DB9F0BC0A
:10CF3000704702461020982A52D01BDC352A3CD07C
:10CF40000BDC022A27D0262A06D1012939D0022952
:10CF500002D0032900D102207047662A3CD0842ADF
:10CF6000FAD129B101292ED002292ED00329F3D1DB
:10CF70000C207047D32A2AD0D42A03D0D62A01D035
:10CF8000DA2AF6D129B1012903D00229F1D10420EE
:10CF90007047022070470929FCD2DFE801F006063D
:10CFA000080A050A0A0C0C00F4E70C207047092057
:10CFB000704702207047012070470029FCD10C20E7
:10CFC00070470C207047092070470220704709B154
:10CFD0000129FBD10C2070470029FCD10C2070479F
:10CFE0000529FCD2DFE801F0030304060800F6E798
:10CFF00001207047022070470420704770B5054635
:10D000000C4610460023002C0ED06DB16178FFF75E
:10D0100090FF102805D2617822462846FFF72FFF9F
:10D0200003460020C4F86002184670BD2DE9FC419B
:10D030000646884615461F460024002001900090B1
:10D04000002E33D04DB3317809072FD50121297037
:10D05000C5F860026A4601A93046FCF7E7FE0446BF
:10D060003CB1444505D89DF804103046FCF7A4FFB8
:10D0700010B1012C19D019E09DF8041069703846E0
:10D08000FFF757FFA870102808D2264401462B4608
:10D090003046009AFFF7F1FD044407E0009808B11C
:10D0A000044403E04FF0FF3400E00024204654E63F
:10D0B0007CB5054616460024002001900090002D06
:10D0C00019D02878000716D56A4601A92846FCF72A
:10D0D000ADFE80B104469DF804103046FFF729FFED
:10D0E0000146102905D22819009AFFF79CFE044436
:10D0F00001E00098044420467CBD0346002000293E
:10D100000AD0002B08D0087820B148780A4601469A
:10D110001846B4E6184659E5704770B505460C4602
:10D120000126002D43D074B3A078A870A27804F132
:10D13000080105F108000D2A34D2DFE802F03407B7
:10D140000A0D1013181B1E2125282B00207A287287
:10D1500029E0A068A86026E0A068A86023E0A06895
:10D16000A86020E0D4E90201C5E902011BE0FDF757
:10D1700090FE18E0FDF702FD15E0FDF776FC12E0E9
:10D18000A068A8600FE012E001F05AFB0BE001F08C
:10D1900067FB08E020892881E068E86003E0000080
:10D1A000940400200026D4F86002C5F860023046DE
:10D1B00070BD2DE9FC5F0646884693460027002097
:10D1C00001900090307800F00700062845D13046E5
:10D1D0006A4601A9FCF72AFE04469DF80490012541
:10D1E0004FF0FF3A305D00F0070106290BD0C14334
:10D1F000490714D000071ED5A8EB040130195A4680
:10D20000FFF756FF1CE030196A4601A9FCF70EFE35
:10D210009DF80410494513D16D1CEDB210E0301992
:10D220006A4601A9FCF702FE9DF80410494507D1A2
:10D230006D1EEDB204E0A8EB04013019FFF704FE07
:10D24000044415B1002804DD0744444503D957467A
:10D2500003E0574601E0002DC4D1384600F0C8B8BD
:10D26000F0B503468DB0084614460027049703978F
:10D270000025002C7DD0102B7BD20125A37004F15A
:10D2800008060D2B0FD2DFE803F0950711171D24B8
:10D290002A30363B41638D000022114603F091F99C
:10D2A00010B10120207285E0277283E00022114630
:10D2B00003F0BFF9A0607DE00022114603F081F980
:10D2C000A06077E000210DF017FC03F0C6FBA06022
:10D2D00070E000210DF010FCC4E902016AE0014693
:10D2E0003046FDF7AEFD054664E001463046FDF7E9
:10D2F00022FC05465EE000253046FDF753FB59E071
:10D300000022114603F095F9A06053E005A906AA92
:10D31000CDE9002107AB08AA2BA103F08DF8032863
:10D3200003D004280BD0002544E00698C3B2079828
:10D33000C2B2089881B2304601F03CF93AE0089850
:10D3400020810798A0720698E0720598207331E05A
:10D3500009A90AAACDE900210BAB0CAA1EA103F072
:10D360006BF8042806D003280DD0022813D000251E
:10D3700020E021E00C9820720B9860720A98A0724D
:10D380000998E07216E00C9820720B9860720A9867
:10D39000A072E7720EE00C9820720B986072A77270
:10D3A000E77207E003AB04AA0FA103F045F80228D7
:10D3B00005D00025C4F860720DB02846F0BD049871
:10D3C00020810398E060F5E72534642F2533642F2E
:10D3D0002533643A253364002533643A2533643AAF
:10D3E0002533642E253364002534643A25376400E0
:10D3F0003CBCBDE8C09F00000A0A027041700220D8
:10D400007047002905D0027812020A804078024352
:10D410000A80022070470A0C02700A0A427081706A
:10D4200003207047002909D0027812040A6043786B
:10D4300042EA03220A60807802430A6003207047B0
:10D440000A0E02700A0C42700A0A8270C17004202F
:10D45000704700290DD0027812060A60437842EA2C
:10D4600003420A60837842EA03220A60C0780243DA
:10D470000A600420704701700120704700290CD019
:10D480000278120603D56FF0FF020A6001E0002265
:10D490000A6000780A6802430A60012070470A0A9D
:10D4A000027041700220704700290FD002781206E6
:10D4B00002D5254A0A6001E000220A6003780A6862
:10D4C00042EA03220A60407802430A600220704761
:10D4D0000A0C02700A0A427081700320704700290A
:10D4E00014D00278120603D54FF07F420A6001E0A3
:10D4F00000220A6003780A6842EA03420A6043781D
:10D5000042EA03220A60807802430A6003207047DF
:10D510000A0E02700A0C42700A0A8270C17004205E
:10D52000704700290DD0027812060A60437842EA5B
:10D5300003420A60837842EA03220A60C078024309
:10D540000A600420704700000000FFFF08B5C278A1
:10D550008DF8002082788DF8012042788DF8022025
:10D5600000788DF8030000980860042008BD034689
:10D5700008461146042802D000220A607047184667
:10D58000E4E777B581B00446164620469DF80810BA
:10D59000FCF7D2FC60B120466A4602A9FCF746FCC3
:10D5A000054660193146FFF7D1FF284404B070BD2D
:10D5B0004FF0FF30FAE708B500909DF803000870BF
:10D5C0009DF8020048709DF8010088709DF80000E9
:10D5D000C870042008BD1CB502788DF80020427880
:10D5E0008DF8012082788DF80220C2788DF8032012
:10D5F00002798DF8042042798DF8052082798DF822
:10D600000620C0798DF80700DDE9000205C1082079
:10D610001CBD034608461146082803D000230B60B2
:10D620004B6070471846D6E71CB5CDE900019DF860
:10D63000000010709DF8010050709DF8020090707D
:10D640009DF80300D0709DF8040010719DF805004E
:10D6500050719DF8060090719DF80700D071082068
:10D660001CBD77B581B00446164620469DF80810CB
:10D67000FCF762FC58B120466A4602A9FCF7D6FBCB
:10D68000054660193146FFF7A6FF28448EE74FF0A4
:10D69000FF308BE77CB50022019200926B4601AA15
:10D6A00001F02FFD0B4D012490B1401C0FD0FDF770
:10D6B000AFFC0199884202DB009A904206DDB1F589
:10D6C000800F04D204490098884200D32C707CBD9E
:10D6D0002C707CBDA0040020FFFF3F002DE9F0432B
:10D6E0008BB00446129F90461E46012007901F20D3
:10D6F0000690634A204601F095FD8146394601A80F
:10D70000FDF77CFC0022114608A800F055F940F214
:10D7100039105C49784301EB400408AB01AA41464B
:10D72000204600F0C4F80546B9F1000F06DC317B55
:10D7300060190123002200F00DFE8BE0307830B13B
:10D74000317B60190123042200F004FE82E04C4882
:10D750000088092874D2DFE800F033481C735D7339
:10D760007373050006AA07A94548FDF74DFF28B1C8
:10D77000317B60190F22FDF70CF96BE09DF8180062
:10D780000090317B60199DF81C300F2200F0FDFDE8
:10D7900060E006AA07A93A48FBF779FB28B1317B7C
:10D7A00060190F22FDF7F5F854E09DF8180000907D
:10D7B000317B60199DF81C300F2200F0E6FD49E036
:10D7C0002F48FAF799FE28B1317B60190F22FDF737
:10D7D000E0F83FE09DF818000090317B60199DF85B
:10D7E0001C300F2200F0D1FD34E02548FBF7C7F8CC
:10D7F00028B1317B60190F22FDF7CBF82AE09DF8A4
:10D8000018000090317B60199DF81C300F2200F049
:10D81000BCFD1FE01A48FCF7C9F828B1317B60193C
:10D820000F22FDF7B6F815E09DF818000090317B47
:10D8300060199DF81C300F2200F0A7FD0AE0FFE7F9
:10D840009DF818000090317B60199DF81C300F2264
:10D8500000F09BFD2B18224608A940460097FDF7D3
:10D86000B0FB0BB0BDE8F08310B504460120A478EE
:10D870008C4204D00020022111700921197010BDC2
:10D8800078B60020E8B8002000280FD000290DD07D
:10D890000A7802704A7842708A788270CA78C270B8
:10D8A0008A888280CA88C280097A017270472DE90D
:10D8B000F04705460E46174698460024A146002D1F
:10D8C00077D0B8F1000F74D098F8000028700020CD
:10D8D000687098F8020008B1802068702EB1308915
:10D8E00018B1687840F0200068703FB1388928B1DD
:10D8F000B87A18B1687840F00800687098F80100AC
:10D9000018B1687840F00400687098F803106878DF
:10D9100001F00301084368700224C6B13189B1B136
:10D92000A81CFFF769FD801CB17A441C2954B07A09
:10D9300050B90CE006EB0900C17A2046641C29545A
:10D9400009F1010909F0FF09B07A4845F2D8C7B1D9
:10D950003989B1B1B87AA0B12819FFF74DFD20443B
:10D96000B97A441C2954B87A58B1002006E0391815
:10D97000CA7A2146641C6A54401CC0B2B97A8142FA
:10D98000F5D82EB1308918B198F808002855641CD4
:10D9900098F8020068B198F804002855641CB8F89B
:10D9A0000400802805D3B8F806102819FFF724FDD5
:10D9B00004442046BDE8F08700280BD041700121C7
:10D9C0000170002181704FF480738380C180C27028
:10D9D000FF21017270472DE9FC5F05468846174616
:10D9E000994600240026A246CDF804A0CDF800A058
:10D9F000002D70D0B9F1000F6DD0287889F80000A3
:10DA00006878C00989F802006878C0F3800089F856
:10DA10000100687800F0030089F8030002246878A8
:10DA20004FF0FF3B800623D5A81C6946FFF7E9FCB1
:10DA3000801C441C285CB8F1000F05D0BDF8001014
:10DA4000A8F8081088F80A0008B307280DD9584626
:10DA500000F07AB82146641C695CB8F1000F02D06E
:10DA600008EB0602D172761CF6B28642F2D30EE0C3
:10DA7000B8F1000F0BD0A8F808A088F80AA008EBAE
:10DA8000060080F80BA0761CF6B2072EF7D3687854
:10DA900001072C4820D501210170281901A9FFF7A1
:10DAA000B0FC2044441C295C1FB1BDF8040038813F
:10DAB000B97229B3072901D95846C9E7002007E000
:10DAC0002246641CAA5C0FB13B18DA72401CC0B23B
:10DAD0008842F5D314E02EE097B180F800A0388991
:10DAE000A0F57F41FF3901D0A7F808A087F80AA068
:10DAF0000020391881F80BA0401CC0B20728F8D3C9
:10DB0000BDF8000028B12046641C285C89F8080094
:10DB100001E089F808A099F8020068B12046641C69
:10DB2000285CA9F8040080280AD3281909F1060105
:10DB3000FFF767FC044403E04FF48070A9F8040089
:10DB4000204685E7A40200203CBCBDE8C09FF0B59C
:10DB500087B005460C4617461E46314602A8FDF71B
:10DB60004DFA31462046FDF744FA00221146384668
:10DB7000FFF722FF3B4602AA21462846FFF797FE01
:10DB80000446FDF764FA0646FDF742FA01462819F5
:10DB900003234FF41672009601F05EF9204407B09B
:10DBA000F0BD30B589B005460C46234601AA04A94C
:10DBB0002846FFF7CCFF03462A4601A904A8009493
:10DBC000FDF7FFF909B030BDF0B587B005460C9FF1
:10DBD00014461E462046FEF7A1FF394602A8FDF76F
:10DBE0000DFA002211463046FFF7E6FE334602AA40
:10DBF00021462846FFF75BFE0446FDF728FA064655
:10DC0000FDF706FA0146281903234FF41672009611
:10DC100001F022F92044C2E730B589B00546144628
:10DC200001AB04AA28460094FFF7CEFF03462A461C
:10DC300001A904A80094FDF7C4F9C3E72DE9F04356
:10DC400089B00746884691461D46294601A8FDF73A
:10DC5000D5F90022114606A8FFF7AEFE40F23910B2
:10DC60003049684301EB400406AB01AA394620461F
:10DC7000FFF71DFE0646A0194A46414601F0BAF9D3
:10DC80003318224606A938460095FDF79AF909B0DF
:10DC9000BDE8F08370B586B005460E4614462146B1
:10DCA00001A8FDF7A6F923463246294601A8FFF749
:10DCB000C5FF06B070BDF0B587B006460F461546E5
:10DCC000294602A8FDF795F90020ADF810009DF84F
:10DCD0000C008DF800009DF80B008DF801009DF8F8
:10DCE0000A008DF802009DF809008DF803009DF8E8
:10DCF0000E008DF804009DF80D008DF80500002140
:10DD000002AC6A466318505C5870491C0629F9DB5E
:10DD10002B463A46314602A8FFF790FF07B0F0BD08
:10DD20008CE7B7E7E8B8002070B5CCB0044604F043
:10DD30000DF98DF80400A07801AE5E2802D0C2284B
:10DD40000CD030E003208DF80500E088000A8DF843
:10DD50000800A0798DF80900062524E02088C01F5E
:10DD6000022815DD10208DF80500E088000A8DF8E6
:10DD70000800A0798DF809002078C01F8DF80A00EE
:10DD80002288F849D21FF01D02F024FB25880AE002
:10DD900006208DF80500F34801788DF808104078CA
:10DDA0008DF80900062520798DF80600E0788DF8B9
:10DDB0000700E9B201A809F0DBFD010A71557119EC
:10DDC000487001A904200BF0F3F901A9042009F01F
:10DDD0005BFF4CB070BD70B5044616460020002CA9
:10DDE00025D03020207061701220A0703288E01C95
:10DDF0000021FCF7AFFBC51C601901217268FCF71C
:10DE0000A9FB01460D4460190221FBF7B0FF054450
:10DE1000002004E0B168095C61556D1C401CF1688C
:10DE20008142F7DC60190221FBF7B4FF284470BD82
:10DE300070B5054616460020002D20D032882846B1
:10DE40000021FCF787FB0446281901217268FCF7C2
:10DE500081FB01460C4428190221FBF788FF04448A
:10DE6000002104E0B068405C2855641C491CF0683F
:10DE70008842F7DC28190221FBF78CFF204470BD93
:10DE800010B50A460021002809D010210170042194
:10DE9000417040F25621801CFFF7CAFF811C0846E2
:10DEA00010BD2DE9F84305460E461446002000211A
:10DEB0000091002E0AD0002C08D028466A46FCF7B4
:10DEC0001DFB4FF0FF38002802DA4046BDE8F8831A
:10DED000074600982080E8196A460121FCF70EFBEE
:10DEE000002801DA4046F1E7074400986060E8192D
:10DEF0000221FCF74BF838B17F1CE819A060F01B39
:10DF0000401EE0603046E1E74046DFE770B5154669
:10DF10000022541E002803D006781EB1204670BD92
:10DF2000204670BD86782E70C578122D01D020460F
:10DF300070BD042905D9091F001D1A46FFF7B1FF5E
:10DF40000246104670BD2DE9FF4FADF22C5D0E4626
:10DF5000934698464FF41A742146B0A802F053FA3B
:10DF6000214616A802F04FFA4FF0000ACDF848A05B
:10DF7000CDF84CA0CDF850A0CDF854A0CDF838A0E5
:10DF8000CDF83CA0CDF840A0CDF844A000254FF03E
:10DF9000000900240EAB744A3146DDF82C05FFF76A
:10DFA000B5FF0AAA0BA91098FBF740FF9DF82C10AB
:10DFB000062921D1109A811C545C8DF832401099A9
:10DFC0000B460A5C411C595C02EB0121ADF8301094
:10DFD000109AC11C515C8DF83310109A011D515CD0
:10DFE0008DF83410109A411D109B525C811D595CB4
:10DFF00002EB0121ADF83610BDF83810ADF848102D
:10E000000F991391584E07217170584F642C20D9E5
:10E01000A6F802A0C22C02D0C62C03D101E0514DBB
:10E0200000E0534D9DB3C22C02D0C62C0DD044E06D
:10E030001099BDF83020C01D0144D21F284602F0BF
:10E04000C9F90CA8FFF770FE37E0494809F0E6FC73
:10E0500033E0BDF836104FF6FF7000EA41007080E3
:10E06000B0F5FA7F0ED8020A7A7038709DF8320047
:10E07000B8709DF83300F8709DF8340038717971EC
:10E08000080AB8715E2C03D0622C09D105E014E0B7
:10E090000CA8FFF749FE334D02E007F051FC344D68
:10E0A0002DB1707872883844294602F093F9B0AAED
:10E0B0002E490620FFF7D4F88146B9F1000F0FD0A2
:10E0C0004FF4F071294802F09EF9B0A92748FEF7F5
:10E0D0007DFD1497159012A9DDF82C05FFF7D0FEF1
:10E0E000414602A8FCF78AFF0022114607A8FFF765
:10E0F00063FC40F239101F4908FB00F001EB4004BB
:10E1000007AB02AA59462046FFF7D1FB0546601926
:10E1100012AA3178FFF75FFE2B18224607A958464E
:10E12000CDF80080FCF74DFF0DF23C5D00F0F8B833
:10E1300070B500235C1E002804D00578102D03D094
:10E14000204670BD204670BD4578042D01D0204684
:10E1500070BD022904D9891E801CFFF7A2FE034668
:10E16000184670BD588B0020A2040020CCBD0020B2
:10E170004C870020E8B8002070B504460E461546CE
:10E180000020002CEDD020704FF41671FBF740FDFD
:10E190006070A6701220E0704FF41571201D2A46A1
:10E1A000FFF746FE001DDCE72DE9F0410446069E20
:10E1B00090461F460020002C39D0502020706170FE
:10E1C0001220A070E01C0021FBF7D1FD0546ED1CDC
:10E1D00060194146FCF70DFA054460193946FCF711
:10E1E00008FA054460190021FBF7D4FD0544328884
:10E1F00060190121FCF7AEF905446019022172682B
:10E20000FCF7A8F9054460190321FBF7B0FD0544AC
:10E21000002004E0B168095C61556D1C401CF16888
:10E220008142F7DC60190321FBF7B4FD2844BDE807
:10E23000F0812DE9FE4304460A9E0F46914698461A
:10E2400000250020029001900090002F64D0002E45
:10E2500062D020460021FBF799FEB0B3601C01AAF2
:10E2600002A9FBF7E3FD451C9DF80800092802D030
:10E27000002000F058B860196A460199FCF795F93A
:10E280000544B9F1000F02D0009889F80000601928
:10E2900001AA02A9FBF7CAFD05449DF80800092858
:10E2A00001D00020E5E760196A460199FCF77DF985
:10E2B0000544B8F1000F02D0009888F800006019FA
:10E2C0000021FBF779FE58B16D1C60196A460121E7
:10E2D000FCF714F94FF0FF38002803DA4046C8E78E
:10E2E0000020C6E705440098308060196A46022184
:10E2F000FCF704F9002801DA4046BAE70544009823
:10E30000706060190321FBF741FE38B16D1C601984
:10E31000B060781B401EF0602846AAE74046A8E798
:10E3200030BCBDE8C08F06BCBDE8F88301460020C4
:10E330003339052905D2DFE801F0030507090B0091
:10E340000120704702207047032070470420704767
:10E350004020704710B50024002808D013B1712365
:10E36000037001E070230370417082700324204623
:10E3700010BD10B50024002905D00AB10178117034
:10E380000BB140781870204610BD70B50446049E4D
:10E390000020002C0DD0502020706170A270E01C75
:10E3A0001946FCF726F9C51C60193146FCF721F91E
:10E3B000284470BDFEB5044617461E4600200025C1
:10E3C00002950195009500290AD0204601AA02A9CC
:10E3D000FBF72CFD05469DF80800092801D0002018
:10E3E000FEBD60196A460199FCF7DFF805440FB1DC
:10E3F00000983870601901AA02A9FBF717FD0544BF
:10E400009DF80800092801D00020FEBD60196A4669
:10E410000199FCF7CAF82844002EF6D00099317013
:10E42000FEBD70B5DDE90456002402290CD90AB1FD
:10E43000047814700BB142781A7033462A46891E4C
:10E44000801CFFF7B7FF0446204670BD81070CD142
:10E450006421B0FBF1F201FB120141B94FF4C87124
:10E46000B0FBF1F201FB120008B10020704701205F
:10E47000704730B58DB005460C463422F7496846E2
:10E4800001F0A8FF0023022C05D12846FFF7DEFF8C
:10E4900008B11D2304E0601E0B2801D81DF82430AC
:10E4A0000DB0184630BD70B50646144600253046FE
:10E4B000FFF7DFFF40F26C718E4204D318B114B144
:10E4C000844200D80125284670BD10B500210028DF
:10E4D00005D0C27881780088FFF7E5FF014608463D
:10E4E00010BD2DE9F04180460E46174600243A46FD
:10E4F00031464046FFF7D7FF58B1012506E02946CF
:10E500004046FFF7B6FF04446D1CEDB2B542F6D3AA
:10E510003C442046BDE8F0812DE9F0470446894699
:10E5200016461F4601254FF0000806E029464846DA
:10E53000FFF79FFF241A6D1CEDB229464846FFF7EE
:10E5400098FFA042F2D308EB0400C0B206B13570C8
:10E55000002F00D03870BDE8F0872DE9F041054666
:10E560000E46174600243A4631462846FFF79BFFE1
:10E57000A0B140F26C7308E004F26D141846FFF786
:10E5800065FF00B1641C5B1C9BB2AB42F4D33A46FE
:10E5900031462846FFF7A5FF0444641E2046B9E72C
:10E5A00010B5FFF7DAFF0721B0FBF1F201FB120013
:10E5B000401C10BD10B50446084611461A46002CF2
:10E5C00005D02080A170E270FFF7EAFF207110BD36
:10E5D0007CB50D4614460023019300936B4601AAB7
:10E5E0002946FFF799FF9DF800309DF80420294641
:10E5F0002046FFF7DFFF7CBD10B50021002805D0C5
:10E60000C27881780088FFF76CFF0146084610BD8C
:10E6100010B50021002805D0C27881780088FFF766
:10E620009CFF0146084610BD2DE9F05F04460F46E9
:10E630009046994640F26C7501264FF0010A40F26F
:10E640006D134FF4B67B0EE02846FFF7FFFE08B1CE
:10E650009C4212D0A4F26D142846FFF7F7FE00B1D9
:10E66000641E6D1CADB25C45EED806E0314628460E
:10E67000FFF7FFFE241A761CF6B231462846FFF754
:10E68000F8FEA042F2D90AEB0400C0B207B13D8007
:10E69000B8F1000F01D088F80060B9F1000F01D087
:10E6A00089F8000000F076BA3EB50C4600220292CE
:10E6B000019200926B4601AA02A9FFF7B5FF9DF8EF
:10E6C00000309DF80420BDF808102046FFF772FFC7
:10E6D0003EBD002100280CD00278182A09D24278C9
:10E6E0003C2A06D282783C2A03D2C078642800D221
:10E6F00001210846704710B50C46FFF7E6FE28B129
:10E700002046FFF7E6FF08B1012010BD002010BD34
:10E7100002460020002A0ED000290CD010880B8859
:10E72000C01A002807D190788B78C01A002802D12F
:10E73000D078C978401A704702460020002A13D0CA
:10E74000002911D010780B78C01A00280CD150780D
:10E750004B78C01A002807D190788B78C01A00280F
:10E7600002D1D078C978401A704730B504460D46BA
:10E7700029462046FFF7CCFF002804D1A91DA01D83
:10E78000BDE83040D8E730BD30B502460020002A51
:10E790001CD000291AD0148840F66B05AC4203D077
:10E7A0000B88AB4200D0E01A00280FD19378FF2BE2
:10E7B00003D08C78FF2C00D0181B002806D1D2780B
:10E7C000FF2A03D0C978FF2900D0501A30BD10B5F8
:10E7D00002460020002A23D0002921D01478FF2CE3
:10E7E00003D00B78FF2B00D0E01A002818D1537803
:10E7F000FF2B03D04C78FF2C00D0181B00280FD122
:10E800009478FF2C03D08B78FF2B00D0E01A0028DF
:10E8100006D1D278FF2A03D0C978FF2900D0501A38
:10E8200010BD30B504460D4629462046FFF7ACFF23
:10E83000002804D1A91DA01DBDE83040C7E730BDA8
:10E84000002809D0002907D00A8802808A788270BF
:10E85000CA78C2700979017170470000F0C10108DF
:10E860000028F9D00029F7D00A7802704A7842705F
:10E870008A788270C978C170EEE710B504460B46FD
:10E88000991DA01DFFF7ECFF2046BDE8104019467A
:10E89000D6E710B5029C002803D001704270837047
:10E8A000C47010BD0029D7D0002AD5D00028D3D0FD
:10E8B000137883715378C37193780372D27842725C
:10E8C0000A8802808A788270CA78C27009790171D8
:10E8D000C2E72DE9F04106AD044695E8E00108469F
:10E8E00011461A46002C0AD02080A170E270FFF772
:10E8F00057FE2071A571E671277284F8098009E638
:10E900004FF461635843C1EB011100EB81001044E7
:10E91000A2E7C0EB001001EB80009DE770B54FF45B
:10E920006164B0FBF4F4E4B26FF0E005654300EB22
:10E9300005103C25B0FBF5F5EDB2A5EB051600EB97
:10E940008600002900D00C7002B11570002B00D099
:10E95000187070BD10B50021002805D0827841786C
:10E960000078FFF7CDFF0146084610BD10B5002125
:10E97000002804D041780078FFF7CBFF014688B229
:10E9800010BD2DE9F04104460F46227AE179A079C5
:10E99000FFF7B6FF3C21B0FBF1F52046FFF738FE4C
:10E9A00002464FF4B46197FBF1F01618A0EB00108B
:10E9B00000EB400007EB4010002812DA4042A8426A
:10E9C00004D9761EC0F5B460284414E0281AB0FBC0
:10E9D000F1F10E44A1EB011101EB410100EB4110FB
:10E9E00009E02844B0FBF1F10E44A1EB011101EB69
:10E9F000410100EB4110C0EB001080000023E21D3C
:10EA0000A11DFFF78BFF21463046BDE8F0414BE6E4
:10EA1000002100281AD00288A2F500636B3B15D1B3
:10EA20008278FF2A12D1C278FF2A0FD10279FF2AF9
:10EA30000CD18279FF2A09D1C279FF2A06D1027A44
:10EA4000FF2A03D1407AFF2800D10121084603E7BD
:10EA50000021002817D00288A2F500636B3B11D07B
:10EA600082780C2A0ED8C2781F2A0BD88279FF2A06
:10EA700008D0C279FF2A05D0027AFF2A02D0407A54
:10EA8000FF2800D101210846E6E6002806D040F61E
:10EA90006B010180FF218170C1700171DCE60028EB
:10EAA00004D0FF21017041708170C170D4E600B5BF
:10EAB0000246002A06D01046FFF7E7FF901D5DF8DA
:10EAC00004EBECE700BD70B505460E460020002DB6
:10EAD0000BD0002E09D031462846FBF7F8FE04463D
:10EAE0002819B11DFBF77CFE204470BD2DE9F041D3
:10EAF00004460F4616460020002C11D0002E0FD0E1
:10EB000020463946FBF733F9054660193146FFF7D1
:10EB1000DAFF01460D4460193946FBF73BF92844FA
:10EB2000F8E42DE9F04105460F4628463946FBF743
:10EB300004FF411C4FF0FF3608D004462819B91DC8
:10EB4000FBF782FE411C03D02044E3E43046E1E4BD
:10EB50003046DFE42DE9F04105460E4614462846CE
:10EB60003146FBF713FA4FF0FF3768B1681C2146B6
:10EB7000FFF7D7FF411C09D0441C28193146FBF789
:10EB80001BFA28B1601CC5E43846C3E43846C1E42A
:10EB90003846BFE430BCBDE8C09FF0B587B007463B
:10EBA0000C4615460026069605960496039603A87D
:10EBB000009004AB05AA06A9384600F072F9401C83
:10EBC00018D0DDE905102A46FAF751FB2978012211
:10EBD000E4B2012910D006290CD1BDF80C0094280C
:10EBE00022D0CDE901263B4600943A4629460698B4
:10EBF00008F05BFD07B0F0BDBDF80C00942809D00B
:10EC0000CDE9004602966A783B462946069808F008
:10EC10004CFDEFE7CDE9004602926A783B46294673
:10EC2000069808F042FDE5E7CDE9004202923B4636
:10EC30003A462946069808F038FDDBE710B586B05D
:10EC400014460021059104910391029102A90091BB
:10EC500003AB04AA05A900F024F9002804DDDDE9CE
:10EC600004102246FAF7A3FB06B010BD2DE9FE43BF
:10EC700080460C4615461F464FF0FF36208809286F
:10EC800062D2DFE800F03745296153616161050018
:10EC90006C496068884202D1FCF7BAF9606060682C
:10ECA000FCF7CDF9002853D02289A2F58070733883
:10ECB00008D0CDE900574046E3686168FCF725FAC3
:10ECC000064645E000200290019000906A4601A9A6
:10ECD00002A8FCF7F1FC3BE06068F9F761FF20B3A4
:10ECE000CDE9005722894046E3686168F9F7C2FF21
:10ECF00006462DE06068F9F70BFBB0B1CDE900578F
:10ED000022894046E3686168F9F75FFB06461FE029
:10ED10006068F9F7A1FC40B1CDE90057228940466F
:10ED2000E3686168F9F716FD064611E06068FAF7D6
:10ED3000B1FC68B1CDE9005722894046E3686168BB
:10ED4000FAF7EDFC064603E0012028701F2038701A
:10ED5000304600F07BB82DE9F04F93B00746DDF860
:10ED60007090884692461E46012008901F2007900A
:10ED7000494602A8FCF742F90022114609A8FEF70D
:10ED80001BFE40F23910304909FB00F001EB400452
:10ED900009AB02AA51462046FEF789FD05463078A8
:10EDA00030B1317B601901230422FFF7D3FA36E03A
:10EDB0000CAA4146384600F0DCFD002806DA317B1B
:10EDC000601901230022FFF7C5FA28E004EB0508CB
:10EDD000317B0CAA404600F035FE834605EB0B0064
:10EDE000204407AB08AA0CA9FFF740FF07463800EC
:10EDF00008D4E8195844204400F04BFE0BEB0701FF
:10EE000008440CE017F1020F14D09DF81C0000908C
:10EE1000317B40469DF820300C22FFF7B6FA2B18C4
:10EE2000224609A95046CDF80090FCF7CAF813B065
:10EE300000F00FB8317B404601230422FFF78AFA25
:10EE4000EDE70000FFFF3F00E8B8002006BCBDE88A
:10EE5000F88330BCBDE8C08F2DE9F0410446069E22
:10EE600090461F460020002C19D010202070002052
:10EE700060700A46A01C0821FBF7F8F9851C601990
:10EE80004146FBF784FB01460D4460193946FBF708
:10EE9000B0FB054460193146FBF779FB2844BDE817
:10EEA000F0812DE9F04786B00446DDF838900E4633
:10EEB0001746984600200590049003900290019018
:10EEC000204602AA03A9FAF7B1FF05469DF80C00F7
:10EED0004FF0FF3A0C2803D0504606B0BDE8F0874B
:10EEE000601904AA05A9FBF774F90544BDF81400DC
:10EEF000082801D05046F0E70EB104983060601940
:10EF000002AA03A9FAF792FF05449DF80C00022813
:10EF100001D05046E1E7601901AA0299FBF7CAFA4D
:10EF200005440FB101983860601902AA03A9FAF7E5
:10EF30007DFF05449DF80C00092801D05046CCE720
:10EF4000601901AA0299FBF730FB054401980428D7
:10EF500001D35046C1E7B8F1000F01D0C8F8000056
:10EF6000601902AA03A9FAF761FF05449DF80C0095
:10EF7000022801D05046B0E7601901AA0299FBF7B8
:10EF800099FA29180198B0F5803F01D35046A4E7BB
:10EF9000B9F1000F01D0A9F8000008469DE7000074
:10EFA000F0B589B015460E9E1F46314601A8FCF704
:10EFB00025F80022114606A8FEF7FEFC06AB01AAC2
:10EFC00029460B48FEF773FC044640F23910084A04
:10EFD000604302EB4000397B092200F092FC2318C9
:10EFE000034A06A928460096FBF7EBFF09B0F0BDDF
:10EFF000E8B8002070B5044616460020002C17D053
:10F0000010202070082060700220420591420FD22B
:10F01000002E0DDB96420BDA0A46A01C0021FBF7FE
:10F0200099FA851C601932460121FBF793FA2844AE
:10F0300070BD2DE9F041044616461F460020002C05
:10F0400020D01020207008206070022042059142DC
:10F0500010D2002E0EDB96420CDA0A46A01C0021CC
:10F06000FBF778FA851C601932460121FBF772FA2A
:10F0700001466818DF212154401CFD212154401C09
:10F080002754401CBDE8F0812DE9F04389B080464B
:10F09000894615464FF0FF36294601A8FBF7AEFF1B
:10F0A0000022114606A8FEF787FC40F239103549C8
:10F0B000684301EB400406AB01AA41462046FEF737
:10F0C000F6FB0746E0194B4632463146FFF7B1FFE3
:10F0D0003B18224606A940460095FBF772FF09B08F
:10F0E000BDE8F08330B585B005460C46214668463C
:10F0F000FBF77FFF224629466846FFF7C5FF05B0AC
:10F1000030BD2DE9FE43044617461E46002000226E
:10F1100002920192009200290BD0204601AA02A976
:10F12000FAF784FE05469DF808004FF0FF3910B14C
:10F13000484600F029B860196A460199FBF7BAF908
:10F14000054400984FF48008404501D207B138606B
:10F15000601901AA02A9FAF769FE05449DF80800A2
:10F16000012801D04846E4E760196A460199FBF797
:10F17000A1F9284400994145DBD2002ED9D0316055
:10F18000D7E70000E8B8002006BCBDE8F8832DE909
:10F19000F04104460F4615460026002C3FD00020C3
:10F1A00020704FF41671FAF733FD6070A7700F20CE
:10F1B000E0702A88201D00216B68FBF745F8061DCA
:10F1C0002A89A0190121FBF722FA01460E44EA68B8
:10F1D000501C04D0A0190221FBF7BCF90644A01969
:10F1E0000321FAF7C4FD3118002004E02A180B1897
:10F1F000127CE254401CD5F868228242F6DCD5F835
:10F2000068024618A0190321FAF7C4FD064495F8D0
:10F210006C2222B1A0190421FBF79CF90644304668
:10F22000BDE8F0812DE9F04786B0054688461446D2
:10F230000027002005900490039002900190002682
:10F24000B8F1000F71D0002C6FD028460021FAF7DA
:10F2500073FE4FF0FF39B0B1681C221D03A9FAF705
:10F26000B8FF471CBDF80C002080E81904AA05A9C6
:10F27000FAF7DCFD07449DF81400012805D0484644
:10F2800006B0BDE8F0874846FAE7E81902AA0499F3
:10F29000FBF78BF9074402982081E81904AA05A915
:10F2A000FAF7C4FD9DF81410022912D0C4F80C908E
:10F2B000E81982460321FAF769FEA0B10298A8EB8B
:10F2C000070182B25046FDF774FFC4F868027F1C44
:10F2D00010E00744E81901AA0499FBF7EBF807448A
:10F2E0000198E060E4E74846CAE7B819A119285C2C
:10F2F0000874761CD4F86802B042F6DCD4F86802D0
:10F300000744E8190321FAF757FE78B17F1C102053
:10F3100084F86C02474519D2E81904AA05A9FAF73E
:10F3200085FD9DF81410042903D00FE06FF0010053
:10F33000A6E73844284401AA0499FBF7BBF807461E
:10F340000198411E0F2903D884F86C02384697E7CC
:10F350006FF0040094E7000070B54FF0FF3344688D
:10F36000C5684669082904D0692918D050291CD0DD
:10F3700020E0A24203D2006850F822301AE061195E
:10F38000914204D9111B806850F8213012E08C1989
:10F3900094420FD9511A006950F821300AE0A24274
:10F3A00008D2006850F8223004E0AA4202D28068F5
:10F3B00050F8223098B270BD0022082904D0692983
:10F3C00008D0502908D008E0C2684168406911445B
:10F3D0000A1802E0426800E0C268104670472DE952
:10F3E000F04F89B081468A4616461C46DD48218981
:10F3F000E26800F0D8FE05462B465246D9494846F9
:10F400000096F8F7DFFE36276FF0010878B3012089
:10F410008DF820001F208DF821002088ADF808000D
:10F42000606803902089ADF81000E0680590CD4831
:10F4300006904FF41670079002A8FCF7A8F9002870
:10F4400022DA811C19D0C11C17D09DF821209DF80B
:10F450002010C44800F0DDFE83460AEB05025B463F
:10F46000C04948460096F8F7ADFE50B11AE0FFE7F4
:10F470006774404609B000F07BB99DF821106174B3
:10F48000F8E767744046F5E70AEB05010A18921C95
:10F49000B2420ADA01EB09030246B249184600F00B
:10F4A00098FE834605EB0B00E4E767744046E1E70E
:10F4B0002DE9FF4F97B081468A4600260024002799
:10F4C0000EA82499FBF79AFD0022114613A8FEF717
:10F4D00073FA249840F239114843A34913AB01EB66
:10F4E00040000EAA16901999FEF7E1F908901A98B3
:10F4F000007820B136208DF83500A71E7EE01A98DE
:10F50000089A017B16988518284600F02FFE0446BD
:10F51000AAEB060109EB060009AA00F087FD002806
:10F5200006DB304486B2BDF82400082802D008E08B
:10F53000074663E08D490A98884202D1FBF768FDCF
:10F540000A9009A9874800F01CFE03464FF4167084
:10F550000090284622468349F8F734FE80B258B11D
:10F560000444AAEB060109EB060009AA00F09EFD7F
:10F57000002807DA074641E036208DF835006FF0A5
:10F5800001073BE0304486B2BDF82C1008293ED07C
:10F5900069293CD050293AD0A1F58070733836D013
:10F5A000A1B2284609AB4FF41672FFF718FF0028E6
:10F5B0007BDD044409EB06000121FAF7FDFC00287D
:10F5C000CFD0761CB6B2674800F040FE03464FF439
:10F5D00016700090284622466249F8F7F3FD80B283
:10F5E00000287BD00444564592D31A988068A042E4
:10F5F00004DA36208DF835006FF00107002F05D0B2
:10F60000B81C79D0781C6BD0FF1C6AD09FE04FF0FB
:10F6100000080C98401C2FD052480C9A00F0C3FDF3
:10F6200083464FF4167828465B4622464D49CDF86E
:10F630000080F8F7C7FD80B290B15C44322202210D
:10F64000484800F0E6FD834628465B462246454989
:10F65000CDF80080F8F7B6FD80B238B15C44A9E778
:10F6600036208DF835006FF00107C7E736208DF89A
:10F6700035006FF00107C1E70191BDF8240002A930
:10F68000FCF7A6F802A80199FFF796FE83465FEA09
:10F690000B0020D1A1B2284609AB4FF41672FFF738
:10F6A0009EFE002802DD044484E71DE00746A5E72E
:10F6B000424602A80199FFF74FFEADF82C00A1B217
:10F6C000284609AB4FF41672FFF789FE002809DDC2
:10F6D000044408F10108D845EAD36BE706E00BE0E3
:10F6E00019E027E0074689E7074687E736208DF8C7
:10F6F00035006FF0010781E79DF83500FEF716FE33
:10F7000002461A98089B017B169818440123FEF7BD
:10F7100021FE04461BE09DF8350000901A98089AD7
:10F720009DF83430017B169810440E22FEF72DFE12
:10F7300004460CE09DF8350000F0C3F802461A9824
:10F74000089B017B1698184400F0DBF804460898E3
:10F7500023182498009013A9169A1998FBF731FCE6
:10F760001BB088E6ACBF0020E8B80020FFFF3F00D8
:10F7700030BCBDE8C08F00002DE9F04FADF5277D0E
:10F780000646DDF8C0A28846934699460024002725
:10F790000120A6901F20A59099F80000002804D011
:10F7A00036208DF89202A51E36E0A8EB040081B247
:10F7B000301909AA00F0EBF90546002D2BDD601980
:10F7C000441C30440121FAF7E1FB08B3A8EB040024
:10F7D00081B2301909AA00F027FA0546002D11DD83
:10F7E0002C44A5AAA6A909A8FBF70EFF38B1301929
:10F7F0000121FAF7E1FB38B10120641C05E0012783
:10F80000BD1E09E0012707E000200128DED11FB955
:10F810004445CADB00E00127514601A8FBF7EEFB97
:10F820000022114606A8FEF7C7F840F23910224917
:10F830000AFB00F001EB400406AB01AA5946204642
:10F84000FEF735F80646002027B3A91C04D0691C32
:10F850000ED0ED1C13D022E09DF89202FEF766FD5B
:10F86000024699F80C10A0190123FEF773FD16E06B
:10F8700099F80C10A01909AA00F0DEFA0FE09DF823
:10F88000920200F01EF8024699F80C10A01900F040
:10F8900038F804E099F80C10A01900F0C2FA3318F7
:10F8A000224606A95846CDF800A0FBF78AFB0DF5C5
:10F8B000277D00F003B80000E8B8002030BCBDE8A8
:10F8C000C08F014600203B390A2907D2DFE801F04A
:10F8D0000507090B0D0F11131517012070470220A2
:10F8E00070470320704704207047052070470620AA
:10F8F0007047072070470820704709207047402054
:10F9000070470023002804D0602303704170827088
:10F9100003231846704710B50024002905D00AB10A
:10F92000017811700BB140781870204610BD70B589
:10F9300004460D4616460020002C19D0207040F2D7
:10F94000C451FAF765F96070A5700C20E0700425C9
:10F950003288B2F5806F05D2201D00217368FAF756
:10F9600073FC051D328960190121FAF750FE284405
:10F9700070BD2DE9F04385B006460F4614460025BC
:10F980000020049003900290019000906FF0020913
:10F99000002C4FD0072F05D23F206076484605B097
:10F9A000BDE8F08330460021FAF7C6FA4FF03E0872
:10F9B000B0B1701C221D02A9FAF70BFC451CBDF862
:10F9C00008002080701903AA04A9FAF72FFA054449
:10F9D0009DF81000012807D084F819804846DEE71A
:10F9E00084F819804846DAE7701901AA0399FAF7F2
:10F9F000DCFD054401982081BD4218D2701903AA8C
:10FA000004A9FAF713FA05449DF8100002280AD158
:10FA1000BD4208D270196A460399FAF74BFD0544B6
:10FA20000098E06006E084F819804846B7E74FF098
:10FA3000FF30E060BD4203D2412060764846AEE729
:10FA40002846ACE770B5044616460020002C1FD0AF
:10FA50003020207061700C20A0703288E01C0021E2
:10FA60007368FAF7F1FBC51C328960190121FAF7B6
:10FA7000CEFD01460D44F268501C04D060190221ED
:10FA8000FAF768FD054460190321FAF770F9284474
:10FA900070BD02460020002A03D003211046FAF769
:10FAA00079B970472DE9F041064617460025002038
:10FAB000002E13D03A463046FFF7C4FF044605E057
:10FAC0003869415D2046641C31546D1C7869A84238
:10FAD000F6DC30190321FAF75DF92044BDE8F08126
:10FAE0002DE9F04186B004460F46154600200590EA
:10FAF000049003900290019000212046FAF71CFA2E
:10FB00004FF0FF38A8B1601C2A1D03A9FAF761FB6A
:10FB1000461CBDF80C002880A01904AA05A9FAF714
:10FB200085F906449DF81400012804D0404606B02B
:10FB3000D4E74046FBE7A01902AA0499FAF735FD7D
:10FB4000064402982881A01904AA05A9FAF76EF9BB
:10FB50009DF8141002290ED0C5F80C80A0190321BD
:10FB6000FAF714FA88B1761CA0192861B81B401E58
:10FB700068613846DBE70644A01901AA0499FAF740
:10FB800099FC06440198E860E8E74046CFE72DE994
:10FB9000FF4706460F46144600200390029001904E
:10FBA00000904FF03F0A6FF00209002E38D0052F69
:10FBB00036D984B3304602AA03A9FAF737F985B2D9
:10FBC0009DF80C004FF03E0808BBAF421FD9781BD0
:10FBD00087B2042F17D3701901AA6946FAF7F9FA08
:10FBE000284485B2BDF80000208001986060781B31
:10FBF00080B220B170190121FAF7C8F960B1284626
:10FC000004B0BDE8F08784F86EA24846F8E784F8AF
:10FC10006E824846F4E703E084F86E824846EFE7D8
:10FC200084F86EA24846EBE72DE9FE4F054689466B
:10FC30001446002002900190009000266FF0020A06
:10FC4000002D72D0B9F1000F6FD0002C6DD0411E85
:10FC5000E160102184F86C12C4F86802284601AAF9
:10FC600002A9FAF7E3F807469DF808004FF03E08AE
:10FC700020B184F86E82504600F01FB9E8196A4638
:10FC80000199FAF792FC074400982081E81901AA2B
:10FC900002A9FAF7CBF807449DF8080001280DD116
:10FCA000E8196A460199FAF705FC07440098E060F4
:10FCB000E81901AA02A9FAF7B9F807449DF8080063
:10FCC00002282ED1E819401EFAF79FF848B37F1E8C
:10FCD0002289A9EB0701E819FDF76BFAC4F868025D
:10FCE0007F1C04E0B819A119285C0874761CD4F8AC
:10FCF0006802B042F6DCD4F86802C619A81901AA55
:10FD000002A9FAF793F806449DF8080002280DD0DE
:10FD1000A819401EFAF782F840B184F86E82504666
:10FD2000AAE784F86E825046A6E715E0A81901AA52
:10FD300002A9FAF77BF806449DF80800032801D0D1
:10FD4000701E99E7A8196A460199FAF7B3FB304487
:10FD5000009984F86C128FE73F2084F86E025046B9
:10FD60008AE770B504460D460020002C09D02070AB
:10FD70004FF41671F9F74CFF6070A5701020E07019
:10FD8000042070BD70B505460020002D0BD0134631
:10FD90000A4600212846FAF757FA04462819012195
:10FDA000F9F7E5FF204470BD02460020002A03D089
:10FDB00001211046F9F7EEBF70472DE9F0410646E4
:10FDC0000F4600240025002E28D03A890021304615
:10FDD000FAF71DFC0446FA68501C04D030190121C2
:10FDE000FAF7B8FB044430190221F9F7C0FF0444C4
:10FDF00004E07819007C3055641C6D1CD7F868024B
:10FE0000A842F6DC30190221F9F7C4FF044497F840
:10FE10006C221AB130190321FAF79CFB2046BDE889
:10FE2000F0810022002805D02022027041701021AC
:10FE3000032281701046704770B5044615460020B5
:10FE4000002C39D05020207061701020A070E01C70
:10FE50000021F9F78CFFC61C95F86D12A019FAF76E
:10FE6000C8FB064495F86E12A019FAF7C2FB0644C7
:10FE7000A0190021F9F78EFF0644A0190121F9F716
:10FE800076FF06442A88A01900216B68FAF7DCF98E
:10FE900006442A89A0190121FAF7B9FB0644EA6849
:10FEA000501C04D0A0190221FAF754FB0644A019F3
:10FEB0000121F9F76FFF304470BD1EBCBDE8E08F33
:10FEC00070B504460D460020002C09D020704FF478
:10FED0001671F9F79DFE6070A5700E20E070042089
:10FEE00070BD70B505460020002D0BD013460A46A4
:10FEF00000212846FAF7A8F9044628190121F9F744
:10FF000036FF204470BD70B5054616460024002D0E
:10FF10000DD00A4600212846FAF779FB0446721CE8
:10FF200005D0281932460121FAF714FB0444204673
:10FF300070BD02460020002A03D001211046F9F7C7
:10FF400029BF70472DE9F0410F4686B08046114623
:10FF50001E46002402A8FFF7B3FF0346224602A96B
:10FF600040460097F8F72EF908B1044654E0002007
:10FF700006B0BDE8F0813288002102A87368FAF764
:10FF800063F90346224602A940460097F8F71AF99A
:10FF900078B10444012102A8F9F7E9FE034622469C
:10FFA00002A940460097F8F70DF920B12518B4686A
:10FFB00022E00020DCE70020DAE72288002102A806
:10FFC000FAF725FB03462A4602A940460097F8F7B0
:10FFD000F9F828B305446268501C0CD0012102A82E
:10FFE000FAF7B8FA03462A4602A940460097F8F7FE
:10FFF000E9F8B8B105442469002CDED1012102A83A
:020000040801F1
:10000000F9F7C8FE03462A4602A940460097F8F7CA
:10001000D9F848B12C18F668002EACD12046A7E7D5
:100020000020A5E70020A3E70020A1E72DE9F84381
:1000300005461446002000220092002D09D0002918
:1000400007D0002C05D0C71E052904D23F206074BC
:100050003846BDE8F88328460021F9F76DFF4FF0D8
:100060003E0878B1681C221D6946FAF7B2F8461CB2
:10007000BDF800002080A8190121F9F787FF28B1F9
:10008000701CE6E784F811803846E2E784F81180B6
:100090003846DEE710B50024002805D021B1012143
:1000A000F9F78AFF00B10124204610BD2DE9FF4772
:1000B00005460F461446002600200390029001904A
:1000C0000090002D50D0EFB3E4B328784FF03E08F5
:1000D00000076FF0020905D484F81180484604B087
:1000E000BDE8F087284602AA03A9F9F79FFE064655
:1000F0009DF80C0018B184F811804846EFE702998A
:100100004FF03F087018B84203D384F81180484676
:10011000E5E7A81901AAFAF748FA064401982081F0
:100120004FF0FF30E060A85D01071DD5C0434007D8
:100130001AD0A81902AA03A9F9F778FE9DF80C10A5
:10014000012900E010E00FD1064402997018B8426E
:1001500003D384F811804846C1E7A8196A46FAF724
:10016000A9F906440098E0603046B8E7002200286C
:1001700005D03022027041700E218170032210469A
:10018000704770B505460020002D0BD00A884B68DB
:1001900000212846FAF758F8044628190121F9F7F2
:1001A000E6FD204470BD70B5054616460024002DBE
:1001B0000DD00A4602212846FAF729FA0446721C95
:1001C00005D0281932460321FAF7C4F90444204621
:1001D00070BD2DE9F04106460F46904600200025EF
:1001E000002E15D030460421F9F7C1FD0446301920
:1001F000B84206D1444406E02046795D641C31547F
:100200006D1C4545F8D330190421F9F7C3FD20448E
:10021000AFE62DE9F04104460F4616460020002CBB
:1002200013D020460521F9F7A2FD0546601939468D
:10023000FAF7DFF9054460193146FAF7DAF90544AF
:1002400060190521F9F7A6FD284492E60246002030
:10025000002A03D001211046F9F79CBD7047F8B57C
:10026000044616461D46002000220092002C1BD09A
:10027000002919D0002E17D0002D15D020460021BE
:10028000F9F75AFE4FF0FF3778B1601C2A466946ED
:10029000F9F79FFF451CBDF800003080601901216F
:1002A000F9F774FE18B1681CF8BD3846F8BD384639
:1002B000F8BD10B50024002805D021B10121F9F7BF
:1002C0007BFE00B10124204610BD2DE9FF47044606
:1002D000884691461E46002500200390029001901A
:1002E0000090002C40D0B8F1000F3DD0B9F1000FC4
:1002F0003AD06EB320784FF0FF37000701D438466C
:10030000EDE6204602AA03A9F9F790FD05469DF8FF
:100310000C00022801D03846E1E6601901AA0299D2
:10032000FAF743F905440198A9F8000045451AD2A7
:10033000605D010717D5C043400714D0601902AAB9
:1003400003A9F9F773FD9DF80C10032901D037605C
:100350000AE0054460196A460299FAF7ABF80544C9
:100360000098306000E037602846B8E62DE9F05F7D
:100370000546002092469B46884606468146402414
:100380001BE0284641464746224600F091FB534673
:100390005A46C01A914110D311461846224600F021
:1003A00078FB2D1A67EB01084F46224601200021F9
:1003B00000F06FFB17EB00094E41201EA4F1010471
:1003C000DFDC484631462A46434600F000B830BCE0
:1003D000BDE8C09F40EA01039B0703D009E008C9BC
:1003E000121F08C0042AFAD203E011F8013B00F8FA
:1003F000013B521EF9D27047D2B201E000F8012B46
:10040000491EFBD270470022F6E710B513460A4694
:1004100004461946FFF7F0FF204610BD30B50446EC
:100420000020034600E05B1C934203D2E05CCD5CFD
:10043000401BF8D030BD00000FB400B58DB010A93E
:1004400009900B9000914FF0FF300A9000200C9023
:1004500005480690054807906A4609A80F9900F0DC
:1004600067FB0DB05DF814FB4D0B01086B0B010829
:100470002DE9FF5F1D464FF0FF3BD5E90146914650
:100480005F464FF00008A9697F1C01988847296AD8
:10049000824688470028F6D1BAF1FF3F0CD024F4F9
:1004A000C064002E19DD600614D5BAF12B0F09D0F7
:1004B000BAF12D0F0ED103E0584604B000F07EB81B
:1004C00044F48064A9697F1C01988847761E82469F
:1004D000002E02DDBAF1300F03D0B9F1000F26D0A3
:1004E00032E0A969761E44F400747F1C01988847A5
:1004F0008246002E05DDBAF1780F06D0BAF1580F0A
:1005000003D0B9F1000F10D01EE0B9F1000F02D0F6
:10051000B9F1100F18D1A969761E24F400747F1C5C
:10052000019888478246102002E0082000E00A2057
:10053000814609E008FB0908A969761E44F40074A5
:100540007F1C019888478246002E05DD49465046AB
:1005500000F0D9FA0028EDDAE96901988847A0058A
:1005600002D46FF00100A8E7E00725D1600613D59B
:10057000600502D5C8F1000000E0404629680A1D68
:100580002A600968220501D5087015E0220701D507
:10059000088011E008600FE02868011D29600068EC
:1005A000210502D580F8008006E0210702D5A0F8D9
:1005B000008001E0C0F8008038467EE730BCBDE82E
:1005C000C09F2DE9F04791460F468046044600261D
:1005D00014F8015B2DB1F7F70FFE0068405DC0070E
:1005E000F6D12B2D02D02D2D18D0641E4A46394647
:1005F000204600F0CBFA27B13968A14201D1C7F8F3
:10060000008071054FF002040BD54042002803DD45
:1006100005F086FE0460A007BDE8F08746F480661A
:10062000E4E70028F8DA05F07BFE04606FF0004094
:10063000F2E72DE9F05F93460F4680460446002618
:1006400005F06EFED0F80090824614F8015B2DB1E3
:10065000F7F7D2FD0068405DC007F6D12B2D02D020
:100660002D2D1AD0641E0021CAF800105A463946B2
:10067000204600F08BFA014627B13868A04201D12C
:10068000C7F80080DAF80000022809D0CAF8009004
:10069000700505D5484200F005B846F48066E2E7EB
:1006A0000846F8E730BCBDE8C09F2DE9FE4F804604
:1006B00081EA0300C00F0C46009021F0004123F0B6
:1006C0000045B8EB0200A94105D2404621469046BC
:1006D0001C460B46024623F00040104347D0270D2E
:1006E000C7F30A00C3F30A510290401A0190402850
:1006F0006BDAC3F3130040F4801B0098924620B1DC
:100700000023D2EB030A63EB0B0B01985946C0F1AF
:100710004002504600F0BDF906460D465046594687
:10072000019A00F0D5F910EB08006141002487EA36
:10073000115284EAE7731A4340D0009A62B3019AD7
:10074000012A4FEA075215DC001B61EB02014FF052
:10075000004202EA0752CDE90042001C41F5801137
:1007600032462B4600F0F8FA03B000F045B8404698
:100770002146F9E7001B61EB0201001C41F58013E3
:1007800000185B412018A2F5001747EB030140EA6F
:10079000D570B6196D4111E06D084FEA360645EA8D
:1007A000C0754FEA0752001B61EB0201001C41F5C6
:1007B000801149084FEA30000019514132462B465A
:1007C00003B000F01CB800F0B8BA00980122400055
:1007D0000023D0EB020263EBE073009821464FEA5E
:1007E000E074B8EB000061EB0401E9E783F000433B
:1007F0005BE781F0004158E730BCBDE8C08F30BCFA
:10080000BDE8C04FFFF7DFBF2DE9FE4F81EA0304CB
:1008100004F0004421F0004100944FF0000B23F05D
:10082000004350EA01045ED052EA03045BD0C3F3F4
:100830000A54C1F30A552C44A4F2F3340194A0FBEA
:100840000254C1F3130141F48011C3F3130343F4C1
:10085000801301FB024400FB034E840A970A44EA1A
:10086000815447EA8357A4FB076802958D0A05FB6C
:1008700007854FEA932C04FB0C542705029D4FEA91
:10088000065847EA1637B5EB08056EEB070C870EDE
:10089000920E47EA811742EA8312A7FB0201B6EBE8
:1008A0000B0164EB00042B0D43EA0C335E1844EBA0
:1008B0001C50DA465146E7FB0201C5F313044FEA28
:1008C0000B3343EA14534FEA0432019C43EA060314
:1008D000A4F10C040294009CCDE900B400F03CFAB1
:1008E00003B000F003B800200146F9E730BCBDE8D2
:1008F000C08F2DE9F04D81EA030404F0004B21F094
:10090000004514464FF0000A23F0004150EA05026A
:1009100020D054EA01021DD0C5F30A570246C5F3A0
:100920001303C1F31300C1F30A5640F4801543F4D6
:100930008013A7EB0608101BD64608F2FD3873EBB0
:10094000050002D308F1010801E092185B41B8F1FB
:10095000000F03DA00200146BDE8F08D00204FF4BF
:100960008011064684460EE0171B73EB050705D37E
:10097000121B63EB050306434CEA010C49084FEADE
:10098000300092185B4150EA0107EDD152EA0300B2
:1009900012D082EA040083EA0501084305D0101B47
:1009A000AB4106D20122002306E000224FF00043B3
:1009B00002E06FF0010253101AEB06004CEB0851F5
:1009C00010EB0A0041EB0B01BDE8F04D00F0B5B9AA
:1009D0000EB5C10F80EAE0700844CA07002140F25A
:1009E00033438DE80E000A460B4600F0B5F903B01C
:1009F00000BD0EB540F2334102910021CDE9001156
:100A00000A460B4600F0A8F903B000BD20F00040F4
:100A1000C10DC0F3160040F400007F2901DA002068
:100A20007047962903DCC1F19601C840704796399A
:100A30008840704700F0004230F000400AD0C10DFD
:100A400001F56071C0F3160042EA0151C208400787
:100A50001143704700200146704701F0004330B455
:100A600021F0004150EA010206D00A0DA2F56072A1
:100A7000C1F31301002A02DC30BC00207047440F90
:100A800044EAC104C100E01830BC00EBC25000F0E1
:100A90001DB9202A04DB203A00FA02F10020704739
:100AA0009140C2F1200320FA03F3194390407047AC
:100AB000202A04DB203A21FA02F00021704721FAB3
:100AC00002F3D040C2F1200291400843194670471A
:100AD000202A06DBCB17203A41FA02F043EAE07302
:100AE00006E041FA02F3D040C2F1200291400843EF
:100AF0001946704710B50446F7F77EFB0068005DA5
:100B000000F0010010BD3A2800D2303820F0200259
:100B1000412A01D3A2F13700884201D34FF0FF30C0
:100B2000704700000268114413780160184670474E
:100B3000D1600449516104491162002111611146DB
:100B400000F09AB9250B0108F50A0108426842B184
:100B5000016811F8013B23B1521EC0E9001218468A
:100B600070470121C160881E704742685AB1C3684E
:100B7000016843B983688B4205D0491E521CC0E905
:100B80000012002070474FF0FF3070472DE9F05FF2
:100B900082460078002715468B460AF10104B946C3
:100BA000302801D09DB113E014F8010B01277828FB
:100BB00003D0582801D045B10AE00DB1102D07D15E
:100BC0000027102514F8010B02E0082500E00A2593
:100BD0000026B0460EE005FB080005FB06F10127E4
:100BE00001EB10461FFA80F8B6F5803F00D3B946F6
:100BF00014F8010B2946FFF786FF0028EBDABBF15A
:100C0000000F05D00FB1641E00E05446CBF8004041
:100C1000B9F1000F06D005F083FB02210160C81E68
:100C200000F003B848EA0640FAE730BCBDE8C09FD0
:100C30000FB4002300B589B00CA900910B996FF097
:100C40000042CB601E4B06931E4B07930423CDE955
:100C500001321D4A089202466B46002000F03AFB22
:100C600009B05DF814FB70B586B006464FF0FF3052
:100C70000091CDE90101002015460C460490324652
:100C8000694604A8FFF7D4FF02460498211825B14D
:100C900008B1084600E020462860049800280DD0DE
:100CA000002A02DD0098884208D0081B0094CDE994
:100CB00001043246694604A8FFF7BAFF06B070BDCA
:100CC0004D0B01086B0B0108F50A01080029A8BFAC
:100CD0007047401C490008BF20F00100704710B465
:100CE000B0FA80FC00FA0CF050EA010404BF10BC1A
:100CF000704749B1CCF1200421FA04F411FA0CF147
:100D000018BF012121430843A3EB0C01CB1D4FEA7F
:100D100000614FEA102042BF002010BC704700EB7A
:100D2000C35010440029A4BF10BC7047401C4900A8
:100D300008BF20F0010010BC704710B5141E73F1FD
:100D4000000408DA401C41F1000192185B411A438B
:100D500001D120F0010010BD2DE9F04D92469B46D7
:100D600011B1B1FA81F202E0B0FA80F2203290467D
:100D7000FFF78FFE04460F4640EA0A0041EA0B01E6
:100D800053465A46084313D0114653EA010019D07E
:100D9000C8F140025046FFF78BFE05460E4650460E
:100DA00059464246FFF775FE084305D0012004E08E
:100DB00020463946BDE8F08D0020054346EAE0763E
:100DC0002C4337430A986305E40AA0EB080000228D
:100DD000FD0A44EA47540A3002D500200146E9E7FB
:100DE000010510196941DDE9084500196941BDE8AF
:100DF000F04DA2E770B521F0004303430CD0C1F3DE
:100E00000A550024D5EB040564EB0403D617AD1A8C
:100E1000B34102DB0020014670BD201841EB0251B6
:100E200070BD000030B5041E71F1000404DB4FF00A
:100E30000044404264EB0101141E73F1000405DB21
:100E40001C464FF00043524263EB0403994208BF33
:100E5000904230BD064C074D06E0E06840F00103CB
:100E600094E8070098471034AC42F6D3F7F792F9AC
:100E70009CC30108BCC301082DE9F34F8BB04FF0B0
:100E8000000801F10C000C464FF0010B46460DF135
:100E9000080A01906269012101989047051E2DD032
:100EA000252D2CD0216A8847C0B1626901210198A3
:100EB0009047216A88470028F7D1411E626901984E
:100EC000904700E0761CA1690B988847216A884703
:100ED0000028F7D1E1690B988847DBE7A1690B98F7
:100EE00088470746A84201D1761CD3E7E1690B98F1
:100EF00088477F1C02D1B8F1000F6FD046E1002770
:100F000062693D463946019890472A2804D16269B2
:100F10000121019890470125DFF88492626901213F
:100F200001989047A0F130010A290AD24F45E5DC2B
:100F300007EB870100EB4107303FDFD445F0100598
:100F4000ECE7E90601D46FF000476C280AD04C2882
:100F500014D0682815D06A280DD074281CD07A289F
:100F60001AD01DE062690121019890476C2802D0D7
:100F700045F0040514E045F002050DE045F02005BC
:100F80000AE06269012101989047682802D045F083
:100F9000080505E045F40065626901210198904764
:100FA000C4E9015765283DD019DC58287AD00CDCFB
:100FB000452837D004DC252826D0412831D131E01E
:100FC00046282FD047282CD12CE05B2877D06128E9
:100FD00028D063287CD0642823D15AE0D0E06F2841
:100FE00048D008DC66281DD067281BD0692821D08E
:100FF0006E2816D127E0702845D0732868D0752850
:1010000047D078280DD14DE0A1690B988847054657
:1010100025283FF469AFE1690B9888476D1C3FF4C0
:101020006AAFB3E023466A466FF001000B9900F007
:1010300051F99EE045F040006060A80723464FF05C
:10104000000236D43EE0E8077FF447AF2068011D78
:1010500021600068290501D506701BE7290701D525
:10106000068017E7A90703D5F117C0E9006111E76A
:1010700006600FE745F040006060A80723464FF088
:10108000080216D41EE040F60E0125EA0100606059
:1010900016E045F040006060A80723464FF00A02C2
:1010A00007D40FE045F040006060A80708D523464C
:1010B00010226FF001000B99AFF3008059E007E0B8
:1010C000234610226FF001000B99FFF7D1F950E091
:1010D0004FF000094F464B46632802D05B2806D0EC
:1010E00040E0E80601D40120A06001273AE06269EF
:1010F0000121019890475E2805D14FF001096269EE
:10110000494601989047216939B900210A4653465A
:1011100043F82120491C0829FADBB0B3216969B9D9
:10112000C11700EBD16253110AEB830122F01F02B9
:10113000821A01200B68904003430B606269012111
:10114000019890475D28E8D1B9F1000F09D000203F
:10115000514651F82020D24341F82020401C082855
:10116000F7DB02AB224600976FF001000B99AFF35B
:10117000008000280CDA401C08D1BBF1000F05D01C
:101180004FF0FF300DB000F00DB8FFE74046F9E733
:10119000E90701D108F1010806444FF0000B79E698
:1011A000CCCCCC0C30BCBDE8C08F00002DE9FF4F8B
:1011B000087883B09946FF2805D0491C2D2804D013
:1011C0000024002008E000200BE00124F9E700EBF8
:1011D000800003EB4000491C0B78FF2BF7D104B1D2
:1011E000404200230293147819461D462D2C01D04D
:1011F0002B2C04D1521C2D2C13D000240294AA466F
:101200001478FF2C0FD00A25A3FB057801FB05817C
:101210004FF0000C03FB0C11521CE3194AEB0101C7
:10122000EEE70124EAE7814453EA010002D019F510
:10123000C87F06DA03980021C0E9001107B000F06A
:1012400065B90025AE4E2F46DFF8B882184600F08B
:10125000C9F9CDE90001B9F1000002DAC9F10004D1
:1012600000E004460023A74A1AEB030B42EB045AA2
:1012700012E0E00707D02A46334638464146FFF7DA
:10128000C3FA074688462A46334610461946FFF7F2
:10129000BBFA05460E466410002CEAD1DDE90001D8
:1012A000B9F1000F5A46534606DAFFF722FB3A46D9
:1012B0004346FFF71EFB05E0FFF7A6FA3A46434612
:1012C000FFF7A2FA029A0AB181F00041039AC2E93B
:1012D0000001B3E72DE9FF4F1F468DB0D7E9014666
:1012E0004FF0FF382E2045464FF000090B90B969AA
:1012F0006D1C0E988847396A824688470028F6D1C7
:10130000BAF1FF3F0AD024F4D064002E11DDBAF107
:101310002B0F08D0BAF12D0F0BD102E0404611B0CF
:101320008DE744F48064B9696D1C0E988847824645
:10133000761E6946600501D52D2000E02B208DF832
:10134000000001F1010B0DF1200809E0B9696D1CE5
:101350000E98884782460F9844F40074761E056004
:10136000002E02DDBAF1300FF0D00B998A453ED144
:1013700044F0800406E00F99681CA9F1010944F4C7
:1013800000740860B9696D1C761E0E988847824605
:101390003028F0D02BE00B998A4505D1200603D4E4
:1013A00044F08004761E18E0504606F077F908B342
:1013B0000DF11301761E44F400748B4508D2AAF196
:1013C00030000BF8010B200607D5A9F1010003E05E
:1013D000200602D409F101008146A00502D50F992B
:1013E000681C0860B9696D1C0E9888478246002EFB
:1013F000D1DC53E0002E51DDBAF1650F02D0BAF115
:10140000450F4BD1A00549D5B9696D1C24F4407432
:10141000761E0E9888478246002E0CDD2B2804D0BD
:10142000BAF12D0F07D144F48074B9696D1C0E9880
:1014300088478246761EE00501D52D2100E02B214C
:1014400008F8011BCDF82C8021E00DF12901761E52
:1014500044F4007488450CD2AAF1300010F0FF006B
:1014600088F8000002D10B99884509D908F10108D4
:1014700006E0E00501D5244801E042F20F70814604
:10148000B9696D1C0E98884782460F980560002E3A
:1014900004DD504606F002F90028D6D1F9690E980D
:1014A0008847FF208BF8000088F800000020069095
:1014B00007904B466A4608A906A8FFF777FEA005E5
:1014C00002D46FF001002AE714F0240F0AD0E007DD
:1014D00014D1DDE906123868031D3B600068C0E9DD
:1014E00000120BE0DDE90601FFF7B7FA0146E0075D
:1014F00004D13868021D3A600068016028460EE792
:10150000000014400000F03FF1D8FFFF30BCBDE800
:10151000C08F2DE9F04D00231A461B1A8A4103DBC8
:1015200000200146BDE8F08DC1F30A52C1F313015A
:1015300041F480154FF0000BD10702D100186D4126
:10154000521E0027044640F2FF11384601EB620AA2
:101550003E468046024600204FF48011FFF7A8FA6D
:10156000C2197141BB1846EB0100B4EB030C75EBDB
:10157000000C04D3E41A65EB000517460E46241947
:1015800008F101006D4180463428E3DDF91946EB8E
:101590000600091BA84103D24FF0FF32134601E0B9
:1015A000002213461BEB070046EB0A51BDE8F04D45
:1015B000FFF7C3BB30B5041E71F1000404DB4FF02C
:1015C0000044404264EB0101141E73F1000405DB8A
:1015D0001C464FF00043524263EB04038B4208BFAA
:1015E000824230BD0EB540F2334202920022CDE974
:1015F00000221346FFF7B0FB03B000BD70B58C1896
:1016000010F8015B15F0070301D110F8013B2A1116
:1016100006D110F8012B03E010F8016B01F8016B03
:101620005B1EF9D12B0705D40023521E0DD401F8FF
:10163000013BFAE710F8013BCB1A921C03E013F8C8
:10164000015B01F8015B521EF9D5A142D8D30020FD
:1016500070BD00002DE9F04104460E4600250068EB
:1016600003F00AFE0746206803F0FEFD074357D04B
:101670002068C168890111D5617E01290ED1217EC2
:1016800001290BD10126274902E08D4239D26D1C78
:101690000268D2435206F8D440210160224D022E46
:1016A0000FD0206803F0E8FD48B120688168C1F3DD
:1016B000400121B98168294041F010018160012E6B
:1016C0000DD0206803F0D0FD48B120688168C1F3D7
:1016D000400121B98168294041F020018160022E3A
:1016E00008D0032E04D0042501F06CFD064613E05B
:1016F0000C25F9E70825F7E701F064FD801B0528B4
:101700000AD9606D40F010006065A06D40F00100E6
:10171000A0650120BDE8F081206880682842EBD1F7
:101720000020F7E7000040A3C0FFFF7F10B5846AE8
:10173000616D11F0500F06D0616DC90625D52046A8
:1017400000F0B8FE10BD606D40F400706065206868
:101750000168090716D503F093FD78B12068C068C9
:10176000800400280ADB606D20F480706065606D85
:10177000C00403D4606D40F001006065204600F0B5
:10178000E0FD10BDC0688007EBE7E16C496BBDE888
:101790001040084710B5806A416D41F04001416535
:1017A000816D41F00401816500F084FE10BD10B52B
:1017B000806A00F0C7FD10BD70B5044600688168FE
:1017C000C1F3400503F054FD28B325BB20688168B0
:1017D00001F00D01012910D18168104A1140891CC6
:1017E000816021680320086001F0ECFC05460EE0F2
:1017F00001F0E8FC401B022809D9606D40F01000A0
:101800006065A06D40F00100A065012070BD2068FA
:101810008068C007ECD1002070BD0000C0FFFF7FD2
:1018200070B50446006803F023FD48BB206881685A
:10183000144A114215D18168D6433140491C816058
:1018400001F0C0FC054616E003F012FD20B9206847
:1018500081683140491C816001F0B4FC401B0228C2
:1018600009D9606D40F010006065A06D40F0010086
:10187000A065012070BD20680168C943C907E3D194
:10188000002070BD3F0000802DE9F0472C4800F09B
:101890005BFD2B482B49002501604FF40031C0E966
:1018A000011501210822C560C0E9041205764176C0
:1018B0000322C26180F82050C0E90915C56280F892
:1018C00030100903416380F8385000F0F5FD1E48E0
:1018D0001B4C062190F8008064341C4807227F23AB
:1018E0004FF0040C656184E80F10194E0C27144862
:1018F0004FF01209B8F1010F214616D000F02CFB71
:1019000021460F48C4E9006700F026FB1148C4E9EE
:1019100000090B490A48643100F01EFBBDE8F0479E
:1019200003220D49064800F02BBF00F015FB0449C7
:1019300003486431C4E9006700F00EFB0748E6E79E
:10194000A80A002000000450870100204000201950
:101950000008302E001060324800002000002143B3
:101960002DE9F0411C49022008702C211B48FEF78C
:101970004AFD1A4C7820042120701020A080E180BC
:10198000082222720127678140F2DC52A2814FF6C1
:101990007063E38122615242626106F008FE104EDC
:1019A00084F828000025022006F0A8F805F07EFE45
:1019B000A070800605D4B6F84C00401CA6F84C0078
:1019C00003E06D1CEDB20A2DEDD336F84E0F401C2E
:1019D00030806770BDE8F08186010020F40B0020A4
:1019E000EE0800200020704700207047002070475C
:1019F00000207047FEE7000010B54FF47A7006F043
:101A0000B3FD06490220887108F042F908F02AF96E
:101A100008F0FFF8BDE8104008F00FB98001002081
:101A20002DE9F05F0024DFF8E8A03A4D3A4FA346D5
:101A30004FF00409AAF1500801261AF804100129F0
:101A400014D159460AF804B0B4B1012C38D0022C94
:101A500046D0032C4ED008EB8400304990ED000AAC
:101A6000BCEEC00A10EE100A21F81400641CE4B2A7
:101A70000B2CE2D300F062B8294AD8F8000090425B
:101A800001D1E97119E02749884201D1EE7114E0D2
:101A90002549884201D102200BE02449884201D126
:101AA000032006E02249884205D02249884202D11B
:101AB0000520E87101E085F8079005F0C5FE0DE00E
:101AC0001348503890ED010AB5EEC00AF1EE10FA55
:101AD000CCD1BCEEC00A10EE100A28733E70C5E7E8
:101AE0000B48503890ED020A1348BCEEC00A80ED56
:101AF000010A08E00648503890ED030ABCEEC00A1F
:101B000010EE100AA8713E7005F062FEAEE700000C
:101B100038870020AC05002068010020EE08002076
:101B20000000164600009646000016470000614778
:101B30000000E147000096478002002030BCBDE86D
:101B4000C09F00EBC000052190FBF1F000F5A070F4
:101B500000B270470D4910B50B480860084600F008
:101B6000F6FE0A4800211430002241600221816003
:101B70000146143800F05EFE04491022BDE8104012
:101B80001431024800F056BE00740040240B0020BF
:101B90000E4810B5C06C00F0CDFF0F4A0C490D4C3B
:101BA00010780B8824F81030C8344B8824F8103093
:101BB00004F1C803898823F81010401CC0B21070CB
:101BC000642801D30020107010BD0000A80A002076
:101BD00048000020E20D0020EC01002030B590F814
:101BE000444004F01C050124AC40056C6C600468A2
:101BF00063608368102B036803D099600068C2603B
:101C000030BD9A600068C16030BD7047044805A1CE
:101C10000968016072210171052004F041BB0000D8
:101C2000C20700206572726F72000000124A107FB6
:101C30001249012801D003280BD10B6843F400633B
:101C40000B600B6823F400630B600B6843F40073B4
:101C50000B60022801D003280BD1086840F48050A3
:101C60000860086820F480500860086840F48060CC
:101C70000860002010777047FC010020002002401F
:101C8000C107054803D0416941F004014161416940
:101C900041F48031416170470020024008494A699F
:101CA000C0B222F47E7242EAC0004861486940F046
:101CB00002004861486940F4803048617047000084
:101CC00000200240054910B54C6944F001044C6104
:101CD0000260BFF36F8F436010BD00000020024020
:101CE000094B10B55C69402244F480245C61EFF339
:101CF000108372B610C910C0521E12F0FF02F9D143
:101D000083F3108810BD00000020024070B5044627
:101D100001F058FA0646174D08E0601C06D001F0A5
:101D200051FA801BA04201D3032070BD2869C00373
:101D3000F3D4296910480140A86900F00040084325
:101D400011D00E494A6802434A60810F04D0A96944
:101D500000F040421143A961810002D020F04040D0
:101D60002861012070BD2869C00701D001202861C9
:101D7000002070BD00200240FAC30200FC010020D8
:101D80000D4910B509684FF48023CC432204120C8E
:101D900009D00A04920902F10062824205D9A0F139
:101DA0000060C00A10BD1A46F5E72204120C01D0EB
:101DB00009048B09C01AF2E7E075FF1F004870475D
:101DC0003000002018B90B2901D2012070470020F3
:101DD000704700009FED010A7047000000000000FE
:101DE000014840887047000080020020004870478A
:101DF000900200200548407A602803D05A2803D07A
:101E000003A0704704A0704704A07047AC050020F1
:101E10006E756C6C00000000414653005452414EF8
:101E2000445543455200000078BB0B2A64D2344924
:101E30003448F2EE040A5BD2DFE802F00625282ED1
:101E40003040424446495400C97951B101290AD071
:101E500002290AD003290AD0042910D0052910D05C
:101E600008E0294904E0294902E0294900E029491C
:101E7000C0F81E10D0F81E0000EE100A7047264968
:101E8000F6E72649F4E7097B2FE035E0244991ED98
:101E9000010AB8EE400A22E0897926E0CA7B21498E
:101EA00091ED000ADAB1B3EE021A20EE010A80EEDB
:101EB000201A9FED1D0A31EE000A10E01B4904E0D4
:101EC0001B4902E01B4900E01B490968D0E71B4998
:101ED000098800EE101AB8EE401A81EE200A10EEC2
:101EE000101AC5E71649B1F80C1100EE101AD0E728
:101EF000144931F81210F8E7B7EE000A70470000F5
:101F0000AC050020C0860020000016460000964662
:101F100000001647000061470000E14700009647B7
:101F200080020020A801002000000042A40100203F
:101F3000B4010020AC010020B00100208E0100207F
:101F400052090020EE080020704700000148807907
:101F500070470000AC0500202DE9F84F002704462B
:101F6000009790F85000DFF8A8930D46B846012876
:101F700010D0012684F85060206803F07DF958B134
:101F8000606D40F020006065012784F8508038467D
:101F900000F0D4B90220FBE768680C23052812D8AA
:101FA000022807D0032807D0042807D0052807D027
:101FB000062007E06B6006E0122003E0182001E035
:101FC0004FF480706860D5E90021206803EA91131E
:101FD0001844036B01F01F014FF01F0C0CFA01FCB9
:101FE000C2F3846223EA0C038A401343036320682C
:101FF00003F042F98246206803F036F95AEA0001FC
:102000001DD1AA682968206803F042F920686A692E
:10201000C168C1F3C10149008A40296904290FD070
:1020200000EB81002B68016EDFF8E8C203F0F84393
:1020300001EA0C011343194341F00041016672E0CB
:10204000002103F00BF9400320684FF0000171D02C
:1020500003F004F990FAA0F0B0FA80F12868420386
:102060006DD090FAA0F0B0FA80F0814204D1002245
:102070001146206803F01BF90121206803F0EEF8F7
:10208000400320684FF001015CD003F0E7F890FABC
:10209000A0F0B0FA80F12868420358D090FAA0F07E
:1020A000B0FA80F0814204D100220121206803F0BF
:1020B000FEF80221206803F0D1F8400320684FF0B9
:1020C000020147D003F0CAF890FAA0F0B0FA80F10C
:1020D0002868420343D090FAA0F0B0FA80F0814221
:1020E00004D100220221206803F0E1F803212068D6
:1020F00003F0B4F8400320684FF0030132D003F03E
:10210000ADF890FAA0F0B0FA80F1286842032ED022
:1021100090FAA0F0B0FA80F0814204D100220321AD
:10212000206803F0C4F8206803F0A2F810B3AAE016
:1021300000E004E003F092F8C0F384618EE7C0F39E
:10214000846092E703F08AF8C0F38461A3E7C0F3E8
:102150008460A7E703F082F8C0F38461B8E7C0F3B6
:102160008460BCE703F07AF8C0F38461CDE7C0F384
:102170008460D1E721682A7B286851F8B03FC0F31A
:10218000120C23EA0C0302F0180C634A22FA0CF238
:10219000024013430B60E968494574D12868410344
:1021A0001AD090FAA0F1B1FA81F1491C01F01F0197
:1021B00009294FEA403130D8002910D090FAA0F117
:1021C000B1FA81F101F1010101F01F0106FA01F6F6
:1021D00008D1C0F3846109E0C0F38461E5E7C0F38E
:1021E0008461EFE790FAA0F1B1FA81F101F1010108
:1021F00001F01F0146EA816102D1C0F3846003E06F
:1022000090FAA0F0B0FA80F000F1010000F01F0099
:1022100000EB400041EA005131E000290DD090FA76
:10222000A0F1B1FA81F101F1010101F01F0106FAFB
:1022300001F605D1C0F3846106E0C0F38461F2E7E2
:1022400090FAA0F1B1FA81F101F1010101F01F0151
:1022500046EA816102D1C0F3846003E090FAA0F005
:10226000B0FA80F000F1010000F01F002B4A00EBF3
:10227000400002EB005041EA000141F00071AA6801
:10228000206803F005F82648296801423FF47DAE36
:10229000244A9068244D254B00F0E070A9421AD1E1
:1022A000050218D4216899427FF46FAE916840F41A
:1022B000000021F0E071014391601D481D49006854
:1022C000B0FBF1F000EB4000800000E0401E009009
:1022D0000028FBD159E6184DA94207D1C50105D404
:1022E00021689942F6D140F080700AE06FF0004515
:1022F000E942EFD14102EDD421689942EAD140F49C
:102300008000916821F0E071014391603DE600009A
:1023100000007F4000F0FF03FFFF0700000020FEE9
:102320000000088000030450000052C70000045061
:102330001C020020400D0300000084CB18BCBDE847
:10234000E08F70477047000070B504000FD0606DDB
:1023500040F00200606503212046FFF77BF905008D
:102360002068C16841F40011C16002D008E001207A
:1023700070BD2046FFF720FA050001D101206065FD
:10238000206841686FF30A014160216840F2FF70E4
:1023900008602068816821F0A04181602068816820
:1023A00041F0005181602068C1683D4A1140C16020
:1023B0002068C16841F00041C160206801696FF385
:1023C0000A0101612068416901F0404141612068D2
:1023D000816901F0784181612068016A01F0F02192
:1023E00001622068416A01F0FF2141622068816A30
:1023F00001F0FF2181622068016B2A4A11400163CC
:102400002068416B274A103A114041632068816B74
:10241000114081632068C16B40F2DF729143C16358
:102420002068026E20490A4002662068426E0A4017
:1024300042662068826E0A4082662068C26E0A4048
:10244000C266206850F8A01F6FF312010160206877
:1024500050F8A41F6FF312010160206850F8B01FFC
:102460006FF312010160206850F8B41F21F07F1152
:1024700001600E488168C1F3000129B9D0F8081342
:102480000B4A1140C0F80813204600F0E9F800207C
:10249000A065E0652066606584F85000284670BD40
:1024A00004800080300882E000F0FF030000045048
:1024B000FFFF00FE70470000F8B54FF00005040074
:1024C0002E46009502D0606D10B107E00120F8BDE6
:1024D000204600F0E5F8A66584F850602068816821
:1024E000C1F3407119B18168554A1140816020687B
:1024F0008168C1F3007179B98168524A114041F095
:1025000080518160504851490068B0FBF1F000E013
:10251000401E00900028FBD120688168C1F3007143
:1025200041B9616D41F010016165A16D41F001019A
:10253000A165012502F0A0FE616DC90600D430B18D
:10254000606D40F01000606501252846F8BD606DA3
:1025500020F4807040F002006065206802F088FE80
:1025600058B93B488068C0F3000030B93949606809
:102570008A6822F47C1202438A60E168606B627EA2
:102580000843A16841EA4231084394F8201040EA28
:102590000140012904D1A18C2F4A02EB414108439B
:1025A000A16A29B101F47071E26A014342EA0100B3
:1025B0002168CA68294B1A400243CA60206802F0A9
:1025C0005BFE0646206802F04FFE064315D1207ED2
:1025D00094F83010800340EA41012068C26844F258
:1025E00002039A430A43C26094F8380001280CD0D1
:1025F0002068016921F0010101612069012820683A
:10260000016B21F00F0110D012E0D4E90F1001434B
:10261000D4E91102104301432068026940F2FC73BF
:102620009A43114341F00101E6E7E269521E11436A
:102630000163606D20F0020040F00100606584E7F6
:10264000C0FFFF5FC0FFFF7F1C020020400D0300A2
:1026500000000450000304500000FEFF07C0F0FF1C
:1026600010B5044600680B49884212D10A48C16C73
:1026700021F40051C164C3214FF0904000F05AFC96
:102680000321064800F056FCE06CBDE8104000F065
:1026900003BA10BD000004500010024000040048BE
:1026A00070B53249064686B051F84C0F40F0010033
:1026B00041F80409486800F001000590486840F0BE
:1026C00002004860486800F002000590486840F445
:1026D00000504860486800F400500590086C40F0D5
:1026E00040500864086840F00100086008680B2446
:1026F00000F0010005901E48002501784FF0904041
:10270000012927D0C2218DE83200694600F08CFCF7
:10271000194C1848C4E900058020A560C4E903509D
:10272000400060618000A0612020E061C001206263
:10273000204600F0B1F9204600F05AFAF464002275
:1027400001210B20A66201F0C3F80B2001F0B2F8C2
:1027500006B070BD42218DE83200694600F064FC8D
:1027600002208DE8310069460448CFE7001002409E
:102770008701002008000240600A00200004004891
:1027800070B5044615460E46006802F075FDE0BBC4
:1027900094F85000012842D0012084F850002046CF
:1027A000FFF73EF8002110B184F8501070BD606D45
:1027B00040F60162904340F480706065606DC00433
:1027C00004D5A06D20F00600A06500E0A165E26CD4
:1027D0001448D062E26C14481063E26C13485063F2
:1027E00022681C20106084F850102068416841F075
:1027F000100141602068C16841F00101C160216899
:102800002B4632464031E06C00E008E000F060FA10
:1028100021688A68064B1A40121D8A6070BD02202A
:1028200070BD00002D170108AF17010895170108AA
:10283000C0FFFF7F2DE9F0470446407900270E4690
:1028400001280BD04FF0010984F805900220207177
:10285000306802F01005042803D043E00220BDE8F0
:10286000F0874FF0030802BB00F0ACFC074604E021
:1028700000F0A8FCC01B01280FD82068406B0004A2
:10288000F6D4012000F05CFA2168B069086416E013
:1028900000F098FCC01B012807D9206940F008000F
:1028A000206184F804800320D9E72068406B002869
:1028B000EEDB012000F044FA2168B069486420682A
:1028C000816C40F2FF32AA409143F269AA40114361
:1028D00081642068C16CFF22AA409143326AAA40F9
:1028E0001143C1643069012808D12068826B1F211F
:1028F000A9408A437169A940114381632068C26B72
:102900000721A9408A43B36831681943F368194322
:10291000A9401143C163206801684FF48042AA4076
:10292000914301602068026840F6FC71A9408A4327
:102930007168A9401143016020680168C022AA4063
:102940009143016084F804900020607187E770B5BE
:10295000040003D02079002510B105E0012070BDEE
:102960006571204600F008F80220207125610120E1
:102970002071002070BD000010B50068144986B0B9
:10298000884222D11348816D41F000518165816DEB
:1029900001F000510591C16C41F00101C164C06CAE
:1029A0004FF0904400F001000590102000900320AB
:1029B0000190002002906946204600F035FB20215E
:1029C00000916946204600F02FFB06B010BD0000C4
:1029D000007400400010024018B5046800940068BC
:1029E000104421B1143000900360002018BD08305D
:1029F000F9E730B54279012A14D00123437102224C
:102A000002710268146801F0100503FA05F52C4301
:102A10001460002901680A6806D0C2F38342012AC3
:102A20000AD00DE0022030BDC2F38302012A07D193
:102A30004A6842F0010202E04A6842F002024A603B
:102A4000037100214171084630BD10B590F8251082
:102A50000024022903D00421C16301241AE0016883
:102A60000A6822F00E020A6001680A6822F0010278
:102A70000A6090F84410012301F01C0203FA02F1ED
:102A8000026C516080F82530002180F82410816BA1
:102A900001B18847204610BD30B590B101680A6881
:102AA00022F001020A60204C026814211F4BA2424E
:102AB00009D21F4C1444B4FBF1F18900C0E9103174
:102AC0000BE0012030BD184C64421444B4FBF1F11A
:102AD000890041641449083901640021116090F8AB
:102AE000442002F01C040122A240046C6260046CC9
:102AF0000F229C4202D153F8A84F02E00A4BA033A8
:102B00001C6890F8445005F01C05AA4094431C60D2
:102B1000C162016341638163C16380F8251080F85D
:102B20002410002030BD00000804024000000240D4
:102B3000F8FFFDBFF0B4016C0B6801680A6890F8FB
:102B40004440042504F01C0405FA04F61E4211D08A
:102B500056070FD50A68920603D40A6822F00402C9
:102B60000A6090F8441001F01C018D40016C4D602A
:102B7000016B1DE0022606FA04F71F424FF0000C1D
:102B80004FF0010518D0970716D50A68920605D4AC
:102B90000A6822F00A020A6080F8255090F8441072
:102BA00001F01C018E40016C4E6080F824C0C16AA7
:102BB00000291AD0F0BC08470826A6401E4214D0AF
:102BC000120712D50A6822F00E020A6090F844102B
:102BD000026C01F01C0105FA01F15160C56380F837
:102BE000255080F824C0416BE2E7F0BC704700003C
:102BF00070B568B1334C01681423334AA14209D23D
:102C0000324C0C44B4FBF3F39B00C0E910230BE0FF
:102C1000012070BD2B4C64420C44B4FBF3F39B00C9
:102C20004364284B083B0364022380F825300C687A
:102C300047F6F0739C43D0E902352B43D0E90456A4
:102C400035432B4385692B43C5692B43056A2B43C9
:102C500023430B608168B1F5804F29D0016C0F23AD
:102C6000914212D152F8A81F90F8444004F01C047D
:102C7000A3409943116090F84430416803F01C036D
:102C8000994013681943116012E00E49A0310A6897
:102C900090F8444004F01C04A3409A430A6090F862
:102CA0004430426803F01C039A400B681A430A60E0
:102CB0000021C163012280F8252080F824100846F5
:102CC00070BD00000804024000000240F8FFFDBF94
:102CD00070B5044690F82400002501280CD001208E
:102CE00084F8240094F825600020012E06D084F892
:102CF00024000225284670BD022070BD022684F8FB
:102D00002560E0632068066826F00106066020461C
:102D1000FEF764FF206B00282068016802D041F0B4
:102D20000E0106E021F0040101602068016841F015
:102D30000A0101602068016841F001010160D9E7E2
:102D400070B5044600F03EFA0546601C02D0044807
:102D50004068044400F036FA401BA042FAD370BD2C
:102D6000F00100202DE9F05F0446344889460178DF
:102D700001290CD00125804605704CF2503B584685
:102D8000FEF7C4FF06004FF0000A03D052E0022015
:102D900000F058B851464046C8F804A0284F3A6899
:102DA00092050ED5396821F40071396039684905FA
:102DB00005D5396821F480613960032109E0057780
:102DC00008E03A68520504D5396821F48061396019
:102DD000022101772068012807D04FF0FF31C9F8A0
:102DE000001040F2FA3BA5681DE06068FEF748FF5E
:102DF0005846FEF78BFF0646786920F0040078619C
:102E000016E028466168FEF749FF4CF25030FEF7A5
:102E10007DFF0600786920EA0B00786102D0C9F8CE
:102E2000005005E06D1CD4E902010844A842E8D82E
:102E3000FEF7FCFE88F800A03046A9E7FC01002060
:102E40000020024030BCBDE8C09F0000034841693B
:102E500041F0004141610020704700000020024025
:102E60002DE9FF5F254F05460024387891469B46A3
:102E7000012809D0012038704CF25030FEF746FF8F
:102E80000600A24604D035E0022004B000F03AB8B3
:102E90005046C7F804A0DFF86880D8F8001049054C
:102EA00006D5D8F8001021F48061C8F8001002207F
:102EB000387725B1012D09D0022D07D00DE04A4603
:102EC0005B460198FEF7FEFE012406E049460198A4
:102ED000FEF706FF022D00D16C044CF25030FEF7D5
:102EE00015FF064624B1D8F81410A143C8F81410F1
:102EF000FEF79CFE87F800A03046C6E7FC010020E4
:102F00000020024030BCBDE8C09F00000649002000
:102F10004A69002A07DA054A8A60054A8A604969CF
:102F2000002900DA01207047002002402301674594
:102F3000AB89EFCD2DE9F04F0022DFF8D4A04FF0A0
:102F4000010B4FF00F095DE00BFA02F717EA0103DE
:102F500057D022F003055544AC6896074FEA167C1B
:102F600009FA0CF606EA0408B0F1904F04D0294C97
:102F7000A04203D1012407E0002405E0264CA04232
:102F800001D1022400E0072404FA0CF444451ED1C8
:102F9000DFF888C0DCF800409C43CCF800400CF11E
:102FA000040CDCF800409C43CCF800400CF1040C0D
:102FB000DCF800409C43CCF800400CF1040CDCF839
:102FC00000409C43CCF80040AB68B343AB6004685E
:102FD00055000323AB401C430460D40800EB840479
:102FE000266A55074FEAD56C09FA0CF5AE432662FE
:102FF00084689C4384604468BC434460C4689C43C8
:10300000C460521C31FA02F39ED100F009B80000EE
:10301000000001400004004800080048000401408E
:1030200030BCBDE8C08F00002DE9F84FDFF85891A3
:10303000002209F1040A0AF1040B4FF00F080BF10A
:10304000040E9AE00126964033407DD04C68022C55
:1030500001D0122C11D1D40800EB84073D6A54072B
:10306000E40E08FA04FC25EA0C05D1F810C00CFAAD
:1030700004FC4CEA050CC7F820C00768540003257F
:1030800091F804C0A5400CF0030CAF430CFA04FC0B
:103090004CEA070CC0F800C04F68012F05D0022F82
:1030A00003D0112F01D0122F11D18768D1F80CC095
:1030B000AF430CFA04FC4CEA070CC0F808C04768A0
:1030C000B7430E79C6F3001696403E434660C66885
:1030D000AE438D68A5403543C5604C68E4004BD5D0
:1030E0002A4C256E45F001052566246E22F0030565
:1030F00004F001040094264C2E19B7689407250F9C
:1031000008FA05F4A743B0F1904F04D0214CA04237
:1031100003D1012407E0002405E01F4CA04201D1A7
:10312000022400E00724AC403C43B460D9F80040DE
:103130004D464E689C43F60300D51C432C60DAF8DC
:10314000004055469C4300E016E04E68B60300D5AB
:103150001C432C60DBF800405D464E689C43F60241
:1031600000D51C432C60DEF8004075464E689C4339
:10317000B60200D51C432C60521C0B6833FA02F4D3
:103180007FF460AF00F00AB8000401400010024074
:1031900000000140000400480008004818BCBDE8D9
:1031A000E08F0069084000D00120704742690A4260
:1031B00001D081627047816170470AB181617047B7
:1031C000816270470148806870470000F00100206C
:1031D00010B5040013D0242084F841002068016851
:1031E00021F001010160204600F07EFA00206064B9
:1031F00084F8410044F8300FA074207410BD012001
:1032000010BD90F84100704770B5040004D094F8E8
:103210004100002510B106E0012070BD84F8405047
:10322000204600F075FA242084F8410020680168E7
:1032300021F0010101606068216820F07060086180
:103240002068816821F400418160E0680128A0685D
:1032500007D040F4044021688860E068022803D069
:1032600006E040F40040F6E721684FF40060486053
:1032700020684168114A114341602068C16821F407
:103280000041C160D4E904010843A16940EA01207A
:103290002168C860D4E907010843216808602068F4
:1032A000016841F0010101606564202084F841005B
:1032B000256384F84250002070BD000000800002A9
:1032C0002DE9FF4F83B00446DDE9108790F84100F7
:1032D000DDF848909A469346202876D15FEA0800A8
:1032E00014D09FB194F8400001286ED0012084F8DA
:1032F0004000FFF767FF0546012200901923D10324
:10330000204601F0C9FD002873D103E04FF400709E
:1033100060646EE0222084F84100402084F842007E
:1033200000266664C4F8248067856663CDE900954D
:1033300053465A462046049901F034FD10B184F8F2
:10334000406056E0618D3648FF274FF080784FF09F
:10335000007AFF2904D927853A464346009005E0C4
:10336000618D2185009094F82820534620460499C9
:1033700001F07CFD4B46002204212046009501F01F
:103380008BFDB0BB2068406A616A0870208D0128FF
:1033900002D9616A491C6162401E80B22085618D3C
:1033A000491E6185618DD9B1D0B94B46002280217B
:1033B0002046009501F070FDD8B9608DFF2805D931
:1033C00027853A464346009606E026E0608D208534
:1033D000009694F8282053462046049901F046FDB3
:1033E000608D0028C6D12A464946204601F080FD5E
:1033F00018B1012007B000F017B820682021C16182
:1034000020684268074B1A40426084F8411084F8F3
:10341000426084F840600020ECE70220EAE7000008
:103420000024008000E800FE30BCBDE8C08F000032
:103430002DE9F84F0446DDE90A8790F84100DDF8F0
:1034400030A08B46202804D04A498889401C8881B6
:103450001BE05FEA080014D09FB194F840000128F7
:1034600013D0012084F84000FFF7ACFE054601228E
:1034700000901923D103204601F00EFD002867D1EA
:1034800006E04FF40070606462E0022000F078B85B
:10349000222084F84100402084F84200002666641F
:1034A000C4F8248067856663618D3348FF274FF039
:1034B00080784FF00079FF2904D927853A464346A2
:1034C000009005E0618D2185009094F828204B46FE
:1034D0005946204601F0CAFC5346002204212046EA
:1034E000009501F0D9FC98BB2068406A616A0870B9
:1034F000606A401C6062208D401E80B22085618D14
:10350000491E6185618DD1B1C8B953460022802121
:103510002046009501F0C0FCD0B9608DFF2804D989
:1035200027853A464346009605E0608D2085009643
:1035300094F828204B465946204601F097FC608DB0
:103540000028C9D12A465146204601F0D1FC08B1D5
:1035500001209BE720682022C26120684168074B58
:103560001940416084F8412084F8426084F840604A
:1035700000208BE7EE0800200024008000E800FE19
:1035800018BCBDE8E08F00002DE9FF4F83B0044672
:10359000DDE9108790F84100DDF848909A4693469F
:1035A000202871D15FEA080014D09FB194F8400040
:1035B000012869D0012084F84000FFF703FE064689
:1035C000012200901923D103204601F065FC002858
:1035D0006ED103E04FF40070606469E0212084F84C
:1035E0004100402084F8420000256564C4F824802E
:1035F00067856563CDE9009653465A46204604998F
:1036000001F002FC10B184F8405051E0608DFF27BA
:103610004FF080784FF0007AFF2804D927853A468A
:103620004346009505E0608D2085009594F828209C
:1036300053462046049901F019FC3246494620467B
:1036400001F07CFCA0BB606A216800788862606A37
:10365000401C6062608D401E6085208D401E80B2DF
:103660002085618DD9B1D0B94B46002280212046FA
:10367000009601F011FCD8B9608DFF2805D9278587
:103680003A464346009506E026E0608D2085009589
:1036900094F8282053462046049901F0E7FB608DFA
:1036A0000028CAD132464946204601F021FC18B113
:1036B000012007B000F014B820682021C161206803
:1036C0004268064B1A40426084F8411084F8425028
:1036D00084F840500020ECE70220EAE700E800FE12
:1036E00030BCBDE8C08F00000068074988420AD19D
:1036F0000648816D21F4001181654FF4C0614FF0DF
:103700009040FFF717BC7047005400400010024083
:1037100010B586B0044614216846FCF774FE1349C0
:103720002068884220D1124CE06C40F00100E06437
:10373000E06C694600F0010005904FF4C060009015
:103740001220019001200290002003900420049098
:103750004FF09040FFF768FCA06D40F40010A065AA
:10376000A06D00F40010059006B010BD005400409C
:103770000010024070B5040011D021684CF6CC4016
:103780000860216845F255500860D4E900014160A5
:103790002168A0688860FFF715FD054608E0012054
:1037A00070BDFFF70FFD401B302801D9032070BD0D
:1037B0002068C0680028F4D120680269E1688A4264
:1037C00001D0016102E04AF6AA210160002070BD2B
:1037D00000684AF6AA21016000207047024881680B
:1037E0004268114481607047F001002010B5002448
:1037F000032000F08DF8002000F008F808B1012443
:1038000001E000F03DF8204610BD000000B5014683
:1038100087B00022192000F05BF8192000F04AF868
:103820001348016E41F400610166006E05A900F4C1
:1038300000600690684600F0A7FA00F0D7FA0D493C
:103840000D4AB0FBF1F10D48491E0260416040F2A3
:10385000E7320021C0E90321816000F0BAFD10B118
:10386000012007B000BD054800F0F4FDF9E70000B5
:103870000010024040420F00002C01403C1000208C
:103880000B4882B0016E41F001010166016E01F04A
:1038900001010091816D41F080518165806D0022B0
:1038A00000F0805000900F21901E02B000F010B880
:1038B00000100240002809DB00F01F0201219140A6
:1038C0004009800000F1E020C0F8001170470000BE
:1038D000F0B40E4B1B68C3F30223C3F10704042C9E
:1038E00000D904241D1D072D01D2002300E0DB1E9A
:1038F000012606FA04F56D1E0D409D409E40761E81
:10390000164045EA0601F0BC02F0F9BC0CED00E0FF
:10391000064A00F0070110684FF6FF03184040EA1E
:103920000120034908431060704700000CED00E0DF
:103930000000FA05012080F31388BFF34F8F05487C
:103940000168054A01F4E06111430160BFF34F8F44
:1039500000BFFDE70CED00E00400FA051649B0F5E4
:10396000007F0868C0F3412009D0022805D008680C
:1039700020F4C06040F48060086000207047012897
:10398000FBD0086820F4C06040F4007008600B4869
:103990003222006850430A4AB0FBF2F0401C00E0BB
:1039A000401E4A69520501D50028F9D148694005F1
:1039B000E3D5032070470000007000401C02002087
:1039C00040420F000248006800F4C06070470000E9
:1039D000007000402DE9F84F0446002500889B4EFA
:1039E0002F46000515D5E06B60B1B0F5000F04D08F
:1039F000B0F5400F2BD001250AE0F06840F480308C
:103A0000F06024E00021201D01F05CFC05001ED0C8
:103A10002F462068800365D5B06D4FF00009C000C7
:103A200009D4B06D40F08050B065B06D4FF0010921
:103A300000F080500090DFF818A2DAF8001041F48E
:103A40008071CAF80010FFF7BDFB804610E0D6F881
:103A50008800E16B20F440000843C6F88800D8E7EE
:103A6000FFF7B0FBA0EB0800022801D9032531E0E5
:103A7000DAF80000C005F3D565BBD6F8900010F465
:103A8000407014D0216D814211D0D6F89000D6F844
:103A9000901020F4407041F48031C6F89010D6F8B0
:103AA000901021F48031C6F89010C6F89000C0073D
:103AB0007ED0FFF787FB804641F2883A05E0FFF7AA
:103AC00081FBA0EB08015145D0D8D6F890008007C3
:103AD000F5D5EDB32F46B9F1000F03D0B06D20F04E
:103AE0008050B0652078C00707D0D6F88800216ADA
:103AF00020F003000843C6F888002078800707D527
:103B0000D6F88800616A20F00C000843C6F88800E7
:103B10002078800607D5D6F88800A16A20F4406096
:103B20000843C6F888002088800507D5D6F88800A5
:103B3000616B20F440200843C6F8880020884005C7
:103B400009D5D6F88800A16B20F44010084300E0A6
:103B50002EE0C6F888002078400607D5D6F8880001
:103B6000E16A20F440500843C6F888002088C00568
:103B700007D5D6F88800216B20F440300843C6F8FA
:103B8000880020884FF0006580044FF0806820D5C1
:103B9000D6F88800216C20F040600843C6F8880001
:103BA000206CA8420DD1F06840F48010F06010E065
:103BB000D6F89000216D20F440700843C6F89000BC
:103BC00089E7404505D10121201D01F07BFB00B1B3
:103BD00007462068400317D5D6F88800616C20F0AE
:103BE00040600843C6F88800606CA84204D1F068C1
:103BF00040F48010F06007E0404505D10121201D10
:103C000001F060FB00B107462088400411D5D6F8CA
:103C10008800A16C20F040500843C6F88800A06CD2
:103C2000B0F1805F05D10221201D01F04BFB00B1F6
:103C300007462088000406D556F8880FE16C20F06E
:103C4000804008433060384600F004B8001002405D
:103C50000070004018BCBDE8E08F00002DE9F0477F
:103C60000D4604005ED0DFF80C81D8F8000000F0AB
:103C70000700A8420CD2D8F8001021F00701294310
:103C8000C8F80010D8F8000000F00700A84249D199
:103C90002078394EC0072BD06068032811D0022845
:103CA00012D0316898B1490500293BDAB16821F09A
:103CB00003010143B160FFF785FA074641F28839F5
:103CC0000FE031688901EFE731688903ECE7890784
:103CD000EAE7FFF777FAC11B494502D90320BDE89F
:103CE000F087B068616800F00C00B0EB810FF0D194
:103CF0002078800705D5B068A16820F0F00008435F
:103D0000B060D8F80010404601F00701A9420BD975
:103D1000016821F0070129430160006800F00700F5
:103D2000A84201D00120DAE72078400705D5B06825
:103D3000E16820F4E0600843B0602078000706D511
:103D4000B068216920F4605040EAC100B06000F022
:103D50005FF8B168094AC1F30311515C01F01F011A
:103D6000C8400749086007480068BDE8F047FFF70A
:103D70004DBD0000002002400010024080BE01083E
:103D80001C020020F00100200F2202600C4A936800
:103D900003F003034360936803F0F00383609368C8
:103DA00003F4E063C36092684FF4E06303EAD20275
:103DB00002610448006800F00700086070470000D6
:103DC000001002400020024005480649006889684A
:103DD000054AC1F30221515C01F01F01C840704740
:103DE0001C02002000100240C0BE01080548064920
:103DF00000688968054AC1F3C221515C01F01F01C6
:103E0000C84070471C02002000100240C0BE0108DC
:103E100070B5254B002210469968DC6811F00C0142
:103E200004F00306214C4FEA640508D00C2904D0A5
:103E3000042931D0082931D010E0012E10D11A68A0
:103E4000120704D4D3F89420C2F3032202E01A68C4
:103E5000C2F30312164E56F82220D9B10C2918D1FC
:103E6000D86800F0030002281AD003281AD01046A0
:103E7000D968DA68C1F30211C2F306224243491C31
:103E8000B2FBF1F0D968C1F34161491C4900B0FBB4
:103E9000F1F070BD104670BD204670BD284670BD63
:103EA0002046E5E72846E3E7001002400024F4003E
:103EB00090BE01082DE9F84304006ED0FB4DA868C0
:103EC00000F00C06E86800F003072078C00663D510
:103ED00076B10C2E01D1012F0AD0A06900282868E4
:103EE00078D040F001002860FFF76CF980465BE075
:103EF0002868800702D5A0690028DED0216A2868DA
:103F0000000703D5286800F0F00004E0D5F894001D
:103F1000F02202EA1010814216D9084601F066FA32
:103F200000283AD1286840F0080028602868216AF3
:103F300020F0F000084328606868E16920F47F40C1
:103F400040EA0120686015E0286840F00800286019
:103F50002868216A20F0F000084328606868E16959
:103F600020F47F4040EA01206860206A01F03EFAB8
:103F70000028D6D1FFF74CFFA968CD4AC1F3031141
:103F8000515C01F01F01C840CA490860CA48006876
:103F9000FFF73CFC00287DD12CE0C6E0FFF712F9CA
:103FA000A0EB0800022876D828688007F6D5286894
:103FB00040F0080028602868216A20F0F0000843DB
:103FC00028606868E16920F47F4040EA0120686069
:103FD00010E0FFE720F001002860FFF7F3F88046CB
:103FE00005E0FFF7EFF8A0EB08000228DBD828680F
:103FF0008007F6D42078C00740D0082E18D00C2EA9
:1040000001D1032F14D06068B0F5803F17D0B0F510
:10401000A02F286817D020F480302860286820F46A
:10402000802028606068E0B1FFF7CCF8804614E09B
:104030002868800322D56068002876D01EE02868B2
:1040400040F48030EDE740F480202860F7E7FFF788
:10405000B9F8A0EB08006428A5D828688003F6D535
:104060000CE0FFF7AFF8804605E0FFF7ABF8A0EBF8
:104070000800642897D828688003F6D42078800741
:1040800039D5042E11D00C2E01D1022F0DD0E068AD
:10409000002801E05EE1B3E028681DD040F48070A4
:1040A0002860FFF78FF807460BE0286840050BD51E
:1040B000E0680028C1D007E0FFF784F8C01B0228A1
:1040C00094D828684005F7D56868217C20F0F8501E
:1040D00040EA016068600EE020F480702860FFF71D
:1040E00071F8074604E0FFF76DF8C01B0228B3D84B
:1040F00028684005F7D42078000728D56069002893
:10410000D5F8940012D040F00100C5F89400FFF7F4
:1041100059F8074604E0FFF755F8C01B02286FD88E
:10412000D5F894008007F6D511E049E120F00100B0
:10413000C5F89400FFF746F8074604E0FFF742F899
:10414000C01B02285CD8D5F894008007F6D42078EC
:10415000400766D5A86D4FF00008C00009D4A86DCF
:1041600040F08050A865A86D4FF0010800F0805025
:10417000009052480168C90511D40168814641F494
:1041800080710160FFF71EF8074604E0FFF71AF898
:10419000C01B022834D8D9F80000C005F6D5A068A5
:1041A000012815D00528D5F8900016D020F0010080
:1041B000C5F89000D5F8900020F00400C5F89000F4
:1041C000A06841F28839B8B1FEF7FCFF07460EE05F
:1041D000D5F8900040F00100F0E740F00400C5F889
:1041E0009000F5E7FEF7EEFFC11B494508D8D5F86A
:1041F00090008007F6D50DE0FEF7E4FF074605E0E6
:1042000081E0FEF7DFFFC11B49457CD8D5F890005F
:104210008007F6D4B8F1000F03D0A86D20F08050CD
:10422000A8652078800627D5606A0028D5F8980010
:1042300011D040F00100C5F89800FEF7C3FF074613
:1042400004E0FEF7BFFFC01B02285CD8D5F8980039
:104250008007F6D510E020F00100C5F89800FEF7C1
:10426000B1FF074604E0FEF7ADFFC01B022870D87F
:10427000D5F898008007F6D4A06AB0B10C2E70D0A3
:104280000228286820F0807028601BD02868000170
:1042900003D4E86820F00300E860E86808490840B3
:1042A000E860FEF78FFF044656E08BE00010024006
:1042B00080BE01081C020020F001002000700040B8
:1042C000FFFFEEFEFEF77EFF064604E0FEF77AFFF4
:1042D000801B02283DD828688001F7D4F4E90B013F
:1042E0006FF00F0202EB01110843218A52044908C2
:1042F00002EB4151A26841EA02210843217D4FF0BF
:104300007E42490800E024E002EB41610843217B42
:1043100040EAC160E9682C4A11400843E860286817
:1043200040F080702860E86840F08070E860FEF738
:1043300049FF044604E0FEF745FF001B022808D8A9
:1043400028688001F7D53DE0FEF73CFF001B0228FE
:1043500002D90320BDE8F88328688001F4D431E055
:10436000FFE70128F6D0E868E26A00F00301914215
:1043700026D1216B00F070020901103991421FD142
:10438000626B00F4FE41B1EB022F19D194F8382092
:1043900000F07841B1EBC26F12D1A18F00F4C002DE
:1043A00049084905A1F50011914209D194F840103E
:1043B00000F0C06049084906A1F10071814201D0B6
:1043C0000120C7E70020C5E78C809D01704770473A
:1043D000704710B5040003D094F83D0010B107E019
:1043E000012010BD002084F83C00204600F00CF8AD
:1043F000022084F83D00211D206801F099FC012075
:1044000084F83D00002010BD38B5114CA06D40F07F
:104410000100A065A06D002200F0010000900321C2
:104420001C20FFF755FA1C20FFF744FA206E40F4D9
:1044300080302066206E002200F48030009003213E
:104440001820FFF745FABDE838401820FFF732BAC8
:10445000001002400168CA6842F00102CA600168A7
:104460008868064A1040062806D0B0F5803F03D081
:10447000086840F001000860002070470700010054
:10448000704770B50446006801694FF00005C943E4
:10449000890715D4C168C943890711D4E91E016190
:1044A00001202077206880698007204602D0FFF72E
:1044B000E7FF04E000F0A7F8204600F0A5F8257714
:1044C00020680169C943490717D4C168C94349072E
:1044D00013D46FF004010161022020772068806905
:1044E00010F4407F204602D0FFF7CAFF04E000F03E
:1044F0008AF8204600F088F8257720680169C943CA
:10450000090716D4C168C943090712D46FF008011E
:104510000161042020772068C0698007204602D00E
:10452000FFF7AEFF04E000F06EF8204600F06CF8F4
:10453000257720680169C943C90617D4C168C943F2
:10454000C90613D46FF0100101610820207720689C
:10455000C06910F4407F204602D0FFF791FF04E0CD
:1045600000F051F8204600F04FF8257720680169E7
:10457000C943C90708D1C168C943C90704D1891E05
:104580000161204600F042F820680169C94309062C
:1045900009D4C168C943090605D46FF080010161DF
:1045A0002046FFF714FF20680169C943C90509D4F3
:1045B000C168C943090605D46FF4807101612046C2
:1045C000FFF704FF20680169C943490609D4C1689F
:1045D000C943490605D46FF040010161204600F04F
:1045E00033F820680169C94389060BD4C168C943FF
:1045F000890607D46FF0200101612046BDE87040B4
:10460000FFF7E6BE70BD70477047000010B5006848
:104610000A49884210D1FFF7E1F809488168491C2E
:1046200081600848018841F28832914202D20188B3
:10463000491C00E00021018010BD0000002C014059
:10464000B0020020540400207047704770470000FB
:104650002DE9F04102680446D0691168936810F0B2
:104660000F0F4FF000055BD003F0010601F49077C7
:10467000374369D0C70707D0CF0505D50127176293
:10468000E26F42F00102E267820708D5DA0706D03E
:10469000276802223A62E26F42F00402E2674207B0
:1046A00008D5DA0706D0236804221A62E26F42F0C6
:1046B0000202E26702070AD501F02002324306D067
:1046C000236808221A62E26F42F00802E267E26F92
:1046D000002A32D0800605D5880603D5216E09B19F
:1046E00020468847E06F21688968490601D40007A1
:1046F00025D5204601F0ECFB20688168490619D5D4
:10470000816821F040018160E06E98B120498163A9
:10471000E06EFEF79AF900280FD0E06E816B06E09C
:10472000860611D58E060FD5216E1EE02046BDE807
:10473000F04108472046FFF789FFBDE8F081204699
:10474000FFF784FFE567F8E7C60209D55B0207D5E6
:104750004FF4801010622046BDE8F041FFF775BFAE
:10476000030605D50B0603D5616E0029DED1E4E70B
:104770004006E2D54806E0D51168204621F0400108
:10478000116020216167656600F00AFAD5E7000034
:10479000BD5E010810B5040002D0606F10B107E0E3
:1047A000012010BD002084F87000204600F026F89B
:1047B000242060672068016821F001010160204623
:1047C00001F00EFC0128ECD0606A10B1204601F027
:1047D000E5FA2068416821F49041416020688168D1
:1047E00021F02A0181602068016841F00101016027
:1047F0002046BDE8104001F035BB00002DE9F04334
:1048000087B0054614216846FBF7FDFD2B49286853
:1048100000262B4C02274FF003084FF0070988426F
:1048200022D1A06D40F40030A065A06D00F40030EE
:104830000590E06C40F00100E064E06C02AA00F03A
:10484000010005900C20CDE9000782E8400369468D
:104850004FF09040FEF7E8FB012200212620FFF7F1
:1048600037F82620FFF726F816492868884221D114
:10487000206E40F480402066206E00F48040059059
:10488000E06C40F00200E064E06C02AA00F002007C
:104890000590C020CDE9000782E8400369460A4838
:1048A000FEF7C2FB002201212520FFF711F8252089
:1048B000FFF700F807B0BDE8F083000000440040B7
:1048C00000100240003801400004004870B5836FBA
:1048D000202B51D121B11AB1284B1B784BB901E0E3
:1048E000012070BD90F87040012C45D0012480F863
:1048F00070404165A0F85820A0F85A2000220266B6
:1049000081684FF48054FF25A14204D10169E1B9C7
:1049100040F2FF111FE07F26A9B1B1F1805F17D0EF
:10492000A0F85C20C2672221816701688D6845F08C
:1049300001058D608168A14201D1016989B11049E9
:10494000016693B90FE0016941B9A0F85C50E9E74D
:10495000016919B13F21A0F85C10E3E7A0F85C60A1
:10496000E0E70849ECE780F870200068016841F44E
:1049700090710160002070BD022070BD23000020F6
:10498000875F01082D5F01082DE9F04706460068A2
:1049900049494A4F884268D1494A3979494C107B84
:1049A0000123012802D0914628B157E023704648E0
:1049B000F7F7D3FD52E0454D2370454C28889846C3
:1049C000502803D22154401C288001E005F0CAFA87
:1049D00028884049404A012815D0032817D00428C8
:1049E0001AD0072825D00988884237D12078FF2897
:1049F00003D099F8061088422ED138490A2081F850
:104A0000008010802AE0502008800320F9E76078B9
:104A1000192823D1062015E0E078A37800EB0320C5
:104A20000A281BD16078062818D10C200880142091
:104A3000E7E76078032807D0062805D0102805D0BE
:104A40004FF40070088009E00820FBE7A07900F12E
:104A500009030B800830D4E705F084FA17490122D6
:104A6000091D1F48FFF732FFB8701E4930688842A1
:104A70001FD11D4978798A1C4B7A9854487A401C7A
:104A8000C0B2487207280CD38878FE2807D1C878AE
:104A9000042804D188794A7900EB0220088000209C
:104AA000487206490E480122491D8030FFF70EFF6B
:104AB000F870BDE8F08700000044004000000020CE
:104AC000AC05002083010020D4B400202600002083
:104AD000C205002024000020460000202200002003
:104AE000AC04002000380140520900202DE9F843B1
:104AF0000446406F1F4615460E4620284ED1CEB1C3
:104B0000C5B194F87000012848D0012084F87000E5
:104B10004FF00008C4F87C8021206067FEF752FB4C
:104B2000A4F850508146A4F85250A068B0F5805FB8
:104B300003D004E00120BDE8F883206910B13546B8
:104B4000002610E000250EE08021204601F06CFBDD
:104B5000B8B9C5B115F8010B21680885B4F8520041
:104B6000401EA4F85200B4F852004B464FF0000229
:104B700000970028E8D14FF04001204601F054FB97
:104B800030B10320D7E736F8020BC0F30800E3E7A3
:104B90002020606784F870800020CCE70220CAE7FC
:104BA0000068064B01220649984201D10A707047FD
:104BB000044B9842FBD14A7070470000004400400B
:104BC0000000002000380140FEE7000010B5034857
:104BD000FEF7FEFABDE8104000F06AB85C0B00205A
:104BE00010B59CB04020009080010B906846FEF705
:104BF000F1FE154CE06C40F00100E064E06C15A99A
:104C000000F001001A904FF4C06015901220169029
:104C10000120179002201890042019904FF0904026
:104C2000FEF702FAA06D40F40010A065A06D00F43C
:104C300000101A90A06B40F40010A063A06B20F449
:104C40000010A0631CB010BD001002403EB5144619
:104C5000094A0D4606991268CDE9003102920146D3
:104C600023462A460548FEF7E3FB10F0FF0401D077
:104C7000FFF7ACFF20463EBDFC0000205C0B00208F
:104C800017B5094C83B00A462468012305A98DE8AD
:104C90001A0001460548FEF777FC040002D0FFF732
:104CA00095FF204606B010BDFC0000205C0B0020E4
:104CB00010B50E48FEF7A5FA002815D10B480C498F
:104CC0000122016040F6146141600021C0E9021236
:104CD000016141618161C1610162FFF781FFBDE84E
:104CE00010400248FEF790BA10BD00005C0B002097
:104CF0000054004001688A69D243920701D400221F
:104D00008A6200688169C943C90703D0816941F09B
:104D100001018161704700002DE9F04104460068FF
:104D200016460D468069C043C00637D44FF00008D0
:104D3000202720688069C043800616D5681CF8D0FB
:104D4000FEF740FA801BA84201D8002DF1D154F89B
:104D5000440F40F0200044F80409677084F8028092
:104D600084F800800120BDE8F08121681020C8612E
:104D70002068C7612046FFF7BDFF54F8440B416827
:104D8000074A11404160206840F0040044F82009BF
:104D9000677784F81E8084F81C80E3E70020E2E750
:104DA00000E800FE2DE9F84304461646DDE90897C1
:104DB00014489846DAB200900023204600F056F8D6
:104DC0003A464946204600F0B9F8B8B9F5B2B8F10C
:104DD000010F08D02168300A88623A4649462046C9
:104DE00000F0ACF850B9206885624B4600224021A3
:104DF0002046009700F050F8002800D00120BDE8C0
:104E0000F8830000002000802DE9F8430446164690
:104E100015489846DDE90897DAB2C30200902046AB
:104E200000F024F83A464946204600F087F8B8B921
:104E3000F5B2B8F1010F08D02168300A88623A460D
:104E40004946204600F07AF850B9206885624B4602
:104E5000002280212046009700F01EF8002800D094
:104E60000120BDE8F883000000200080F0B5006854
:104E7000059C45684FF48066064FC1F3090106EAB8
:104E8000545641EA02413E431943B54321430D4381
:104E90004560F0BDFF63FF032DE9F0411D46174655
:104EA0000E460446DDF8188008E0681C06D0FEF7C0
:104EB00089F9A0EB0800A8420BD855B12068806999
:104EC00036EA000012D00020B842EED00020BDE843
:104ED000F08154F8440F40F0200044F804092020E9
:104EE00060700020A07020700120F0E70120EBE747
:104EF00070B516460D4604460DE03246294620465A
:104F0000FFF70AFF08B1012070BDFEF75BF9801BB7
:104F1000A84207D835B120688069C0438006ECD428
:104F2000002070BD54F8440F40F0200044F80409FC
:104F3000202060700020A0702070E4E770B5164655
:104F40000D4604460FE0324629462046FFF7E4FEB0
:104F500008B1012070BD681C05D0FEF733F9801B35
:104F6000A84207D835B120688069C0438007EAD4D9
:104F7000002070BD54F8440F40F0200044F80409AC
:104F8000202060700020A0702070E2E710B500F0D3
:104F900093F800F0A1FA00F0B7F80A2002F0B0FD93
:104FA00000F078F80A2002F0ABFDBDE8104000F0F8
:104FB00083B8000030B51A4987B0CA6C42F00102CC
:104FC000CA64CA6C02F001020592CA6C42F0020285
:104FD000CA64C96C012401F0020102254FF090421D
:104FE000059104280DD0022809D14FF4C060CDE905
:104FF000000469461046CDE90245FEF715F807B0F2
:1050000030BD8020CDE9000469461046CDE9024557
:10501000FEF70AF81020CDE9000469460148EAE7E6
:10502000001002400004004810B500F045F800F000
:1050300053FA00F053F80A2002F062FD00F02AF85B
:105040000A2002F05DFDBDE8104000F035B870B5F3
:105050000646002400F022FA002500F02DF80A2070
:1050600002F04EFD00F016F86006040E00F0FCF9A8
:1050700008B1641CE4B20A2002F042FD6D1CEDB2DE
:10508000082DEAD31EB1FFF781FF204670BDFFF760
:10509000CBFFFAE7074801784FF09040042905D08C
:1050A000022906D101220902FEF787B801228021D8
:1050B000FAE7704786010020074801784FF09040DA
:1050C000042905D0022906D100220902FEF775B88D
:1050D00000228021FAE77047860100200848007806
:1050E000042807D0022809D1012241024FF0904044
:1050F000FEF763B8012210210248F9E7704700006B
:10510000860100200004004808480078042807D0E1
:10511000022809D1002241024FF09040FEF74DB81D
:10512000002210210248F9E77047000086010020A4
:105130000004004870B5054600F0CEF9FFF7BCFF4B
:105140000024280602D5FFF7C9FF01E0FFF7DCFFC6
:105150006806050E0A2002F0D3FCFFF79BFF0A2029
:1051600002F0CEFCFFF7A8FF0A2002F0C9FC641C85
:10517000E4B2082CE5D370BD10B500F0ADF9FFF72F
:10518000ADFFFFF787FF0A2002F0BAFCFFF7BCFF74
:105190000A2002F0B5FCBDE81040FFF78DBF10B546
:1051A00000F09AF9FFF788FFFFF7AEFF0A2002F040
:1051B000A7FCFFF76FFFFFF791FFBDE810400A2043
:1051C00002F09EBC10B5002400F068F9FFF786FFDE
:1051D0000A2002F095FCFFF75DFF0A2002F090FC28
:1051E00007E0641CE4B2FA2C03D9FFF7D8FF0120D2
:1051F00010BD00F039F90028F3D1FFF75DFF002062
:1052000010BD000010B5F5F7FFFE0B4881790B4883
:1052100041704068F5F7FFFEF3F7B2FF0020F7F7A3
:105220002BFA0749002008700649087006490870E3
:1052300006490B20087010BDAC050020800200203C
:10524000C4020020C5020020C7020020C6020020C0
:105250004FF400414FF09040FDF7A8BF00EB8100F4
:10526000006E00F0F84070478068C0F3C0007047DF
:105270008068C0F3000070478068C0F3800070470A
:10528000C06810F4406F01D00020704701207047C3
:10529000042303EAD15310B518444369C1F3045100
:1052A00007248C40A3438A401343436110BD00EBA5
:1052B0008100016E21F00041114301667047FEE755
:1052C000704770472DE9F041434E05468846F06827
:1052D0000024810728680ED0F16801F003018142A3
:1052E00007D130B1F0686968C0F30210401C8842F1
:1052F0001FD001246DE0012809D002280AD003281C
:10530000F7D13168890309D43168490304E0316871
:10531000890701E0316849050029EADAF1686A681D
:105320006FF00F0321F0730103EB021211430143ED
:10533000F160306820F080603060FDF743FF074681
:1053400004E0FDF73FFFC01B022838D83068000199
:10535000F7D474BBB8F1000F18D0B8F1010F1DD00D
:10536000287D4FF07E41400801EB4060A96840EA8B
:1053700001203169194A114008433061306840F01A
:1053800080603060FDF71EFF07461AE0A868297BA1
:10539000000240EAC1603169114AECE7288A1149EC
:1053A000400801EB4050A96840EA012031690E4AEB
:1053B000E1E70EE0FDF706FFC01B022801D9032438
:1053C00007E030680001F5D51CB93069A9690843C8
:1053D00030612046BDE8F08100100240FF80FFF9F7
:1053E000FF80FF070000E0FFFF809FFFF8B51C4E25
:1053F00005460024B06DC00002D5FEF7E3FA0DE0CB
:10540000B06D40F08050B065B06D00F080500090FD
:10541000FEF7D8FAB16D21F08051B165B0F5007F8B
:1054200004D0802D07D94FF003040AE0802D08D95D
:10543000A02D01D804E001D1022402E0702D00D19A
:1054400001240848016821F0070121430160006838
:1054500000F00700A04201D00120F8BD0020F8BDF7
:10546000001002400020024007480078042806D0BF
:10547000022807D141024FF09040FDF792BE102163
:105480000248FAE770470000860100200004004847
:105490000148C07970470000AC05002000B50C48F9
:1054A000002185B0007804280BD0022807D14002E3
:1054B000CDE9000169464FF09040FDF7B5FD05B01C
:1054C00000BD1020CDE9000169460248F5E7000063
:1054D000860100200004004800B50E480121022288
:1054E000007885B004280DD0022809D14002CDE90A
:1054F0000212CDE9000169464FF09040FDF794FD9E
:1055000005B000BD1020CDE90212CDE900016946C9
:105510000148F3E7860100200004004810B52DED96
:10552000048BB0EE409AF0EE609A19EE100AFBF789
:1055300081FA9FED261B53EC112BFBF7B6F841ECDB
:10554000180B19EE100AFBF775FA9FED221B53ECAE
:10555000112BFBF759F953EC182BFBF7CAF941EC67
:10556000110B9FED1E0B01F06BF99FED1E1B51EC13
:10557000100B53EC112BFBF747F9FBF76EFA00EE1B
:10558000100ADFED1A0A19EE100A20EE290AC0EE01
:10559000209AFBF74FFA9FED161B53EC112BFBF7EC
:1055A00084F89FED150A41EC180B29EE800A10EEE5
:1055B000100AFBF73FFA53EC182BFBF79AF9FBF7AD
:1055C0004CFABDEC048B00EE100A10BD9A99999923
:1055D00099A96D400000000000001E40000000007E
:1055E00000002440713D0AD7A37018400000C84253
:1055F00066666666661271400000594310B510EE8B
:10560000900A2DED088BB0EE40BAFBF713FA41EC8F
:10561000100B01F07DF89FED281B51EC100B53ECA3
:10562000112BFBF7E3F841EC180B1BEE100AFBF70C
:1056300001FA9FED239B53EC192BFBF736F841EC55
:105640001A0B1BEE100AFBF7F5F99FED1F1B53EC2D
:10565000112BFBF7D9F853EC1A2BFBF74AF99FED06
:105660001CAB53EC1A2BFBF720F853EC182BFBF771
:105670001CF8FBF7F2F90446FBF7DCF99FED161B6B
:1056800053EC112BFBF7B2F841EC180B2046FBF75B
:10569000D1F953EC1A2BFBF7ACF853EC192BFBF7B1
:1056A000B3F853EC182BFBF724F9FBF7D6F9BDEC54
:1056B000088B00EE100A10BD000000000000004042
:1056C0009A99999999A96D400000000000001E4028
:1056D00085B185200725E53F185B087250522040B0
:1056E00010B52DED048BB0EE408AF0EE608A18EE16
:1056F000100AFBF79FF99FED3F1B53EC112BFAF7B4
:10570000D4FF41EC190B18EE100AFBF793F99FED4B
:105710003B1B53EC112BFBF777F853EC192BFBF7E2
:10572000E8F841EC110B9FED370B01F089F89FED84
:10573000371B51EC100B53EC112BFBF765F8FBF703
:105740008CF900EE100ADFED330A20EE280AC0EED5
:10575000208A18EE900AFBF76DF99FED2F1B53EC92
:10576000112BFBF746F841EC190B18EE900AFBF7EA
:1057700061F953EC192BFBF7BCF89FED291B53EC97
:10578000112BFBF741F89FED281B53EC112BFBF776
:10579000B0F8FBF762F9FBF74DF941EC190B18EE85
:1057A000100AFBF747F99FED221B53EC112BFBF777
:1057B0002BF89FED211B53EC112BFAF776FF53ECDE
:1057C000192BFBF721F841EC190B18EE100AFBF727
:1057D00031F99FED1B1B53EC112BFBF715F853EC24
:1057E000192BFAF762FFFBF738F9BDEC048B00EEDA
:1057F000100A10BD9A99999999A96D40000000006E
:1058000000001E400000000000002440713D0AD747
:10581000A37018400000C8420000000000AA8F409A
:1058200000000000007083400000000000408F4036
:10583000713D0AD7A370FD3F000000000088A3401F
:10584000295C8FC2F528F03F10B501784FF6FF7242
:10585000407802EA0121084480B2FBF7CAF89FEDC4
:10586000081B53EC112BFAF7CFFF9FED071B53ECEE
:10587000112BFBF73EF8FBF7F0F800EE100A10BD15
:10588000000000000000594000000000E0FFEF4071
:1058900010B501784FF6FF72407802EA0121084402
:1058A00080B2FBF7A6F89FED0A1B53EC112BFAF719
:1058B000ABFF9FED091B53EC112BFBF71AF8FBF71D
:1058C000CCF800EE100ADFED060A30EE600A10BDDB
:1058D0000000000000E0654000000000E0FFEF4035
:1058E000000034420149405870470000000002089F
:1058F00070B50C460A460749002301440D46184678
:10590000FDF7AEFA044A012110B92868A04200D080
:10591000517070BD000002086801002070474FF40C
:1059200080514FF0904308B1012200E00022184658
:10593000FDF743BC704770477047704770470000E1
:105940000E4908784A78CB7800EB02208A78120456
:1059500002EB036202440A4840F8B42F89790175CA
:1059600000F86B1C0749142249688161012100F885
:105970006C1C034804493430FAF72CBDAC050020F8
:105980004C870020800200203000002010B55020FD
:1059900080F31188BFF34F8FBFF36F8F06F04EF87F
:1059A00018B104494FF080500860002080F311883E
:1059B00010BD000004ED00E02DE9F04FADB0442132
:1059C0006846FAF720FD142111A8FAF71CFD4FF4E0
:1059D0000070FDF7C3FF644C00252570442116A814
:1059E000FAF711FD142127A8FAF70DFD01264FF44F
:1059F000A020CDE916604FF0020A4FF00308CDE970
:105A000020A84FF0140B0721CDE9241ACDE9226B11
:105A1000CDF898A016A8FEF74DFADFF850910F27A1
:105A200008B153A00EE0D9F80000800329D5CDE9D4
:105A3000288527972A95042127A82B95FEF70EF98C
:105A4000B0B156A002F0F0FC4FF48030CDE9006018
:105A50001421CDE90AA8CDE90C610721CDE90E1A80
:105A6000CDF840A06846FEF725FA60B154A019E0D1
:105A7000042020705A4931F8520F401C088059A068
:105A80005AE05EA0DEE7D9F80000800327D5CDE913
:105A9000128511971495042111A81595FEF7DEF8CB
:105AA000D0B160A002F0C0FC4FF4A020CDE90060AE
:105AB0003146CDF828A0CDE90B8114210D910721A5
:105AC000CDE90E1AB3464646CDF840A06846FEF72B
:105AD000F1F930B159A013E0267062A02CE063A068
:105AE000E0E7D9F8000080032BD5CDE912651197C6
:105AF0001495042111A81595FEF7B0F8C8B162A05D
:105B000002F092FCA8461020CDE906B80090602172
:105B100008912820CDE90CB0CDE90AAB0720CDE9EA
:105B20000E0A5546CDF840A06846FEF7C3F9B0B955
:105B300009E0052020705CA002F076FC2DB000F09A
:105B4000CBB85DA0DCE7CDE912681197CDF85080A5
:105B5000042111A8CDF85480FEF780F808B1267012
:105B6000ECE72570EAE70000800100200010024009
:105B700048414C5F5243435F4F7363436F6E6669A6
:105B800067284853455F4259504153532D66697207
:105B9000737429206661696C656400004853455F31
:105BA0004259504153532D666972737420436C6F90
:105BB000636B436F6E666967206661696C6564003C
:105BC00048414C5F5243435F4F7363436F6E666956
:105BD000672848534529206661696C6564000000A8
:105BE000EE0800204853455F4259504153532D66FB
:105BF000697273742B504C4C000000004853455F91
:105C00004259504153532D6669727374206E6F74FC
:105C100020726561647920616674657220706F6CB2
:105C20006C00000048534520436C6F636B436F6EFC
:105C3000666967206661696C6564000048414C5F75
:105C40005243435F4F7363436F6E666967284853DF
:105C5000455F42595041535329206661696C656420
:105C6000000000004853452B504C4C004853452041
:105C70006E6F74207265616479206166746572204C
:105C8000706F6C6C000000004853455F42595041F2
:105C9000535320436C6F636B436F6E666967206676
:105CA00061696C65640000004853455F425950418A
:105CB00053532B504C4C00004853455F42595041C0
:105CC0005353206E6F74207265616479206166742D
:105CD000657220706F6C6C0030BCBDE8C08F000036
:105CE0000D48016841F4700101600C48016841F001
:105CF00001010160002181600268094B1A400260C5
:105D00008214C260026822F480220260816102492A
:105D1000C00380390860704788ED00E00010024041
:105D2000FFFFF6EA0148FEF7ACBB00003C10002084
:105D3000F0B50268164C4FF08047A04201D0B8423F
:105D400003D122F070034A681A43124D124EA0424A
:105D500005D0B84203D0A84201D0B04203D122F40A
:105D60004073CA681A434B6922F080021A430260EA
:105D70008A68C2620A688262A04203D0A84201D047
:105D8000B04201D10969016301214161F0BD000008
:105D9000002C0140004001400044014090F82410D4
:105DA000C90706D001684A68836A22F400321A43A0
:105DB0004A6090F82410890706D501684A68C36ACA
:105DC00022F480321A434A6090F82410490706D51D
:105DD00001684A68036B22F480221A434A6090F8F3
:105DE0002410090706D501684A68436B22F4004273
:105DF0001A434A6090F82410C90606D501688A68DB
:105E0000836B22F480521A438A6090F8241089062A
:105E100006D501688A68C36B22F400521A438A606F
:105E200090F82410490611D501684A68036C22F4E1
:105E300080121A434A60016CB1F5801F06D10168D7
:105E40004A68436C22F4C0021A434A6090F8241056
:105E5000090606D501684A68806C22F400220243D4
:105E60004A607047F8B500250446C567FDF7AAF9F2
:105E70000746206800686FF07E46000708D53B465D
:105E800000224FF400112046009600F0CDF960B9D1
:105E90002068006840070AD53B4600224FF4800185
:105EA0002046009600F0C0F908B10320F8BD20207C
:105EB0006067A06784F870500020F8BD10B5806A54
:105EC0000021A0F85A10A0F85210FEF7BFFB10BD39
:105ED00001680A6822F490720A6001688A6822F0F8
:105EE00001028A602021816700210166704700005D
:105EF0000D48C1794FF4E130062912D2DFE801F0F4
:105F00000306090C110F4FF416500AE04FF49640A7
:105F100007E04FF4164004E04FF4614001E04FF415
:105F2000963004F099BE0000AC05002010B5B0F822
:105F30005C20836F0168222B04D0088B40F008009E
:105F4000088310BD898C436D11401980416D891CF7
:105F50004165B0F85A10491EA0F85A10B0F85A100E
:105F60000029EED101680A6822F490720A60016883
:105F70008A6822F001028A6020218167002101667F
:105F8000FEF702FD10BD10B5B0F85C20836F01680C
:105F9000222B04D0088B40F00800088310BD898CA8
:105FA0001140426D1170416D491C4165B0F85A10A5
:105FB000491EA0F85A10B0F85A100029EED1016815
:105FC0000A6822F490720A6001688A6822F001026D
:105FD0008A602021816700210166FEF7D5FC10BD93
:105FE0002DE9F047044600682369A268E6691A4370
:105FF0006369002533431A43824903682F46824E62
:1060000033401343036020684268E36822F440523F
:106010001A4342602268A0698A4201D0236A184369
:10602000936823F4306303439360784B2268784885
:106030009A420DD1D0F8880010F0030006D0012854
:1060400039D0022835D0032821D136E001261FE0BF
:10605000704B9A420BD1D0F8880010F00C0026D07B
:10606000042828D0082824D00C2810D125E08A4202
:106070000DD1D0F8880010F4406018D0B0F5806FD2
:1060800019D0B0F5006F14D0B0F5406F15D01026C0
:10609000614B4FF000084FF400408A424CD176B17A
:1060A000022E0FD0042E0FD0082E18D10FE000269C
:1060B000EEE70226ECE70426EAE70826E8E7FDF724
:1060C00083FE03E0184602E0FDF7A2FE98B3626883
:1060D00002EB4201814202D8B0EB023F01D9012715
:1060E00089E066B1022E0DD0042E13D0082E1BD0ED
:1060F00001274A49A5F5407088427AD9EFE7FDF7B4
:1061000063FE09E05008464B11E00023FAF72EF930
:106110000546EEE7FDF77CFE6268010E05025008B9
:10612000281841EB0801F0E750084FF40003C018AD
:1061300048F10001E9E75EE0E1694FF6EF7981425D
:106140002ED1092E1DD2DFE806F00508121C151C01
:106150001C1C1800FDF738FE01E0FDF747FE41006A
:10616000606801EB5001B1FBF0F085B20AE02D4907
:106170006068F6E7FDF74CFEF1E74FF480316068A8
:10618000EFE70127A5F110004845A8D84FF6F071B8
:1061900005EA0100C5F3420108432168C8602AE00E
:1061A000092E21D2DFE806F0050812201620202053
:1061B0001A00FDF709FE01E0FDF718FE01466068D0
:1061C00001EB5001B1FBF0F085B20EE0606803EB2B
:1061D0005001F7E7FDF71CFEF0E70AE0616800EB0D
:1061E0005100B0FBF1F0EFE70127A5F110004845A1
:1061F00084D82068C560C4F860803846C4F86480DC
:10620000BDE8F08700800040F369FFEF00380140EF
:1062100000100240004400400024F400FFFC0F0086
:10622000000024F40048E8012DE9F0411E4617461D
:1062300088460446069D07E0681C05D0FCF7C2FFAF
:10624000801BA8420BD855B12068C16938EA01000B
:1062500017D00020B842EFD00020BDE8F0812068C0
:10626000016821F4D07101602068816821F001018A
:10627000816020206067A067002084F87000032000
:10628000EBE70120E6E700000148FEF7E1B9000076
:106290002C0500200148FEF7DBB90000AC0400200B
:1062A00010B572B60549064B0246C979064853F83F
:1062B0002130044903F018FC62B610BDAC05002083
:1062C000C8BB0108C2070020AC040020FEE703B4ED
:1062D00001984100009850EAC12018BF04204A0DDF
:1062E00018BF40F0010040F2FF72B2EB515F08BFEF
:1062F00040F00200012808BF052002B070470907DE
:10630000090E002804DB00F1E02080F8001470473B
:1063100000F00F0000F1E02080F8141D704700002D
:1063200000487047A804002070B5D94B00242DED1B
:10633000020B2DED108BDDE91010984205DA20F0EC
:1063400000429A4201D809D141B19DED100B00F0F5
:10635000CDB902B0BDE8704001F046B9B0F5801F7C
:1063600026DA11430BD0002813DA012001F090F94E
:1063700000F0C2B902B0BDE8704001F049B9022096
:1063800001F086F901F018F951EC100B81F0004191
:106390009EE06FF035049FEDC00B53EC102B9DED8C
:1063A000100B51EC100BFAF72FFACDE9100108464B
:1063B00004EB2051C0F31304B948A1F2FF3120448B
:1063C00000F4801080F07F6282F04052224301EBA3
:1063D00020559FEDB50B119253EC102B9DED100B3A
:1063E00051EC100BFAF702FA41EC180BA01CC0F3A9
:1063F00013009FEDAFDB9FEDB0EBB14E7E44032861
:106400006CD296ED000B51EC180B53EC102BFBF7F4
:10641000D1F81DD1002D01BF96ED000BBDEC108B06
:1064200002B070BD2846FAF7D3FA41EC180B53ECD2
:106430001D2BFAF7E9F941EC190B53EC1E2B51EC2B
:10644000180BFAF7E1F953EC192BFAF72EF93FE0A4
:106450009FED9D0B51EC180B53EC102BFAF7D4F970
:106460009FED9B1B53EC112BFAF7C3F941EC190B71
:1064700053EC182B51EC180BFAF7C6F953EC192B07
:10648000FAF7C2F941EC190B002D04BF53EC192B9C
:1064900051EC180B1AD02846FAF79AFA41EC1A0B6D
:1064A00053EC1D2BFAF7B0F953EC192BFAF7A1F9BD
:1064B00053EC182BFAF79AF941EC180B53EC1E2BFE
:1064C00051EC1A0BFAF7A0F953EC182BFAF78EF9E6
:1064D00000F018B902B041EC100B70BD9FED7E0BBF
:1064E00051EC180B53EC102BFAF7DFF841EC100BC2
:1064F00051EC180B53EC102BFAF7FBF941EC190B8C
:106500002846FAF765FA41EC1B0B53EC192B51ECBA
:10651000190BFAF779F941EC1A0B714853EC1A2B65
:10652000261851EC1A0BFAF76FF941EC1F0B6D4866
:10653000C4F1510404F5D724B0EE4F0AF0EE6F0A0F
:106540000321784400F0BCFF53EC1F2B51EC100BDF
:10655000FAF75AF941EC1C0B6348B0EE4F0AF0EE23
:106560006F0A0421784400F0ABFF53EC1A2B51EC76
:10657000100BFAF749F9344353EC1C2BFAF795F852
:1065800041EC1C0B002C4CDD9FED510B51EC180B1A
:1065900053EC102BFAF738F953EC182BFAF734F9BF
:1065A00041EC1A0B55B353EC1D2B51EC1B0BFAF7B6
:1065B0002BF941EC1D0B53EC1C2B51EC1A0BFAF789
:1065C00074F853EC192BFAF71FF953EC1D2BFAF75B
:1065D0006CF853EC1A2BFAF70CF953EC182BFAF76A
:1065E00005F941EC180B53EC1E2B51EC1B0BFAF781
:1065F0000BF953EC182BFAF7F9F869E753EC1C2B5D
:1066000051EC1A0BFAF751F853EC192BFAF7FCF886
:1066100053EC1A2BFAF7EDF853EC182BFAF7E9F8CC
:1066200056E735B353EC1D2B51EC1B0BFAF7ECF886
:1066300041EC1A0B53EC1C2B51EC180BFAF7D6F863
:1066400053EC192BFAF7E0F853EC1A2BFAF7CEF8C3
:1066500053EC182BFAF7CAF841EC180B53EC1E2B2D
:1066600051EC1B0BFAF7D0F853EC182BFAF7BEF8E5
:106670002EE753EC1C2B51EC180BFAF7B7F853EC40
:10668000192BFAF7C1F853EC182BFAF7B2F81FE7F9
:106690000000F07F000000000000000000005043F8
:1066A000645F090000000000000000000000F03FEF
:1066B000763C7935EF39EA3D0000E0FE422EE63FB8
:1066C000E85E000000000000555555555555D53F72
:1066D000000000000000E03F00000000000000405B
:1066E00086EBF9FF6A5D0000605D0000BDEC088B81
:1066F000BDEC08CBFFF72DBEBDEC088BBDEC08CB85
:10670000FFF738BEBDEC088BBDEC08CBFFF7E2BE4F
:1067100070B5414A00252DED020B2DED048BDDE90E
:106720000404944205DA24F00041914201D809D1D1
:1067300040B19DED040BBDEC048B02B0BDE8704090
:1067400000F052BFB4F5801F26DA08430BD0002CAE
:1067500013DA012000F09CFFBDEC048B02B0BDE811
:10676000704000F055BF022000F092FF00F024FFBF
:1067700051EC100B81F0004146E09FED290B6FF0CA
:10678000350553EC102B9DED040B51EC100BFAF773
:106790003BF8CDE904010C4605EB2450A0F2FF3094
:1067A000C10F40F2FF32521A62F31F540844FAF745
:1067B0000FF905949DED040B41EC180B51EC100BF7
:1067C00001F02AFE9FED181B53EC112BFAF71CF871
:1067D0009FED170B41EC190B53EC102B51EC180BE0
:1067E000FAF712F853EC192BF9F75FFF9FED120B34
:1067F00041EC190B53EC102B51EC180BFAF704F881
:1068000053EC192BF9F751FFBDEC048B02B041ECAE
:10681000100B70BD000000000000F07F00000000C1
:1068200000000000000050430EE526157BCBDB3F47
:10683000362BF111F3FE593D00609F501344D33FB6
:106840002DE9F04D2DED040B2DED0E8B96B0DDE90D
:106850002550279CDDF890A025F0004624F0004844
:10686000BAF1000F14BF0121002101EB4502FC49E0
:1068700053184A1093422AD3002814BF012300233F
:1068800003EB44030B44F7498B4220D358EA000141
:106890009FEDF59B76D0DFF8D8B35D4503D1BAF113
:1068A000000F05D188E0BAF1000F08BF002100D029
:1068B000012101EB450111F5001F08D8002814BF84
:1068C0000121002101EB440111F5001F0BD99DEDC1
:1068D000261B9DED240B16B000F0DABD04B0BDE818
:1068E000F04D00F08BBE0027002DBCBFE14988456C
:1068F00021DAE1498845A8BF02271CDAC3451ADC22
:10690000DE4901EB2851142908DDC1F1340220FAD7
:1069100002F101FA02F282420DD108E058B9C1F148
:10692000140228FA02F101FA02F2424503D101F001
:106930000101C1F1020756EA0A0124D1002C22DA32
:10694000002D18BF022F01D0012F0AD0022000F025
:106950009FFE16B000F0A2BD04B0BDE8F04D00F0FF
:106960002BBE022000F094FE00F026FE51EC100B2E
:1069700081F0004141EC100B16B000F095BD04B061
:10698000BDE8F08D18E09FEDBEAB9FEDBF8B0028FA
:1069900071D1B848804522D105F1804010F58010B2
:1069A00008BFBAF1000F07D0B3450ADC002CA8BF1E
:1069B0009DED260BE0DA0DE0B0EE490AF0EE690A33
:1069C000DAE7002C06DA9DED260B51EC100B81F076
:1069D00000416FE0AE48784490ED000BCCE7D8451D
:1069E0004DD1002C48DA2EB186423AD1BAF1000FCF
:1069F00042D126E0BAF1000F13D0022000F048FE89
:106A000000F016FE8DED020B9DED240B8DED000BBD
:106A100010EE900A039961F31E0003909DED020BA6
:106A2000AAE78DED02AB9DED240B1AEE901A10EE45
:106A3000900A8DED000B61F31E0003909DED020B9B
:106A40009AE78DED028B9DED240B18EE901A10EE57
:106A5000900A8DED000B61F31E0003909DED020B7B
:106A60008AE709DA9DED240B51EC190B53EC102B3E
:106A7000F9F73FFF1EE020E09DED240B7CE7864206
:106A80001BDAB4F1804F0DD0A4F10050B0F1FF50EB
:106A900013D1002D11DB9DED240B51EC100B03F0F5
:106AA000F1FF07E09DED240B53EC102B51EC100B84
:106AB00000F0C2BC41EC100B5EE79DED240B51ECE5
:106AC000100B01F024F8BAF1000FCDE90E0142D10C
:106AD0009FED710B46B3A6F1E040B0F17F600CD0A2
:106AE0005E4538D1002D00DAA7B3022F0CBF01207C
:106AF0004FF0FF30F9F76CFFDCE7002D01DD002CD3
:106B00000DDA002D01DD002C1FDB002D16DA002C24
:106B100014DB012F08BF9FED620B3FF42DAFB0EEE9
:106B20004A0AF0EE6A0A27E7022F18BF002D0CD0A0
:106B3000012F0AD1002DFFF61FAF06E0002DB8BFD0
:106B4000002C08DA012F3FF417AFB0EE480AF0EE40
:106B5000680A11E71BE0012000EBE57050EA07012D
:106B600015D0791EB0EE498AF0EE698A084308BF55
:106B70009FED4D8B4E480025804570DD4D494E48B8
:106B8000884514DDB0420DDB002C19DB2FE001201D
:106B900000F07EFD16B000F08DBC04B0BDE8F04DF5
:106BA00000F036BDB34502DC002C09DC1FE0864254
:106BB00002DA002C1BDA03E05E452BDD002C16DD2B
:106BC000022000F065FD00F033FD8DED020B53EC6B
:106BD0001A2B51EC180BF9F717FECDE900010399B8
:106BE000019861F31E0003909DED020BC4E60220A4
:106BF00000F04EFD00F02CFD10EE901A18EE900AF9
:106C00008DED020B8DED008B61F31E0003909DED69
:106C1000020BB1E69DED0E0B53EC192B51EC100B52
:106C2000F9F7E4FD9FED260BCDE9080153EC102B9D
:106C30009DED080B51EC100BF9F7E6FD9FED221BC3
:106C400053EC112BF9F7D5FD9DED081B53EC112BDF
:106C5000F9F7DAFD9FED1E1B53EC112B3CE08CE0A5
:106C6000FFFF1F00FFFF0F00000000000000F03FCB
:106C70000000F03F0000F07F0000404301FCFFFFF8
:106C8000000000000000F07F000000000000000095
:106C90000E5900000000000000000000000000800D
:106CA000000000000000F0FF000000000000F0BF46
:106CB0000000E0410000F043FFFFEF3F0000000054
:106CC000000000000000D03F555555555555D53FA3
:106CD000000000000000E03FF9F78BFD9DED080B80
:106CE00041EC1A0B53EC102B51EC100BF9F78CFD07
:106CF00053EC1A2BF9F788FD41EC1A0B9FEDFE0BB4
:106D000053EC102B9DED080B51EC100BF9F77CFDAB
:106D100041EC1B0B9FEDFA0B51EC1A0B53EC102BB3
:106D2000F9F772FD41EC1A0B9FEDF70B53EC102BAA
:106D30009DED080B51EC100BF9F766FD53EC1A2B87
:106D4000F9F754FD41EC1A0B51EC1B0B53EC1A2BC9
:106D5000F9F7ABFC0690CDE906519DED060B53EC1F
:106D60001B2B51EC100BF9F741FD53EC1A2BF9F7E3
:106D700040FD41EC100B00F0A1B90020B6F5801FDA
:106D80000EDA9FEDE30B53EC102B9DED0E0B51EC47
:106D9000100BF9F739FDCDE90E016FF034000E4606
:106DA00000EB2650A0F2FF37C6F31300DA4940F09B
:106DB0007F6646F040568842D8BF002408DDD74998
:106DC0008142C8BF012403DC0024A6F580167F1C85
:106DD000D348784400EBC4000F9690ED00CB9DEDB6
:106DE0000E0B53EC1C2B51EC100BF9F7FFFC9DED37
:106DF0000E0B41EC1B0B53EC1C2B51EC100BF9F759
:106E000054FC41EC100B51EC190B53EC102BF9F71F
:106E100070FD41EC1D0B51EC1B0B53EC1D2BF9F7D6
:106E2000F3FC41EC1A0BBF488DED10AB7844109584
:106E300090ED000B4FF0005040EA660000EB8440FC
:106E40008DED080B00F5002009909DED080B53EC2B
:106E50001C2B51EC100BF9F7C9FC9DED0E1B53ECEC
:106E6000112BF9F7C6FC41EC100B53EC102B9DEDE8
:106E7000100B51EC100BF9F7C7FC9DED080B41EC22
:106E80001C0B53EC102B9DED100B51EC100BF9F774
:106E9000BBFC53EC1B2BF9F7ACFC53EC1C2BF9F7A8
:106EA000A5FC53EC1D2BF9F7AFFC41EC1C0B53EC8C
:106EB0001A2B51EC1A0BF9F7A7FC41EC1B0B9A4863
:106EC0000621B0EE4B0AF0EE6B0A784400F0F8FAB7
:106ED000B0EE401AF0EE601AB0EE41DAF0EE61DA90
:106EE00053EC1B2B51EC1B0BF9F78EFC53EC1D2BB9
:106EF000F9F78AFC9DED100B41EC1B0B53EC1A2BA0
:106F000051EC100BF9F7D1FB53EC1C2BF9F77CFC7F
:106F100053EC1B2BF9F7C9FB9DED100B41EC1B0B40
:106F200053EC102B51EC100BF9F76EFC41EC1D0BE0
:106F30009FED7FEB53EC1E2BF9F7B7FB53EC1B2BAC
:106F4000F9F7B3FB0890CDE908519DED080B53EC20
:106F50001E2B51EC100BF9F749FC53EC1D2BF9F7E4
:106F600045FC53EC1B2BF9F744FC9DED080B41EC61
:106F70001D0B53EC102B9DED100B51EC100BF9F782
:106F800043FC41EC1B0B53EC1A2B51EC1D0BF9F796
:106F90003BFC9DED080B41EC1A0B53EC102B51EC14
:106FA0001C0BF9F731FC53EC1A2BF9F77EFB41EC83
:106FB0001A0B51EC1B0B53EC1A2BF9F776FB0C90C8
:106FC000CDE90C519DED0C0B53EC1B2B51EC100B30
:106FD000F9F70CFC53EC1A2BF9F70BFC41EC1B0BEB
:106FE0009FED550B53EC102B9DED0C0B51EC100B42
:106FF000F9F70AFC41EC1A0B9FED510B51EC1B0BFE
:1070000053EC102BF9F700FC41EC1B0B9FED4E0BE2
:1070100053EC102B9DED0C0B51EC100BF9F7F4FB1E
:1070200053EC1B2BF9F741FB41EC100B484878441B
:1070300000EBC40090ED001B51EC100B53EC112B36
:10704000F9F733FB41EC1B0B3846F9F7C1FCCDE9EE
:10705000080153EC1B2B51EC1A0BF9F726FB41EC02
:10706000100B3C48784400EBC40090ED00CB51EC91
:10707000100B53EC1C2BF9F718FB9DED081B53EC80
:10708000112BF9F712FB0690CDE906519DED080B87
:1070900053EC102B9DED060B51EC100BF9F7A6FBF2
:1070A00053EC1C2BF9F7A2FB53EC1A2BF9F79EFBC0
:1070B00053EC1B2BF9F79DFB41EC100B9DED261BB0
:1070C00053EC102B8DED001B00959DED260B51EC24
:1070D000100BF9F799FB9DED000B41EC1A0B53ECEB
:1070E000102B9DED260B51EC100BF9F77FFB9DED5E
:1070F000061B53EC112B2FE0000000604715F73FF3
:10710000FE822B654715F73F44DF5DF80BAE543E1A
:1071100000000000000040438E9803007AB60B0088
:1071200052540000B85400008A53000000000000D0
:107130000000000000000840000000E009C7EE3F2A
:10714000FD033ADC09C7EE3FF5015B14E02F3EBEBC
:1071500016520000D0510000F9F756FB53EC1A2BE1
:10716000F9F7A3FA9DED060B41EC1A0B53EC102B2B
:107170009DED000B51EC100BF9F746FBCDE90C012E
:107180009DED0C0B51EC1A0B53EC102BF9F78DFA0B
:10719000CDE902010C46AA498C422FDB611A084353
:1071A00018D19DED0C0B53EC102B9DED020B51EC07
:1071B000100BF9F71BFB41EC1B0B9FEDA30B51ECE4
:1071C0001A0B53EC102BF9F770FA53EC1B2BF9F751
:1071D00029FE2DD2022000F05BFA00F029FA10EE11
:1071E000901A18EE900A8DED020B8DED008B61F375
:1071F0001E0003909DED020BFFF7BEBB944A24F0E6
:107200000041914214D39349214408437FF4EFACE9
:107210009DED0C0B53EC102B9DED020B51EC100B64
:10722000F9F7E4FA53EC1A2BF9F7FCFD7FF6DFAC23
:1072300024F000408849894A002601EB205182420F
:107240002BDA481C4FF4801121FA00F02044844AC4
:10725000C0F30A517A44A1F2FF3192ED000B814A4A
:107260008DED080BCA4020EA0202C0F3130040F47F
:107270008010C1F1140120FA01F60992002CB8BF68
:1072800076429DED080B53EC102B9DED0C0B51EC51
:10729000100BF9F7ABFACDE90C019DED0C0B51EC9D
:1072A0001A0B53EC102BF9F700FA9FED6F0B0890B7
:1072B000CDE9085153EC102B9DED080B51EC100B50
:1072C000F9F7A2FA41EC1B0B9FED690B53EC102B65
:1072D0009DED080B51EC100BF9F796FA9DED0C0B98
:1072E00041EC1C0B53EC102B9DED080B51EC100BDB
:1072F000F9F77CFA53EC1A2BF9F77BFA9FED5E1B3A
:1073000053EC112BF9F780FA53EC1C2BF9F7CDF95C
:1073100041EC1A0B51EC1B0B53EC1A2BF9F7C5F986
:10732000CDE902019DED020B53EC1B2B51EC100B30
:10733000F9F75CFA53EC1A2BF9F75BFA9DED020BA7
:1073400041EC1A0B53EC102B51EC100BF9F75CFAD3
:10735000CDE908014A489DED080B0521784400F06D
:10736000AFF89DED081B51EC100B53EC112BF9F706
:107370004BFA9DED021B53EC112BF9F73AFACDE9CC
:1073800006019DED020B53EC1A2B51EC100BF9F793
:107390003BFA53EC1A2BF9F788F99FED3B0B41ECC4
:1073A0001A0B53EC102B9DED060B51EC100BF9F75B
:1073B0001DFA9DED060B41EC1B0B53EC102B9DEDC4
:1073C000020B51EC100BF9F71FFA53EC1B2BF9F7DA
:1073D00090FA53EC1A2BF9F709FA9DED021B53ECC6
:1073E000112BF9F703FA53EC192BF9F702FACDE94F
:1073F000020101EB065001150029C8BF039015DCFE
:107400009DED020B324651EC100BF9F7F3FCFEF741
:107410005EFF042808BF00F01BF932469DED020B09
:1074200051EC100BF9F7E6FCCDE902019DED020BE2
:1074300051EC180B53EC102BF9F7E6F9FFF73ABBB8
:107440000000904000000000FE822B654715973C2D
:1074500000CC904000346F3F01FCFFFF0000E03F94
:1074600090500000FFFF0F0000000000432EE63F99
:10747000396CA80C615C20BEEF39FAFE422EE63F63
:10748000284F000000000000000000000000004045
:10749000BDEC088BBDEC06CBFFF720BABDEC088B2A
:1074A000BDEC06CBFFF758BABDEC088BBDEC06CBA4
:1074B000FFF765BABDEC088BBDEC06CBFFF76DBBE3
:1074C00070B504462DED028B4D1E00EBC500B0EEED
:1074D000408AF0EE608A90ED000B35F0060017D080
:1074E00053EC182B51EC100BF9F78EF941EC100B03
:1074F0006D1E04EBC50090ED001B51EC100B53EC1E
:10750000112BF9F7D2F841EC100B35F00600E7D15A
:10751000022D36D0042D1CD0062D1CBFBDEC028BD5
:1075200070BD53EC182B51EC100BF9F76DF994ED7D
:107530000A1B53EC112BF9F7B8F853EC182BF9F799
:1075400063F994ED081B53EC112BF9F7AEF841ECFD
:10755000100B53EC182B51EC100BF9F755F994ED77
:10756000061B53EC112BF9F7A0F853EC182BF9F785
:107570004BF994ED040B53EC102BF9F796F841EC12
:10758000100B53EC182B51EC100BF9F73DF994ED5F
:10759000021B53EC112BF9F788F853EC182BF9F771
:1075A00033F994ED001B53EC112BF9F77EF8BDEC89
:1075B000028B41EC100B70BD9FED070B10B553EC27
:1075C000102B9FED070B51EC100BF9F792F941ECE2
:1075D000100B10BD000000000000000000000000C3
:1075E000000000000000F03F10B553EC102B51ECF0
:1075F000100BF9F75AF841EC100B10BD10B553EC15
:10760000112B51EC100BF9F750F841EC100B10BD99
:107610009FED050B10B553EC102B51EC100BF9F747
:1076200068F941EC100B10BD0000000000000000E4
:107630009FED050B10B553EC102B51EC100BF9F727
:10764000E3F841EC100B10BD0000000000000070DA
:107650009FED050B10B553EC102B51EC100BF9F707
:10766000D3F841EC100B10BD00000000000000102A
:1076700002E008C8121F08C1002AFAD170477047FB
:10768000002001E001C1121F002AFBD17047000059
:107690000149086070470000A804002030380A281B
:1076A00001D20120704700207047704708B5044898
:1076B00001226946007802F02BFB9DF8000008BD0E
:1076C000F40B002070B50E4C00231A46247A19469C
:1076D0000A4D04EB840608E005EB4104A48914B1CB
:1076E000521C234492B2491C89B2B1EB460FF3D32A
:1076F000002A02D0B3FBF2F080B270BD5209002024
:10770000800100202DE9F0470027044689460D46F8
:10771000502901D9032000E002208246002600EB18
:107720008A0819E000222949104608E034F8103090
:107730008B4202DB34F910100246401CC0B2A84252
:10774000F4D304EB450104EB4200891E03F0ECF98D
:107750006D1E761CEDB2F6B2B6EB480FE2D3CAF15D
:10776000000000EB800A09EB4A00C5B200261AE0CF
:10777000002247F6FF71104608E034F810308B42C3
:1077800002DC34F910100246401CC0B2A842F4D307
:1077900004EB450104EB4200891E03F0C5F96D1EA0
:1077A000761CEDB2F6B2B6EB480FE1D3002009EB40
:1077B0008A0104E034F81020401C1744C0B2814212
:1077C000F8DC97FBF1F080B2BDE8F0870080FFFFA6
:1077D000084810B5817908484170FE2101700020E9
:1077E000F4F78CF8FDF70EFDBDE810400B210348BF
:1077F000F8F709BEAC050020800200203887002081
:1078000000B587B00E4803F008FA28B10C4803F021
:1078100016FA012000F0D6F80020034600904FF43D
:107820001F72084901A8F3F7D8FB020004D0002317
:10783000044901A8F4F7E4FEFAF7F2F807B000BD36
:1078400088020020DC8800200D48C1794FF4E13027
:10785000062912D2DFE801F00306090C110F4FF4DC
:1078600016500AE04FF4964007E04FF4164004E04B
:107870004FF4614001E04FF4963003F0EDB90000A1
:10788000AC05002070B51B4C2078FF2805D0A4F172
:1078900016018979884200D048BB6078032805D05A
:1078A000062803D0102801D0192820D1124D134EDC
:1078B000688B401C68833079801EC1B20D4800F08F
:1078C00057F8B188214411F8012C11F8021C02EB81
:1078D0000122824203D1AA8B521CAA8302E0EA8BC6
:1078E000521CEA83B1EB102F01D1012070BD0020A2
:1078F00070BD0000C2050020EE080020200000201E
:1079000070B5184C0025A08D642804D1FEF7F0FA5C
:1079100002F028FBA585208D401C80B2A0F56A41AD
:107920002085603903D1FEF7E3FA02F01BFB4FF428
:1079300080514FF09040FBF734FC0B49012801D0F7
:107940004D8170BD4889401C80B24881C828F8D953
:10795000608D401C60854D81FEF7CAFABDE870401D
:1079600002F000BBEE080020800100207047704745
:10797000F0B5FF23094E1C46002206F5807706E08D
:10798000855C521C5D40D2B2735D63407C5D491ED4
:10799000C9B2F5D244EA0320F0BD0000E0BB010803
:1079A000054A5178137841400448405C5840507073
:1079B0000348405C1070704720000020E0BB0108C5
:1079C000E0BC0108064A5168002905D00023814225
:1079D00003D9081A506001D0704753601370704784
:1079E000BC0200200C4810B5C178807801EB002063
:1079F00080B2FFF747FF58B100F03EF9064900207A
:107A000001F0D6FBBDE810400349002000F03CB96E
:107A1000BDE8104002F0A6BAC20500202DE9F047EB
:107A2000314D044628786978EA7800EB0120A9787E
:107A3000090401EB02610844D4F8B41088420FD164
:107A400004F1340114220E462848F8F7E7FC38B157
:107A5000002084F84700142231462448F8F7BAFC85
:107A6000A97994F8C800DFF888900126214FDFF843
:107A7000888081420BD0411EFE2908D2A8713E7039
:107A800088F8010089F8F8000020F3F737FF94F830
:107A9000F80098F8011088420BD050B1FF2808D0A8
:107AA00088F8010089F8F800A8713E700020F3F70B
:107AB00025FFA97994F84900814206D0411EFE298C
:107AC00003D2A8713E7089F84900D4F8CC00D8F8E8
:107AD0000420904206D0002804D0C8F80400F3F730
:107AE0009AFA3E70BDE8F087AC0500203000002017
:107AF0004C870020680100208002002000F034BD87
:107B00000020401C80B20A28FBD37047704782B027
:107B1000CDE9000121F0004001909DED000B02B085
:107B200051EC100B704700000C4910B54FF40040A9
:107B300008610B48FAF724F90A4C60600A48FAF722
:107B40001FF961680123401A401CC4E90203074A77
:107B50000024C2E90210C2E9004310BD0020024027
:107B60000000020868010020FF370208200C0020F6
:107B70000020704740B90B2906D2C1EBC100034970
:107B800000EB40000844704701A07047C8BE0108E0
:107B90006E756C6C00000000F0B5401E4210294C60
:107BA00002EB021204EB42040823228C0026DFF8C9
:107BB00098C08A423DD222888A4235D9082234F8B8
:107BC00012508D4224D804EB420E3EF802EC8E4552
:107BD0001ED3521E04EB420334F812505B88EB1A9A
:107BE00014D0691A6424614391FBF3F102EBC203E0
:107BF00003EB021201EB8201134A283232F9102002
:107C00003CF920004A4392FBF4F1471838B2F0BD2A
:107C100003B9012603EBD3735B108D4201D91A44DB
:107C200000E0D21A002A02DC3CF92000F0BD102A44
:107C300004DB0CEB8000B0F90200F0BD002EBED0DA
:107C40000020F0BD4E000020E0BD010840B90B2926
:107C500006D2C1EBC100034900EB40000844704765
:107C600001A07047C8BE01086E756C6C0000000072
:107C700070475F20704700000248FF21017041708B
:107C800070470000200000202DE9F047C8788A786E
:107C9000012400EB022082B24878F74D06280BD071
:107CA00010287DD1A2F2CB22092A79D8887914280C
:107CB00076D80020F14A5DE3F14B002A71D0022A08
:107CC00070D0062A6FD0072A6ED0082A6DD00F2AEE
:107CD0006CD0102A6BD01E464FF41657F6794FF42D
:107CE000964C4FF416484FF461494FF4E1304FF48D
:107CF000963A0A2A7ED00C2A7DD0112A7CD0122AEC
:107D00007BD0142A7AD0132A79D0632A78D0622AB9
:107D100077D05F2A76D0152A75D0DFF868C3642A39
:107D200072D0DFF86483652A6FD0D848662A6DD098
:107D3000DFF85C93672A6AD0DFF858A3682A67D017
:107D4000DB7B692A7DD06A2A7CD0D34B6B2A7AD020
:107D5000D24E6C2A78D0D24F6D2A76D06E2A75D04A
:107D60006F2A74D0702A73D0712A72D0722A71D09F
:107D7000732A70D0742A6FD0752A6ED0762A6DD08F
:107D8000772A6CD0782A6BD0792A6AD0DFF81483EE
:107D90007A2A67D07B2A66D07C2A65D07D2A07E0C4
:107DA0009FE09AE09FE0A3E0A6E0B0E0B2E0B8E098
:107DB00077D07E2A76D07F2A75D0802A74D0812A07
:107DC00073D0202A72D0512A71D0522A70D0532AEF
:107DD0006FD0542A6ED0552A6DD0582A6CD0592AAB
:107DE0006BD05A2A6AD05B2A69D0232A68D0242A09
:107DF00067D00EE0A6E0BEE0D3E0D7E0DBE0DFE056
:107E0000E4E0E6E0E9E0F0E0F4E0F7E0FAE0FCE0EE
:107E1000FFE00026A44B192A71D0822A70D0832A51
:107E20006FD01D2A6ED0A148392A6CD03A2A6BD067
:107E30003B2A6AD03F2A69D09D4FA2F5007C3B685F
:107E400013E0EAE0F3E0FCE0FEE000E105E108E138
:107E50000BE10DE14CE14FE154E159E15BE15DE102
:107E600062E165E168E16DE170E1BCF1DB0C29D014
:107E7000A2F5007CBCF1DA0C71D05C2A70D05D2ACE
:107E80006FD0A2F2E93008286CD84879097900EB64
:107E90000120884901EB4201A1F58051A1F82E088B
:107EA00028E057E15CE164E166E168E16DE173E1DE
:107EB00078E17DE180E185E18AE18FE194E199E17A
:107EC0009EE1A3E14879097900EB0120B0EB234F53
:107ED00007D0190C09040843EAE1487918700879B9
:107EE0005870BDE8F087487998700879D87001E03B
:107EF000487998712C70F4E748795872FAE78CE168
:107F0000A1E1A6E1ABE1AFE1B4E1B9E1BEE14879BD
:107F10009872EFE748790528E3D8D871FFF794FC09
:107F2000E8E7487918727F28DBD1BFF34F8F6248AA
:107F30000168624A01F4E06111430160BFF34F8FB1
:107F400000BFFDE749790129CBD11973062E25D24F
:107F5000DFE806F003090B0D240F38461EE09BE115
:107F6000ACE1B1E1EEE1604618E0404616E048467B
:107F700014E0504612E049790229B2D81A7D8A42AB
:107F8000AFD01975062E09D2DFE806F00706050402
:107F90000803EEE7EBE7E8E7E5E7DEE702F05CFE83
:107FA000A8E7487902289CD2454914E04879082876
:107FB00097D244490FE04879042892D242490AE016
:107FC0004879411E09298CD8404904E04879404944
:107FD00001E048793F4908708CE748793E4901281B
:107FE000087087D115223DA122E14879012893D854
:107FF000D8737FE748798CF800007BE7487988F8E8
:10800000000077E74979017074E7497989F8001031
:1080100070E749798AF800106CE748790979012BF3
:1080200000EB012001D02E49F5E02E49F3E048791C
:108030000979012B00EB012001D02B49EBE02B4902
:10804000E9E04879187055E74879307052E7487987
:10805000097900EB0120388043E748798CF801006A
:1080600048E7487988F8010044E74979417041E7D9
:10807000497989F801103DE76801002030000020AF
:10808000AC0500203E0100204101002044010020F9
:10809000470100204A010020590100205C01002016
:1080A00060010020EE080020200100209010002038
:1080B000840200207C1000200CED00E00400FA0592
:1080C0007C0100207D0100207E010020880100202D
:1080D0008101002082010020870100204C4F5400C4
:1080E0002A0100202E0100202C0100203001002058
:1080F00049798AF80110FDE64879097900EB0120F9
:108100009E4988E04879097900EB01209C4982E08A
:1081100048795870EEE648797070EBE6487909794D
:1081200000EB01207880DCE648798CF80200E1E67B
:10813000487988F80200DDE6497981703731A8F87E
:108140005A10D7E6497989F80210D3E649798AF8B6
:108150000210CFE64879097900EB012089495AE0FD
:108160004879097900EB012087490880A8F8520076
:10817000C0E648799870BDE64879B070BAE64879AB
:10818000097900EB0120B880ABE64879097900EB6A
:1081900001207E490880A4E64879097900EB012096
:1081A0007B4938E04879097900EB0120794932E0D0
:1081B00048797949087094E64879097900EB0120FB
:1081C000764928E04879097900EB0120744922E0DA
:1081D0004879097900EB012072491CE04879097956
:1081E00000EB0120704916E04879097900EB012085
:1081F0006E4910E04879097900EB01206C490AE0EA
:108200004879097900EB01206A4904E04879097945
:1082100000EB0120684908806CE64879674901282D
:108220000BD00028B0D1CE701E705C70152264A1F6
:1082300062481030F8F7CEF85CE6CC70F9F7DCFB5A
:10824000152263A1F4E748791870022890D91E70AE
:1082500050E64879587002288AD95E704AE6487913
:108260005F4981F8960145E64A79097902EB0121D7
:1082700001803FE64A79097902EB0121418039E624
:108280004A79097902EB0121017333E64A790979C8
:1082900002EB012101712DE64879097900EB0122F9
:1082A000B2EB134F87D0000400EB016099B2084491
:1082B00038602C70BDE8F047F2F7ADBE497901296E
:1082C0003FF619AE817315E6464B91F805C01A8842
:1082D00059881F79DB7BBCF1010FF1D818D1002B35
:1082E000A0D14FF0640302FB03F24FF0FE03B2FB98
:1082F000F3F202804FF0640201FB02F1B1FBF3F1F3
:10830000418017FB02F1B1FBF3F10171C473F1E598
:10831000BCF1000F86D1012B84D1C2EBC2125300F5
:108320006422C1EBC111B3FBF2F34900B1FBF2F1DE
:1083300003804180C7EBC7114900B1FBF2F1017125
:10834000C673D7E5A2F222302F28B9D84879097927
:1083500000EB012008EB4201A1F58051A1F8C00912
:10836000A2F54070333884D0BBE50B18DB79135489
:10837000401CC0B28B798342F7D8BBE536010020A0
:108380003801002022010020240100201A010020D1
:1083900004010020060100205F01002008010020E8
:1083A0000A0100200C0100200E0100201001002015
:1083B000120100209E010020A001002020000020CA
:1083C0005472616E64756365722D534854000000E9
:1083D0005472616E64756365722D434F3200000004
:1083E000400C00209010002030B585B04FF40044C0
:1083F0000120CDE900400020029002204FF090457E
:10840000039069462846FAF70FFE002221462846C7
:10841000FAF7D3FE05B030BD10B541EC100BFDF7F7
:1084200083FF51EC100B10BD09480168C1F34042B5
:1084300001680068C1F34061C0F34003054864323D
:10844000643120F8522F64334180838070470000EC
:1084500000100240EE080020394994B03748086007
:10846000FBF7C4F964213748F7F7CDFFFDF7A4FA0D
:10847000FFF7BAFFFFF758FB00F0C2F8FDF738FD31
:10848000314C20782F49A1F85000F9F7FDF902F09E
:1084900051FBF9F75FFBFFF79BF94FF4165002F021
:1084A00029FC2B48294901600021416040F6FF71F9
:1084B000C1608160FBF75EF908B1F9F7A7FBE079CD
:1084C000012806D02348007840B10220FCF772FD55
:1084D00006E00220FCF76EFD0420F7E7FCF7E8FB5E
:1084E00014221D496846F7F775FF0021684600F021
:1084F00047F8194920641422143105A8F7F76AFFD8
:10850000002105A800F03CF81349606414222831CA
:108510000AA8F7F75FFF00210AA800F031F80E491A
:10852000A06414223C310FA8F7F754FF00210FA8D4
:1085300000F026F8E06400F01EF8FEE70080000876
:1085400008ED00E0EE08002080010020003000402F
:10855000300C00202300002030BE0108014600201E
:10856000842900D0C81C704710B500B9012002F062
:10857000D1FE002010BD10B502F0F2FE002010BDAB
:108580003EB504460D46B0F90800FFF7E7FF02A923
:10859000CDE90001208A2B4682B2D4E9001003F015
:1085A0001FFA012801D000203EBD02983EBD0246C0
:1085B000B020082900D1B820082A18D008DC012AE8
:1085C0000FD0022A10D0042A01D140F005007047D4
:1085D000102A0FD0202A10D0402AF8D140F00100F4
:1085E000704740F00700704740F00600704740F0C9
:1085F0000400704740F00300704740F002007047ED
:108600002DE9F05FFE48002707704FF42A70FDF750
:1086100069F9FC4E401CFC4DF08401242C700020B4
:10862000FDF760F9411C02D14FF001102C70DFF80A
:10863000DC83020A88F8000088F80120020C88F820
:108640000220000E88F803001020FDF74BF9411CB2
:108650000DD01421B18188F806005A2088F809004D
:1086600046462020FDF73EF9411C05D006E00A20D1
:10867000B081FE202C70EEE702202C70B07230200A
:10868000FDF730F9012802D008B100202C703073BA
:108690004FF42270FDF726F9022801D900202C7032
:1086A0003075B1467820FDF71DF9022803D389F80B
:1086B0000E702C7001E089F80E002820FDF712F9E9
:1086C000052804D9042189F807102C7001E089F8E5
:1086D00007003820FDF706F9CD49421C40F6BD568B
:1086E0003CD008804020FDF7FDF8CA49421C4FF4F9
:1086F000AE7836D008804820FDF7F4F8C649421C11
:1087000033D008805020FDF7EDF8C449421C2FD02B
:1087100008805820FDF7E6F8C149421C2CD008809B
:108720006020FDF7DFF8BF49421C2AD0088068208E
:10873000FDF7D8F8BC49421C28D008807020FDF70E
:10874000D1F8BA49421C26D008808020FDF7CAF82B
:10875000B749022824D30C702C7022E00E802C70B4
:10876000C0E7A1F800802C70C5E70E802C70C9E727
:10877000A1F800802C70CCE740F62E1008802C70F9
:10878000CEE74FF4D17008802C70D0E740F6A610E9
:1087900008802C70D2E74FF4E17008802C70D4E789
:1087A00008708820FDF79EF8A249082802D30F70B0
:1087B0002C7000E008709020FDF794F89E49042882
:1087C00002D30C702C7000E008704FF49C70FDF721
:1087D00089F8DFF86882411C16D0A8F81E004FF413
:1087E000A070FDF77FF8411C12D0A8F82000DFF838
:1087F00050B200264FF0980A0AEBC600FDF772F857
:108800007F2809D92C7009E0A8F81E702C70E6E7C3
:10881000A8F820702C70EAE70BF80600761C142EDE
:10882000EAD3DFF820A200264FF4E07B0BEBC60072
:10883000FDF758F8B0F57A7F06D9834830F816105E
:108840002AF816102C7001E02AF81600761C092E62
:10885000ECD34FF4A470FDF745F87C49421C02D0DC
:10886000B0F5800F10D399F8002099F8013099F8ED
:10887000030002EB032299F802301B0403EB0060B3
:10888000104408602C7000E008604FF4A870FDF7F9
:1088900029F8022803D389F80F702C7001E089F8B9
:1088A0000F004FF4B070FDF71DF8411C02D008B165
:1088B0000A2804D9052188F808102C7001E088F8EE
:1088C00008004FF4B470FDF70DF86149DFF88491AA
:1088D000421C13D0C20719D00C70C0F3072189F8CD
:1088E0000010C0F307404A4689F80100022900D968
:1088F000177002280FD989F801700CE00C7089F804
:108900000070022189F801102C7004E00F7089F8C2
:10891000007089F801404FF4B870FCF7E3FF4E494E
:108920003C2809D0142807D01E2805D020B13C20AF
:1089300081F896012C7001E081F896014FF4BC702B
:10894000FCF7D0FF454E411C56D030804FF4C0702C
:10895000FCF7C8FF411C50D070804FF4C470FCF786
:10896000C1FF411C4AD030734FF4C870FCF7BAFF06
:10897000411C44D030714FF40270FCF7B3FF411C2E
:108980007AD0B0734FF40470FCF7ACFF411C74D084
:10899000F0734FF41270FCF7A5FF314E411C6DD0FF
:1089A00030704FF40670FCF79DFFDFF8B8B0411C43
:1089B0007ED08BF800004FF40870FCF793FF411C49
:1089C00077D0294908704FF40A70FCF78BFF411CDF
:1089D00070D0264908704FF40C70FCF783FFDFF865
:1089E00090A0411C67D08AF800004FF40E70FCF78D
:1089F00079FF411C1F4A42E004E106E108E10CE175
:108A000022000020EE08002068010020AC050020B4
:108A10000401002006010020080100200A010020B6
:108A20000C0100200E010020100100201201002086
:108A30007C0100207D0100207E01002080010020BB
:108A4000300000207C1000201CBE010884020020A1
:108A50002300002020010020400C00209010002066
:108A60003E01002041010020440100204701002078
:108A70004A0100202A010020D2E0D4E0D6E07CD0D8
:108A800099F80130022B79D099F80010022975D09D
:108A900010804FF41070FCF725FFB24A411C6ED0D5
:108AA00099F80130022B6BD099F80010022903E0ED
:108AB000BFE0C5E0C9E0CDE062D010804FF4267081
:108AC000FCF710FFA849421C7ED008804FF42870A4
:108AD000FCF708FFA549421C77D008804FF42070AE
:108AE000FCF700FF411C71D070704FF41470FCF75C
:108AF000F9FE411C6BD08BF801004FF41670FCF7A7
:108B0000F1FE411C7BD09A4948704FF41870FCF775
:108B1000E9FE411C74D0974948704FF41A70FCF775
:108B2000E1FE411C6DD08AF801004FF41C70FCF787
:108B3000D9FE9149421C6ED008804FF41E70FCF79C
:108B4000D1FE8E49421C67D008804FF43A70FCF782
:108B5000C9FE411C72D0B0704FF42E70FCF7C2FEFB
:108B6000411C6CD08BF802004FF43070FCF7BAFE59
:108B7000411C6ED07E49887003E070E07FE081E0A8
:108B800094E04FF43270FCF7ADFE411C72D079498D
:108B900088704FF43470FCF7A5FE411C6BD08AF846
:108BA00002004FF43670FCF79DFE411C77D07449EB
:108BB00008804FF43870FCF795FE411C70D0714965
:108BC00008804FF4247003E073E079E07DE07FE0FB
:108BD000FCF788FE411C71D088F801004FF42C701E
:108BE000FCF780FE411C6AD088F802000820FCF7E0
:108BF00079FE411C71D088F8070000F0C5B86DE01F
:108C000071E074E037802C70A0E677802C70A4E6C9
:108C100037732C70A8E66FE071E037712C70AAE60C
:108C2000B7732C70AEE6F7732C70B2E637702C7009
:108C3000B7E628218BF800102C70BCE664E066E0F3
:108C40004B49C82008702C70BDE64A4807702C704C
:108C5000C1E661E064208AF800002C70C5E699F84E
:108C60000110022908D099F80000022804D01780CA
:108C70002C700EE755E058E041480780F8E740497E
:108C8000088006E799F8011002290AD099F8000037
:108C9000022806D04FF47A7010802C700EE749E05D
:108CA0004CE038484FF4FA610180F6E73549088016
:108CB00004E74FF6706008802C7007E744E048E056
:108CC0004FF4AF6008802C7008E777702C700CE7C9
:108CD00028218BF801102C700FE73FE02449C820B1
:108CE00048702C7011E7234847702C7015E76420FA
:108CF0008AF801002C7018E70F802C701DE74FF4E4
:108D00007A7008802C7020E7B7702C7024E7282137
:108D10008BF802102C7027E71549C82088702C703A
:108D20002AE7144887702C7033E764218AF8021010
:108D30002C7036E7124807802C703AE711484FF440
:108D4000FA6101802C703CE7022088F801002C7049
:108D500044E7032188F802102C7047E788F8077071
:108D60002C704AE72C0100202E0100203001002049
:108D70004401002047010020360100203801002076
:108D8000220100202401002030BCBDE8C09F00006B
:108D90002DE9F041184E0F46044675693068001DF4
:108DA00001F0D4FF38B9306890F82C1001208840C9
:108DB000B1698143B161601C07D137B13168BDE849
:108DC000F0410E48091D02F069B830682C44AC42ED
:108DD0004460316805D2B068BDE8F041091D02F079
:108DE00045B87068091D02F041F8306B844200D22A
:108DF0003463BDE8F0810000200200207C110020D7
:108E00002DE9F041054602F011FA2E4E3069401C62
:108E1000306130682C4F10B1F06940B32DE03560FF
:108E20003069012829D1002404EB840007EB80007D
:108E300002F00EF8641C072CF6D323488C3002F0A5
:108E400007F82148A03002F003F81F48B43001F0C1
:108E5000FFFF1D48C83001F0FBFF1B48DC3001F06C
:108E6000F7FF19488C3070601430B06005E030684E
:108E7000E96AC06A884200D83560F06A0121401C66
:108E8000F062E86AB26981401143B16100EB800091
:108E900007EB8000291D02F001F802F0E7F9F06904
:108EA00000280CD03068E96AC06A884207D20749B6
:108EB0004FF080500860BFF34F8FBFF36F8FBDE856
:108EC000F081000020020020A010002004ED00E04E
:108ED00010B50446006B02F0DDF92046BDE81040F5
:108EE00002F0D8B90F4847F23051420705D0C01DF3
:108EF0000C4A20F00700821A891A0B4A0023014409
:108F0000C2E900030839103A21F0070111604B60F3
:108F10000B600B1AC0E9001393604FF000405360E0
:108F2000D0607047901100206C020020134E144D49
:108F3000A6F1C8074FF08058DFF8489011E002F022
:108F400075F9F068C468201D01F000FF2869401E13
:108F50002861E868401EE86002F088F92046FFF7C3
:108F6000B7FFE8680028EAD138680128F9D9C9F8BC
:108F70000080BFF34F8FBFF36F8FF2E768110020BF
:108F80002002002004ED00E02DE9F0479A46DDE9DB
:108F9000098481466FF00303206B03EB82021044C7
:108FA000089D20F00706700707D0502080F3118835
:108FB000BFF34F8FBFF36F8FFEE723180A5C83F870
:108FC00034200A5C12B1401C1028F6D3002784F824
:108FD0004370072D00D30625E562C4E91157201D13
:108FE00001F041FF04F1180001F03DFF2461C5F1DB
:108FF00007006462A061E76484F8507052464946F5
:10900000304600F0BFF82060B8F1000F01D0C8F87A
:109010000040BDE8F087000030B5114900E011467E
:109020000A688242FBD34B685C18844203D14068D3
:1090300018444860084643681C18944209D1084CFB
:10904000103C2468A24209D052681A4442600A685F
:1090500012680260814200D0086030BD0460F9E708
:109060006C02002006484168096829B14168C96856
:10907000C9684968016370474FF0FF31FAE70000A3
:109080002002002008484068401C4FF0500080F348
:10909000118804D0BFF34F8FBFF36F8FFEE7BFF38C
:1090A0004F8FBFF36F8FFEE7740200202DE9F04170
:1090B0000546002602F088F9314F386808B9FFF7F5
:1090C00011FFF86805424BD1C5B3083568070ED0CB
:1090D00005F00700C0F108000544680707D05020DC
:1090E00080F31188BFF34F8FBFF36F8FFEE72DB36F
:1090F0007868854234D8224910310846046801E076
:10910000214604466068A84202D220680028F7D1B0
:109110003868844224D00E68206808606068083689
:10912000411B10290FD96019420708D0502080F345
:109130001188BFF34F8FBFF36F8FFEE710E04160E0
:109140006560FFF769FF61687868401A7860BA68FF
:10915000904200D2B860F86801430020C4E90001E1
:1091600002F0D0FC700707D0502080F31188BFF3C5
:109170004F8FBFF36F8FFEE73046BDE8F0810000F0
:109180005C02002010B5031F4FF080741C601B1F91
:1091900021F001011960191F044B0B6014390A609A
:1091A000091F6FF0020244380A6010BD8590010863
:1091B0002DE9F34F0E46C878897883B000EB012083
:1091C00080B2009070780025DFF83094062839D0FE
:1091D000102837D0A9F21628032854D019286ED1A8
:1091E00030784C4689F80000FEF7DAFB7078607042
:1091F000FEF7D6FB98F806004546A070FEF7D0FBB8
:109200002878E070FEF7CCFB68782071FEF7C8FB89
:10921000A8786071FEF7C4FBE878A071FEF7C0FB88
:10922000F7494878E07108782072A879B1788842C7
:1092300045D8F178884242D3092005B000F046BCF9
:10924000FDF72EB800244F46305D78556D1CADB249
:10925000305DFEF7A5FB641CE4B2062CF4D3E84AAB
:10926000507878556D1CA8B212783A54401C039A75
:1092700080B2042A03D0002A21D1C0B2DDE7707980
:109280004200F91C38E270790190317889F80010B9
:10929000DA4970780324487070794000887030781B
:1092A000FEF77EFB7078FEF77BFB70794006000EC0
:1092B000FEF776FB4FF0000AD24F4D4608E290E3EE
:1092C0000098504481B2032903D8002018F80120E7
:1092D00024E204297ED006297DD007297CD00829E4
:1092E0007BD00A297AD00C2979D00F2978D010297F
:1092F00077D0112976D0122975D0132974D014296A
:1093000073D0152972D05F2971D0632970D062297A
:109310006FD018296ED01C296DD019296CD08229E4
:109320006BD083296AD01D2969D01E2968D01F29D6
:1093300067D0202966D021297ED04A297DD03829BE
:109340007CD039297BD03A297AD03B2979D03C2965
:1093500078D03D2977D03E2976D03F2975D05C2939
:1093600074D05D2973D0232972D0242971D0252986
:1093700070D026296FD022296ED027296DD04B2995
:109380006CD04C296BD04D296AD04E2969D04F2919
:1093900068D0282967D0292966D02A2965D02C29A8
:1093A0006FD030296ED031296DD02B296CD02D296A
:1093B0006BD02E296AD02F2969D0512968D0522923
:1093C00067D0532971D0582970D059296FD05A29A4
:1093D0006ED018E05EE060E063E06AE06DE070E0AF
:1093E00073E076E079E07BE07DE083E085E088E093
:1093F0008AE08EE090E091E092E095E098E09AE0DB
:109400009EE09FE0A0E05B2970D054296FD05529E1
:109410006ED0A1F50070DA382DD0A1F50070DB38E0
:1094200067D0A1F50070CA3871D0401E09286FD8E6
:10943000734A81B2103219E08BE09DE0A0E0A1E018
:10944000A2E0A3E0A6E0A9E0ABE0ADE0B0E0B3E0CD
:10945000B6E0B8E0B9E0BCE002E105E10AE10BE109
:109460000CE10FE14EE155E15AE15BE112F8110028
:1094700002EB41015CE264480168080EC1F3074257
:109480004CE151E152E153E154E155E15CE15DE130
:109490005EE15FE10020302240E1002098F80620E4
:1094A0003CE1002098F8092038E157E159E15AE100
:1094B0005BE1002098F80A2030E1002098F80C20A9
:1094C0002CE1002098F8142028E1002098F80720CB
:1094D00024E1002098F8082020E100204B4925E0F5
:1094E00000204B4922E000204A491FE03FE140E1D3
:1094F00041E142E10020484918E0002098F80F209F
:109500000CE10020454911E0002045490EE036E11C
:1095100038E10020434909E0434816E0434814E09D
:1095200037490020CA78F9E0414900200A78F5E07F
:1095300000203F49FCE13F49002091F89621EDE0F1
:109540003D4802E03D4800E03D48018804E1CAB2E0
:10955000E4E02B48C07808B13A4817E23A49087865
:10956000D1E12855641CA1B205F80190491C8CB2C8
:10957000FEF716FA4846A5E03248B0F80C11EBE0C9
:1095800032481EE03248E0E73148D4E1304900205B
:109590000A7BC3E02E4900204A7BBFE02C4881684B
:1095A0006BE72B480189B2E0294900200A79B5E030
:1095B000274900208A7BB1E025490020CA7BADE025
:1095C00024480188A3E02448FBE724480188214877
:1095D0004DE02248B0F90000F8F7B3FADFF874B0B4
:1095E000BBF800100844C0F307291C48B0F900007C
:1095F000F8F7A7FA9BF80010084455E0C2070020CE
:10960000200000203E010020840200207C01002078
:109610007D010020880100207E01002087010020BC
:109620008101002082010020980100209C0100207F
:1096300020010020400C0020180100201E01002005
:109640001A01002052090020D80D0020D601002068
:10965000901000209E010020A00100208E0100201B
:10966000E148B0F8921152E0E0480188E0480088F3
:1096700001444CE0DF48A4E7DF48A2E7DF48018867
:10968000DC4842E0DFF874B3BBF90000F8F759FAA0
:10969000D8490988401AC0F30729BBF90000F8F738
:1096A00050FAD4490978401A05F8049000F0FF0BED
:1096B000641CA0B205F800B0401C84B24846FEF716
:1096C0006FF95846FEF76CF90AF1010000F0FF0A45
:1096D00001998A45FFF4F4ADC949487809782855BD
:1096E000641CA0B22954401C039980B204297FF461
:1096F000C4AD70794200E91C05B0C24800F0EBB976
:10970000F6F768BEC0480188BB480088091AC1F353
:1097100007201CE7B448B0F894111DE0914620E7FB
:10972000BA484EE7BA484CE7BA484AE7BA4848E769
:10973000BA4846E7BA4844E7BA480078012801D059
:10974000B94890E0B94821E1B848F4E0B7482BE1C6
:10975000B748FAE6B748F8E6080AF8E60020B6493E
:10976000E4E6B648F1E6B648EFE6B648EDE6B648B8
:10977000EBE6B648E9E6B648E7E6B64821E700205A
:109780005622CBE7642945D0652946D066294DD0BD
:10979000672952D0682957D069295DD06A296AD0D3
:1097A0006B297ED06C297FD06D296ED06E296DD04B
:1097B0006F296CD070296BD071296AD0722969D059
:1097C000732968D0742967D0752970D076296FD035
:1097D00077296ED078296DD079296CD07A296BD011
:1097E0007B296AD07C2969D07D2968D07E2967D001
:1097F0007F2970D080296FD081296ED0A1F2E93005
:1098000008286BD8944800EB4100A0F58050B0F8D0
:109810002E18A1E700203A7880E73978002009B1B6
:109820008E4915E08E4913E089469AE63978002082
:1098300009B18C490CE08C490AE03978002009B163
:109840008A4905E08A4903E03978002011B1894945
:109850000978E9E78849FBE7387840B198F80F00C4
:10986000012806D085480188C1F3072090E084488C
:10987000F9E78448F7E7387878B198F80F000128BD
:109880000DD08148EFE70CE00EE01AE01BE01DE090
:1098900027E02DE033E03AE03FE07C48E3E77C4816
:1098A000E1E700207B4941E600207B493EE63AE0C3
:1098B0003CE03FE041E043E049E04FE055E05CE060
:1098C00061E0764841E600207A7827E77978002041
:1098D00029B1624917E05FE061E064E066E0604959
:1098E00011E07978002009B15E490CE05E490AE098
:1098F0007978002009B15D4905E05D4903E0797898
:10990000002011B15B4949788EE75B49FBE7787825
:1099100008B16348A7E76348A5E7787808B16248CB
:10992000A1E762489FE700205A4901E05A49002018
:109930004A78F3E6594841880EE70020BA78EDE608
:10994000B978002009B1454913E0454911E0B978DB
:10995000002009B143490CE043490AE0B9780020EE
:1099600009B1424905E0424903E0B978002011B14C
:109970004049897858E74049FBE7B87808B14C4836
:1099800004E04C4802E0B87820B14B480188080A4E
:10999000C9B249E74948F9E700203E4901E03E499C
:1099A00000208A78BAE63D488188D5E6B1F5487F3F
:1099B00011D0A1F5407021380AD0401E30280DD8B2
:1099C0003F4800EB4100A0F58050B0F8C019C3E655
:1099D00000203C49AAE500203B49A7E500200246BB
:1099E0009CE605B000F07CB8400C00208C01002003
:1099F000A0010020E8010020EA010020E001002091
:109A000020000020588B0020DE0100209001002063
:109A10009201002094010020E2010020E4010020D6
:109A2000E60100208701002096010020D8010020D7
:109A300004010020060100205F0100200C0100202D
:109A40000E0100201001002012010020080100205A
:109A50000A010020840200207C1000204101002027
:109A60004D0100204401002050010020470100204A
:109A7000530100204A010020560100202A01002045
:109A8000320100202E0100202C0100203401002092
:109A900030010020590100205C01002060010020FD
:109AA000360100203A010020380100203C0100204E
:109AB000220100202601002024010020280100208E
:109AC000EE080020030000200200002030BCBDE8AA
:109AD000C04FFFF7B5BB30BCBDE8C04FFFF710BEAD
:109AE00030BCBDE8C08F00002DE9F05F904689468C
:109AF000074603B97B681B4E1B48B6FBF3F50168AC
:109B000041F080710160194C00206060206840F0D5
:109B1000010020604FF4805A4FF0904B01225146D3
:109B20005846F9F74AFB4FF47A734246494638469D
:109B3000FAF7DCFF3868C1694906FCD50C4805EB2B
:109B400045010068B0FBF6F0484361686268521A4C
:109B50008242FBD35146584600F00CB80022F9F778
:109B60002CBB000040420F00FCED00E0001000E0C4
:109B70001C02002030BCBDE8C05FFFF7EFBF70479C
:109B80007CB514460D4601AA694600F017F8002876
:109B900010D1BDF8000045F273514843064901EB6E
:109BA00050302860BDF8040043F2D4014843400B14
:109BB000206000207CBD00003850FFFFFEB5144639
:109BC0000D46064600214EF60542684600F075F83F
:109BD00002466946622000F06FF9002818D14FF460
:109BE0007A7000F0B8F906226946622000F0F0F8B9
:109BF00000280DD1684600F05DF830806E46B01C3C
